:100000006DC700009CC700009AC7000098C7000099
:1000100096C7000094C7000092C7000090C7000078
:100020008EC700008CC700008AC7000088C7000088
:1000300086C700000C94C14D82C7000080C7000035
:100040007EC700007CC700007AC7000078C70000A8
:1000500076C7000074C7000072C700000C94BE4948
:100060006EC700000C94935C0C946A5C68C7000037
:1000700066C7000064C7000062C7000060C70000D8
:100080005EC700005CC700005AC7000058C70000E8
:1000900056C7000054C7000052C700000C94D95046
:1000A0004EC700004CC700004AC7000048C7000008
:1000B00046C7000044C7000042C7000040C7000018
:1000C0003EC700003CC700003AC700000C94415CEA
:1000D0000C94185C34C700000C94EF5B0C94C65B66
:1000E0002EC700001832FA311F321F321F321F3262
:1000F0001F321F321F321F321F321F32C11F3021E9
:100100009A23A223AA23B22369257826F02606275C
:100110000A271F321D274F29432A482BBF2CF42DB5
:10012000542E302FAC2F0E3016311F321F321F329B
:100130001F321F321F321F321F321F321F32513106
:100140001F321F321F321F321F321F324D325C5896
:100150005F584E58525858589658635867586D58BB
:10016000715875587B587F588358965889588D58C0
:100170009158084AD73B3BCE016E84BCBFFDC12FCE
:100180003D6C74319ABD56833DDA3D00C77F11BE88
:10019000D9E4BB4C3E916BAAAABE000000803F0789
:1001A000634236B79BD8A71A39685618AEBAAB5512
:1001B0008C1D3CB7CC5763BD6DEDFD753EF61772D7
:1001C00031BF000000803F08000000BE92244912A9
:1001D0003EABAAAA2ABECDCCCC4C3E00000080BECD
:1001E000ABAAAAAA3E00000000BF000000803F00AA
:1001F00000000000084178D3BB4387D1133D190E9E
:100200003CC3BD4282AD2B3E68EC8276BED98FE105
:10021000A93E4C80EFFFBE01C4FF7F3F00000000FD
:1002200000004E414E494E495459494E46CDCCCC22
:100230003D0AD7233C17B7D13877CC2B329595E6BA
:10024000241FB14F0A000020410000C84200401C9A
:100250004620BCBE4CCA1B0E5AAEC59D7400407AE7
:1002600010F35A00A0724E18090010A5D4E800003F
:10027000E87648170000E40B54020000CA9A3B00DD
:100280000000E1F505000080969800000040420F54
:10029000000000A08601000000102700000000E818
:1002A00003000000006400000000000A00000000DD
:1002B000000100000000002C76D888DC674F08237E
:1002C000DFC1DFAE59E1B1B796E5E3E453C63AE6E4
:1002D00051997696E8E6C28426EB898C9B62ED40C4
:1002E0007C6FFCEFBC9C9F40F2BAA56FA5F4900513
:1002F0005A2AF75C936B6CF9676DC11BFCE0E40D47
:1003000047FEF520E6B500D0ED902E03009435773A
:10031000050080841E080000204E0A000000C80C62
:10032000333333330F986E12831141EF8D211489CB
:100330003BE65516CFFEE6DB18D1844B381BF77C25
:100340001D901DA4BBE424203284725E228100C96A
:10035000F124ECA1E53D2723616E6F74686572207E
:10036000495220696E7075743D0023696E70757412
:100370002044535463616C6962726174653A002071
:10038000766F6C746167653D0023547572626964B1
:10039000697479205570706572204C696D69743A82
:1003A000200020766F6C746167653D0023434F32F7
:1003B000207A65726F20766F6C74202800234F328C
:1003C0002063616C6962726174696F6E3A20002308
:1003D000547572626964697479204C6F7765722014
:1003E0004C696D69742056313A2000235061726166
:1003F0006D6574657273004E6F20445320546865B8
:10040000726D6F6D657465722100234E6F20736588
:100410006E736F7220666F7220504D21004E6F20F8
:1004200073656E736F722100504D313A322E353A3A
:100430003130004D6561737572696E672E2E005400
:10044000757262696469747900233A53686F772F13
:1004500048696465204C4344002A3A546869732013
:1004600048656C700044433A436C656172204C43AC
:10047000440044423A5265736574204C6F67676567
:10048000720044373A4D6F74696F6E0044363A44D7
:10049000532054656D700044353A555620496E74AA
:1004A000656E736974790044343A4F3220636F6E1D
:1004B000632E0044333A434F3220636F6E632E0045
:1004C00044323A504D28313A322E353A31302900F3
:1004D00044323A504D28313A322E353A3130292AB9
:1004E0000044313A54757262696469747900443029
:1004F0003A566F6C7461676500393A6F7220334405
:1005000020616363656C2E00393A496E636C2E205E
:10051000616E672E00383A70482076616C75650010
:10052000373A49522054656D7000373A4952205489
:10053000656D702A00363A4D61676E657469632097
:100540006669656C6400353A476173204C65766571
:100550006C00343A495220466C616D6500333A4C68
:100560006967687420496E742E00323A616E6420A7
:1005700048656967687400323A54656D702050723E
:1005800065737375726500313A54656D70204875F6
:100590006D696469747900303A536F756E64204CEC
:1005A0006576656C00303A536F756E64204C6576E5
:1005B000656C2A00234E6F2073656E736F72206620
:1005C0006F722074656D7020262068756D6964698E
:1005D000747921004E6F2053656E736F7221002372
:1005E00057726F6E672073656E736F7220666F72DD
:1005F0002074656D7020262068756D696469747952
:10060000210057726F6E672053656E736F72210001
:1006100054656D702048756D6964697479004C6922
:1006200067687420496E74656E7369747900466CEE
:10063000616D65204952004E6F2073656E736F7255
:10064000210049522054656D706572617475726540
:10065000004D6561737572696E672E2E00704820BB
:1006600076616C756500496E76616C6964206B65B6
:10067000792100237265706C6965733D006765744C
:1006800053656C665465737442697428293A200076
:100690006973496E74657272757074456E61626CCF
:1006A00065642831293A2000676574496E74657263
:1006B000727570744D617070696E672831293A20C7
:1006C00000676574496E74657272757074536F75E6
:1006D0007263652831293A2000676574496E746534
:1006E0007272757074536F7572636528293A2000B1
:1006F0006765745261746528293A20332E3134318C
:1007000035393F00616363656C2E69734C6F7750B8
:100710006F77657228293A2000616363656C2E69E2
:100720007341736C65657028293A200061636365C5
:100730006C2E6973546170536F757263654F6E5A96
:1007400028293A2000616363656C2E6973546170D7
:10075000536F757263654F6E5928293A20006163A3
:1007600063656C2E6973546170536F757263654F66
:100770006E5828293A2000616363656C2E697341C5
:1007800063746976697479536F757263654F6E5AD5
:1007900028293A2000616363656C2E697341637494
:1007A0006976697479536F757263654F6E5928293C
:1007B0003A200069734163746976697479536F757F
:1007C0007263654F6E5828293A200069735461702E
:1007D000446574656374696F6E4F6E5A28293B20B7
:1007E00066616C73653F2000697354617044657481
:1007F000656374696F6E4F6E5A28293B2074727559
:10080000653F200069735461704465746563746961
:100810006F6E4F6E5928293B2066616C73653F20CF
:10082000006973546170446574656374696F6E4FD9
:100830006E5928293B20747275653F2000697354F6
:100840006170446574656374696F6E4F6E582829D2
:100850003B2066616C73653F20006973546170448E
:100860006574656374696F6E4F6E5828293B2074F8
:100870007275653F2000676574537570707265739B
:100880007342697428293B2066616C73653F2000C0
:100890006765745375707072657373426974282943
:1008A0003B20747275653F200069734163746976FB
:1008B000697479416328293A20006973496E61633C
:1008C0007469766974795A456E61626C6564282929
:1008D0003A20006973496E61637469766974795965
:1008E000456E61626C656428293A20006973496E1F
:1008F000616374697669747958456E61626C656488
:1009000028293A2000697341637469766974795AB9
:10091000456E61626C656428293A20006973416301
:1009200074697669747959456E61626C65642829C9
:100930003A20006973416374697669747958456E29
:1009400061626C656428293A2000676574467265A7
:100950006546616C6C4475726174696F6E28293AE2
:1009600020006765744672656546616C6C546872F8
:100970006573686F6C6428293A2000676574546950
:100980006D65496E616374697669747928293A20C6
:1009900000676574496E6163746976697479546837
:1009A000726573686F6C6428292000676574416301
:1009B0007469766974795468726573686F6C6428B9
:1009C000292000676574446F75626C6554617057C7
:1009D000696E646F7728292000676574446F7562BB
:1009E0006C655461704C6174656E637928293A2096
:1009F000006765745461704475726174696F6E2824
:100A0000293A2000676574417869734F666673659B
:100A1000742826782C2026792C20267A293A200042
:100A20006765745461705468726573686F6C64288C
:100A3000293A200058595A2047733A200058595AE9
:100A400020434F554E54533A20007365742067611C
:100A5000696E735B5D3A006761696E735F6F72699F
:100A6000675B5D3A00000020002300260029002C6F
:100A7000002F0032000001000003010601090105FA
:100A8000050505070508080808020202020A0A0807
:100A9000080404040401010101010101010303032D
:100AA0000303030303040707070C0C0C0C0C0C0CCA
:100AB0000C0202020206060606060606060B0B0BD1
:100AC0000B0B0B0B0B01021020200808102040100C
:100AD0002040800201020108040201010204081002
:100AE0002040808040201008040201800402018020
:100AF0004020100804020108040201010204081049
:100B00002040800102040810204080005EBCE261A9
:100B10003FDD83C29C7E20A3FD1F41009D23BE4676
:100B2000DB65F88C11AF32CA57E97443616C6962B6
:100B3000726174696F6E2050726573737572653D72
:100B400000536561206C6576656C20502863616C8C
:100B500063293D00234572726F723A707265737338
:100B600075726520424D503038352C2063686563BE
:100B70006B20776972696E67210049522054656D58
:100B8000702073656E736F7220666F756E640050AF
:100B90004D322E352073656E736F72206C696B65F4
:100BA0006C7920666F756E6400536F756E64204CAF
:100BB0006576656C2073656E736F7220666F756EF7
:100BC000640053656E736F7220736C6F7420616E76
:100BD0006420747970653A0057656C636F6D6520A9
:100BE000746F20456455484B003E4D6F74696F6EBD
:100BF00020627920756C747261736F6E6320736507
:100C00006E736F723A0A0000002100240027002A48
:100C1000002D003000330001010000040107010A2B
:100C20000100002200250028002B002E0031003496
:100C30000002010000050108010B0100000A0B027F
:100C4000090C0D0E0807030401000000000000005D
:100C50000000000000000000000000000000000094
:100C60000000000000000012111000000000000051
:100C70000000000000000000000000000000000074
:100C800000416E676C65732F004572726F72206E43
:100C9000756D62657220666F72207468652061727E
:100CA00072617920746F206176726167696E672165
:100CB0002F6E00434F3220436F6E630053656E7397
:100CC0006F72206572726F722100234E6F20736500
:100CD0006E736F722100434F3220436F6E63004D7D
:100CE0006561737572696E67004F3220436F6E6382
:100CF0000020202020202020202020202020202014
:100D00002000202020202020202020202020202003
:100D100020200020202020202020202020202020F3
:100D200020202000202020202020202020202020E3
:100D300020202020002020202020202020202020D3
:100D400020202020002020202020202020202020C3
:100D50002020202000236B6579323D00236B6579CC
:100D6000323D004F6666206169722D636F6E6421AB
:100D7000004974277320746F6F20636F6F6C2100BC
:100D800054656D702069732066696E652100497332
:100D9000206169722D636F6E64206F6E3F0049742D
:100DA000277320717569746520686F742100497418
:100DB0002773207665727920686F742120004F6652
:100DC00066206169722D636F6E6421004974277318
:100DD00020746F6F20636F6F6C210054656D7020FD
:100DE00069732066696E6521004973206169722DFF
:100DF000636F6E64206F6E3F0049742773207175B6
:100E000069746520686F74210049742773207665C2
:100E1000727920686F74210054656D702048756D7B
:100E2000696469747900232D2D2D2D2D2D2D2D2DE7
:100E30002D2D2D2D2D2D2D2D2D2D2D2D2D2D2D2DE2
:100E40002D2D2D2D2D2D2D2D2D2D2D002352657366
:100E50006F6C7574696F6E3A20202000234D696EA7
:100E60002056616C75653A2020202000234D617862
:100E70002056616C75653A202020200023556E694C
:100E80007175652049443A2020202000234472696E
:100E9000766572205665723A202020002353656ED5
:100EA000736F723A2020202020202000232D2D2D2A
:100EB0002D204D61676E657469632053656E736F95
:100EC00072202D2D2D2D2D2D2D2D2D2D2D2D2D2D1A
:100ED0002D2D2D2D2D2D00002B7BDB8411241FBEED
:100EE000CFEFD1E2DEBFCDBF00E00CBF1BE0A0E042
:100EF000B2E0ECE3F3E201E00BBF02C007900D9219
:100F0000AC3AB107D9F721E1ACEABBE001C01D92D0
:100F1000AC3BB207E1F717E0CDE6D7E000E006C052
:100F200021970109802FFE010E94F28ECC36D10755
:100F300080E00807A9F70E948A7D0C948D9160C813
:100F40002F923F924F925F926F927F928F929F92D9
:100F5000AF92BF92CF92DF92EF92FF920F931F93C7
:100F6000CF93DF93CDB7DEB7EA970FB6F894DEBF25
:100F70000FBECDBF86EC9BE00E944934892B09F45B
:100F800068C20E9444540E94216D6BE07AE0CE0159
:100F900001960E94AB5A4AE050E060E070E0CE015A
:100FA00001960E94B66ECE0101960E94E159809191
:100FB0001F118823B9F06FEB7AE083E79EE00E946F
:100FC000C55B4091CA0B5091CB0B6091CC0B7091DB
:100FD000CD0B20E183E79EE00E940D5B83E79EE05E
:100FE0000E94A25B8091CA0B9091CB0BA091CC0B7D
:100FF000B091CD0B883025E09207A105B10509F429
:1010000005C208F08DC0893461E09607A105B105DD
:1010100009F4FFC1E0F58434E1E09E07A105B105C4
:1010200009F4E8C1E8F4813421E09207A105B10593
:1010300009F4D1C138F480349140A105B10509F417
:10104000BBC1EAC1823471E09707A105B10509F47B
:10105000CBC183349140A105B10509F4C8C1DCC1FD
:101060008634F1E09F07A105B10509F4C9C108F470
:10107000C4C1873441E09407A105B10509F4C3C197
:1010800088349140A105B10509F4C0C1C5C18230C1
:1010900075E09707A105B10509F4A6C1E8F4843706
:1010A000F1E09F07A105B10509F451C138F4823779
:1010B0009140A105B10509F455C1AEC1811565E0A6
:1010C0009607A105B10509F477C181309540A105C6
:1010D000B10509F480C1A0C18530E5E09E07A105F6
:1010E000B10509F48AC170F4833025E09207A105A7
:1010F000B10509F47CC184309540A105B10509F41E
:1011000079C18AC1863065E09607A105B10509F469
:1011100077C187309540A105B10509F474C17CC140
:101120008D3BE2E49E07EFEFAE07B10509F435C150
:1011300008F04BC08F3E20E192072FEFA207B105C8
:1011400009F461C118F5823365E09607A105B10580
:1011500009F408C138F489309540A105B10509F4B6
:1011600058C15AC18433F5E09F07A105B10509F4C0
:10117000EEC08D3F9240AF4FB10509F04DC16EE713
:1011800075E083E190E10E947E59E9C08D3D42E225
:1011900094074FEFA407B10509F4D9C038F4873E8E
:1011A0009841AF4FB10509F428C136C18F3CE0E347
:1011B0009E07EFEFAE07B10509F41CC1873C9843C9
:1011C000AF4FB10509F422C127C1873928E692073C
:1011D0002FEFA207B10509F4FEC048F58D3A62E58C
:1011E00096076FEFA607B10509F4C8C038F4853B30
:1011F0009A44AF4FB10509F4DFC00EC1853AFAE554
:101200009F07FFEFAF07B10509F403C18D3992467F
:10121000AF4FB10509F000C16BE775E083E190E1E4
:101220000E947E5910929D118CEF9FEF8DC08735E3
:1012300048EA94074FEFA407B105F9F078F4853830
:101240007AE797077FEFA707B10509F4D9C087367A
:101250009849AF4FB10509F4C7C0DEC08F34F0EB39
:101260009F07FFEFAF07B10509F4C1C08D33924C62
:10127000AF4FB10509F476C0CFC082E080931C0F58
:101280001092200F00E010E08CEA9BE00E944934AD
:10129000892B69F40F5F1F4F093E43E0140739F0B3
:1012A0006EE170E080E090E00E94965DEDCF80916D
:1012B0001F118823B9F067E573E083E79EE00E9481
:1012C000D45A4091B00B5091B10B6091B20B709118
:1012D000B30B2AE083E79EE00E940D5B83E79EE06C
:1012E0000E94A25B8091B00B9091B10BA091B20BC8
:1012F000B091B30B853065E09607A105B10509F4FF
:101300004EC308F0CEC28734E1E09E07A105B105C7
:1013100009F451C308F0A5C2833421E09207A10566
:10132000B10509F42AC308F092C2813461E096073E
:10133000A105B10509F084C26AE675E087E090E195
:101340000E947E5989EF9FEF0E94481F7CC06EE784
:1013500075E083E190E10E947E5910929D118BEF20
:101360009FEFF2CF61E875E083E190E10E947E5942
:1013700081E080939D118DEF9FEFE6CF64E875E0EB
:1013800087E090E10E947E5964E875E083E190E196
:101390000E947E598EEF9FEFD7CF67E875E087E018
:1013A00090E10E947E5967E875E083E190E10E9438
:1013B0007E598FEF9FEFC8CF65E775E087E090E13A
:1013C0000E947E5965E775E083E190E10E947E59B5
:1013D00080E090E0B9CF68E875E087E090E10E9496
:1013E0007E5981E090E0B0CF82E090E0ADCF83E025
:1013F00090E0AACF84E090E0A7CF85E090E0A4CF72
:1014000086E090E0A1CF87E090E09ECF88E090E07A
:101410009BCF89E090E098CF60E070E0CE0101962C
:101420000E946644BE016F5F7F4F87E090E10E949B
:10143000A859CE0101960E94E15964E670E080E06F
:1014400090E00E94965D82E080931C0F1092200F26
:1014500009C16CEF7AE083E190E10E947E5910921D
:10146000BD0B6CEF7AE083E190E10E947E5901E0D0
:1014700083E79EE00E9464572091BD0B1816190661
:101480000CF0DEC22111DCC29FC28091970C9091BA
:10149000980C892B71F46FE776E0CE0101960E94DB
:1014A000AB5ACE0101960E94FD75CE0101960E94B5
:1014B000E1598091970C9091980C019771F46EE826
:1014C00076E0CE0101960E94AB5ACE0101960E94B1
:1014D000FD75CE0101960E94E15960915402709110
:1014E00055024AE0CE0145960E94705A68E976E0BE
:1014F000CE0101960E94AB5ABE016B5E7F4FCE01BA
:1015000001960E943359BC01CE0183960E94A35AD2
:10151000CE0183960E94FD75CE0183960E94E1590B
:10152000CE0101960E94E159CE0145960E94E159F3
:1015300040910002509101026091020270910302F9
:1015400022E0CE0145960E94155A65EB76E0CE0169
:1015500001960E94AB5ABE016B5E7F4FCE01019691
:101560000E9433596EEA78E00E941C59BC01CE01FA
:1015700083960E94A35ACE0183960E94FD75CE01E8
:1015800083960E94E159CE0101960E94E159CE0155
:1015900045960E94E15940910C0250910D026091D4
:1015A0000E0270910F0222E0CE0145960E94155A5C
:1015B00065EC76E0CE0101960E94AB5ABE016B5EEF
:1015C0007F4FCE0101960E9433596EEA78E00E9467
:1015D0001C59BC01CE0183960E94A35ACE0183966A
:1015E0000E94FD75CE0183960E94E159CE010196BD
:1015F0000E94E159CE0145960E94E159B12C80919B
:10160000171090911810039708F0E7C50E944454F2
:101610000E94216D6BE07AE0CE0101960E94AB5AE8
:101620004AE050E060E070E0CE0101960E94046E56
:10163000CE0101960E94E1598091171090911810E7
:101640008130910509F057C5E0911310F091141005
:10165000309711F40C94221F1081812F0E94147670
:101660000E94B2490E94B2496093C20B7093C30BAF
:101670008093C40B9093C50BD5C089E39DE00E9475
:1016800042578093BC0B8A3009F4E6C18D3009F4CF
:10169000E3C19091BD0B9111DFC189831A8241E0B2
:1016A00050E0BE016F5F7F4F83E190E10E94EF58F1
:1016B0008FEFE81AF80A6FE070E080E090E00E9497
:1016C000965D89E39DE00E94645718161906ACF2F6
:1016D00062E370E080E090E00E94965DEF2839F1CF
:1016E00063E975E0CE0145960E94AB5A63E170E173
:1016F000CE0145960E943359BC01CE0101960E944D
:10170000A35ACE0101960E94546FCE0101960E9409
:10171000E159CE0145960E94E15989E39DE00E947E
:10172000F25764E670E080E090E00E94965D2091C0
:10173000BD0B8091171090911810222309F483C1DA
:101740000197D1F56EEA78E0CE0101960E94AB5A7E
:10175000CE0101960E940F63811198C169E975E07D
:10176000CE0145960E94AB5ACE0145960E940F636A
:1017700001E0811100E0CE0145960E94E159CE01C1
:1017800001960E94E159002389F060E070E0CE01EB
:1017900001960E946644BE016F5F7F4F87E090E133
:1017A0000E94A859CE0101960E94E15964E170E0BF
:1017B00080E090E00E94965D6AE070E080E090E05A
:1017C0000E94965D8091171090911810009709F073
:1017D0005FC10E94C177182F81110C94921E8091D5
:1017E0009D1181110C94B01E0E94B2490091C20B50
:1017F0001091C30B2091C40B3091C50BDC01CB01C0
:10180000801B910BA20BB30B88349E4EA105B10532
:1018100048F01092101160E085E091E10E947B4D4C
:101820001092D90480919D11882311F40C942F1FDC
:1018300064E670E080E090E00E94965D0C942F1FBB
:1018400082349140A105B10509F48EC0F6CD8534EE
:10185000E1E09E07A105B10509F4A1C008F496C016
:10186000A7C0813025E09207A105B10509F464CD38
:1018700070F4883461E09607A105B10509F49EC0B3
:1018800089349140A105B10509F49BC0D6CD8330C0
:10189000E5E09E07A105B10509F46FC008F464C036
:1018A00075C08F3C20E392072FEFA207B10509F422
:1018B0006DC068F5883065E09607A105B10509F4AB
:1018C0007DC070F48630E5E09E07A105B10509F4FE
:1018D0006FC087309540A105B10509F46CC0ADCD4E
:1018E0008F3E20E192072FEFA207B10509F463C0F4
:1018F000873E48E194074FEFA407B10509F44FC0B4
:1019000089309540A105B10509F097CD5AC08739B6
:1019100078E697077FEFA707B10509F40DCD78F4B6
:10192000873CF8E39F07FFEFAF07B10509F446C016
:10193000853A9A45AF4FB10509F443C07ECD87364D
:1019400048E994074FEFA407B10571F08F3460EBBD
:1019500096076FEFA607B10581F085389A47AF4F1C
:10196000B10509F06ACD24C06DE675E087E090E12D
:101970000E947E5988EF9FEFE7CC60E775E087E033
:1019800090E10E947E5987EF9FEFDECC63E775E020
:1019900087E090E10E947E5986EF9FEFD5CC67E704
:1019A00075E087E090E10E947E5985EF9FEFCCCCF7
:1019B00084EF9FEFC9CC83EF9FEFC6CC82EF9FEF00
:1019C000C3CC81EF9FEFC0CC83E79EE00E944257DB
:1019D0008093BC0B8A3071F08D3061F089831A825C
:1019E00041E050E0BE016F5F7F4F83E190E10E94D4
:1019F000EF581FC00093BD0B6AE875E0CE01459615
:101A00000E94AB5A63E170E1CE0145960E943359C2
:101A1000BC01CE0101960E94A35ACE0101960E94FC
:101A2000546FCE0101960E94E159CE0145960E9465
:101A3000E1596AE070E080E090E00E94965D18CD88
:101A4000211175CE05C0009709F07ACE0C94F71ECF
:101A5000E12CF12C01E035CE8091171090911810F7
:101A6000892B09F428CE0093BD0B89E39DE00E94E9
:101A70006457181619060CF01ECE6CEF7AE083E15D
:101A800090E10E947E591092BD0B15CE00E077CEFA
:101A90000197E1F56BE975E0CE0183960E94AB5AA0
:101AA000CE0183960E940F6381110C94291F6FE66B
:101AB00079E0CE0145960E94AB5ACE0145960E9430
:101AC0000F63811112C067E17AE0CE0101960E9496
:101AD000AB5ACE0101960E940F6301E0811100E034
:101AE000CE0101960E94E15901C000E0CE01459669
:101AF0000E94E159CE0183960E94E159002331F002
:101B000063E170E187E090E10E94935980911710A2
:101B1000909118100497E8F56DE975E0CE010196F3
:101B20000E94AB5ACE0101960E940F63082FCE018E
:101B300001960E94E159002361F161E070E0CE015D
:101B400001960E946644CE0101960E94474F2AEFFB
:101B5000C22EDD24DA94ED2CFD2C46015701861AA5
:101B6000970AA80AB90AB501A4012AE0CE01459650
:101B70000E94445ABE016B5E7F4F87E090E10E9455
:101B8000A859CE0145960E94E159CE0101960E94C6
:101B9000E1596FE975E0CE0145960E94AB5ACE013E
:101BA00045960E940F63811113C063EA75E0CE0170
:101BB00001960E94AB5ACE0101960E940F6301E08C
:101BC000811101C000E0CE0101960E94E15901C0DF
:101BD00001E0CE0145960E94E159002309F488C234
:101BE0006BEE73E0CE0101960E949B5ACE010196E6
:101BF0000E94FD75CE0101960E94E15967EA75E0E9
:101C0000CE0101960E94AB5A6FEF70E1CE010196B2
:101C10000E943359BC01CE0145960E94A35ACE01C1
:101C200045960E94FD75CE0145960E94E159CE0170
:101C300001960E94E1596091A9027091AA028091D7
:101C4000AB029091AC020E94148A20E030E048EC94
:101C500052E40E94648CAB01BC0122E0CE014596A7
:101C60000E94155A6DEB75E0CE0101960E94AB5AA9
:101C7000BE016B5E7F4FCE0101960E9433596CE02E
:101C800077E00E941C59BC01CE0183960E94A35AA2
:101C9000CE0183960E94FD75CE0183960E94E15984
:101CA000CE0101960E94E159CE0145960E94E1596C
:101CB0004091A5025091A6026091A7027091A802DE
:101CC00024E0CE0145960E94155A62ED75E0CE01E2
:101CD00001960E94AB5ABE016B5E7F4FCE0101960A
:101CE0000E943359BC01CE0183960E94A35ACE01B3
:101CF00083960E94FD75CE0183960E94E159CE0124
:101D000001960E94E159CE0145960E94E159409109
:101D1000990250919A0260919B0270919C0222E07C
:101D2000CE018F960E94155A4091910250919202D5
:101D3000609193027091940223E0CE0189960E94F3
:101D4000155A40919D0250919E0260919F027091A0
:101D5000A00222E0CE0183960E94155A409195027E
:101D600050919602609197027091980223E0CE0103
:101D700045960E94155A6FEE75E0CE0101960E94BD
:101D8000AB5ABE016B5E7F4FCE0101960E94335964
:101D900064E076E00E941C59BE016D5D7F4F0E9499
:101DA000335967E076E00E941C59BE01675D7F4FA2
:101DB0000E94335964E076E00E941C59BE01615DC7
:101DC0007F4F0E9433596DE076E00E941C59BC01A0
:101DD000CE01C5960E94A35ACE01C5960E94FD75FC
:101DE000CE01C5960E94E159CE0101960E94E159AB
:101DF000CE0145960E94E159CE0183960E94E15999
:101E0000CE0189960E94E159CE018F960E94E15938
:101E100040914C0250914D0260914E0270914F02E0
:101E200023E0CE0183960E94155A209144023091FE
:101E30004502409146025091470260E070E080E226
:101E400091E40E94128EAB01BC0121E0CE014596C7
:101E50000E94E65962E176E0CE0101960E94AB5AFB
:101E6000BE016B5E7F4FCE0101960E94335965E241
:101E700076E00E941C59BE016D5D7F4F0E94335970
:101E80006BE276E00E941C59BC01CE0189960E944B
:101E9000A35ACE0189960E94FD75CE0189960E94B3
:101EA000E159CE0101960E94E159CE0145960E946A
:101EB000E159CE0183960E94E15940914802509128
:101EC000490260914A0270914B0223E0CE01839651
:101ED0000E94155A209140023091410240914202E5
:101EE0005091430260E070E080E291E40E94128E23
:101EF000AB01BC0121E0CE0145960E94E6596EE29D
:101F000076E0CE0101960E94AB5ABE016B5E7F4F18
:101F1000CE0101960E94335965E276E00E941C5979
:101F2000BE016D5D7F4F0E9433596BE276E00E94E7
:101F30001C59BC01CE0189960E94A35ACE018996F4
:101F40000E94FD75CE0189960E94E159CE0101964D
:101F50000E94E159CE0145960E94E159CE01839637
:101F60000E94E15940918D0250918E0260918F0242
:101F70007091900222E0CE0145960E94155A61E4CC
:101F800076E0CE0101960E94AB5ABE016B5E7F4F98
:101F9000CE0101960E94335967E576E00E941C59F4
:101FA000BC01CE0183960E94A35ACE0183960E9463
:101FB000FD75CE0183960E94E159CE0101960E94E3
:101FC000E159CE0145960E94E15940918902509114
:101FD0008A0260918B0270918C0222E0CE014596BC
:101FE0000E94155A6EE576E0CE0101960E94AB5A2A
:101FF000BE016B5E7F4FCE0101960E9433596BE2AA
:1020000076E00E941C59BC01CE0183960E94A35A1F
:10201000CE0183960E94FD75CE0183960E94E15900
:10202000CE0101960E94E159CE0145960E94E159E8
:1020300009E7C02E02E0D02EEE24E394F12C07E154
:1020400080917702909178028E159F050CF41DCA3D
:10205000F601A190B1906F014AE0B501CE018396DF
:102060000E94705A4AE0B701CE0145960E94705A0C
:1020700061E776E0CE0101960E94AB5ABE016B5E2D
:102080007F4FCE0101960E94335963E97BE00E94A5
:102090001C59BE016D5D7F4F0E94335969E776E0A0
:1020A0000E941C590A9DB0010B9D700D11246A54A9
:1020B0007D4F0E941C59BC01CE0189960E94A35AF3
:1020C000CE0189960E94FD75CE0189960E94E15944
:1020D000CE0101960E94E159CE0145960E94E15938
:1020E000CE0183960E94E159FFEFEF1AFF0AA8CFB5
:1020F000BB24B39484CA029709F0AFCA6DE975E0B6
:10210000CE0101960E94AB5ACE0101960E940F6348
:10211000082FCE0101960E94E159002309F49DCABF
:102120008091171090911810029740F0E0911310D1
:10213000F0911410309711F0818101C080E01A8273
:1021400019821C821B821E821D828D8B1E8ABE01FB
:102150006B5E7F4FCE0101960E947E59BE016F5F7C
:102160007F4F87E090E10E94A859CE0101960E941E
:10217000E1598091171090911810892B41F0E0914E
:102180001310F0911410309711F0108101C010E07D
:1021900080911F11882309F460CA65ED76E0CE01B5
:1021A00001960E94AB5A63E170E1CE0101960E9454
:1021B00033596BE07AE00E941C59BC0183E79EE032
:1021C0000E94C65ACE0101960E94E15967E070E173
:1021D00083E79EE00E94B55B40CA41E050E060E0CA
:1021E00070E0CE0101960E942444BE016F5F7F4FD4
:1021F00085EF9FE00E94A859CE0101960E94E15907
:1022000068E077E0CE0145960E94AB5ACE01459634
:102210000E940F63811113C063E17AE0CE01019641
:102220000E94AB5ACE0101960E940F6311E081110A
:1022300001C010E0CE0101960E94E15901C011E0F9
:10224000CE0145960E94E159112309F4B2C062E023
:1022500070E0CE0101960E946644BE016F5F7F4F21
:1022600085EF9FE00E94A859CE0101960E94E15996
:1022700065EF7FE0CE0101960E94A35ACE01019640
:102280000E94546FCE0101960E94E1590E94E94ECE
:1022900020E030E048EC52E40E94738A0E94FD8CFA
:1022A000AB01BC014093A9025093AA026093AB0218
:1022B0007093AC022AE0CE0101960E94445ACE01EE
:1022C00001960E94546FCE0101960E94E1596091DF
:1022D000A9027091AA028091AB029091AC028B018D
:1022E0009C0100591F452140310901341C49210539
:1022F000310588F06BED76E0CE0101960E94AB5A75
:1023000065EF7FE0CE0101960E9433596EEE76E0D4
:102310000E941C5952C119821A821B821C821D8282
:102320001E821F8218860E94148A20E030E048EC4A
:1023300052E40E94648C8E010F5F1F4F22E047E041
:102340000E944085BC018BEF9FE00E947E596EEF9A
:1023500076E0CE0145960E94AB5A6BEF7FE0CE014E
:1023600045960E9433596BE077E00E941C59BC01EE
:102370008BEF9FE00E949359CE0145960E94E15950
:1023800010924911109248118091A9029091AA02CD
:10239000A091AB02B091AC028093210C9093220CDF
:1023A000A093230CB093240C80E090E00E94D144D1
:1023B0000DC160E177E0CE0145960E94AB5ACE0197
:1023C00045960E940F63811113C066E177E0CE014C
:1023D00001960E94AB5ACE0101960E940F6311E054
:1023E000811101C010E0CE0101960E94E15901C0A7
:1023F00011E0CE0145960E94E159112309F467C00E
:1024000046E050E065E070E0CE0101960E94244471
:10241000BE016F5F7F4F85EF9FE00E94A859CE01FC
:1024200001960E94E15985EF9FE00E94474F6B01A2
:102430007C0165E576E0CE0101960E94AB5ACE01A3
:1024400001960E94F54EBC016F5F7F4FCE0145960D
:102450000E946644BE016B5E7F4F85EF9FE00E9445
:10246000A859CE0145960E94E159CE0101960E94DD
:10247000E15985EF9FE00E94474FDB01E7E7F2E07B
:1024800041E050E02091770230917802241735071F
:102490005CF0228133812A173B0711F413821282E8
:1024A0004F5F5F4F3296EECF9601220F331FF90137
:1024B000E958FD4F7183608382E090E00E9493555C
:1024C00063E170E183E79EE00E94B55B87C26CE147
:1024D00077E0CE0145960E94AB5ACE0145960E9408
:1024E0000F63811113C062E277E0CE0101960E9472
:1024F000AB5ACE0101960E940F6311E0811101C019
:1025000010E0CE0101960E94E15901C011E0CE0118
:1025100045960E94E1591123F1F0E7E7F2E081E0EE
:1025200090E020917702309178022817390774F0F3
:10253000863091051CF49383828305C09C012E5F35
:102540003F4F3383228301963296EBCF82E090E0B7
:102550000E94935543C268E277E0CE0145960E94FF
:10256000AB5ACE0145960E940F63811113C060E300
:1025700077E0CE0101960E94AB5ACE0101960E94EF
:102580000F6311E0811101C010E0CE0101960E949D
:10259000E15901C011E0CE0145960E94E159112395
:1025A00059F168E377E0CE0101960E94AB5A69EFDA
:1025B00070E1CE0101960E943359BC018BEF9FE080
:1025C0000E949359CE0101960E94E1596FEB7AE087
:1025D000CE0101960E94AB5A6BEF7FE0CE010196CF
:1025E0000E943359BC01CE0145960E94A35ACE01E8
:1025F00045960E94FD759DC162E477E0CE01459647
:102600000E94AB5ACE0145960E940F63811113C000
:1026100069E477E0CE0101960E94AB5ACE010196A3
:102620000E940F6311E0811101C010E0CE010196FC
:102630000E94E15901C011E0CE0145960E94E15986
:102640001123A9F060E577E0CE0101960E94AB5A14
:102650006FEF70E1CE0101960E943359BC018BEF00
:102660009FE00E949359CE0101960C94531D6FE593
:1026700077E0CE0145960E94AB5ACE0145960E9466
:102680000F63811113C064E677E0CE0101960E94CA
:10269000AB5ACE0101960E940F6311E0811101C077
:1026A00010E0CE0101960E94E15901C011E0CE0177
:1026B00045960E94E159112309F43FC065E576E093
:1026C000CE0101960E94AB5ACE0101960E94F54EB2
:1026D000BC016F5F7F4FCE0145960E946644BE01EC
:1026E0006B5E7F4F85EF9FE00E94A859CE01459613
:1026F0000E94E159CE0101960E94E15985EF9FE0C9
:102700000E94474F6115710521F481E08093DA043E
:1027100005C06130710531F41092DA040E945354FF
:102720000C94320B6230710511F00C94320B81E085
:102730008093DA041092D904F1CF69E677E0CE01F4
:1027400045960E94AB5ACE0145960E940F638111B7
:1027500013C06DE677E0CE0101960E94AB5ACE0120
:1027600001960E940F6311E0811101C010E0CE01BB
:1027700001960E94E15901C011E0CE0145960E94E8
:10278000E159112309F470C063E070E0CE010196B5
:102790000E946644BE016F5F7F4F85EF9FE00E94FD
:1027A000A859CE0101960E94E15965EF7FE083E7C9
:1027B0009EE00E94B55B109249111092481165EF9E
:1027C0007FE08FEF90E10E9493598DE39CE0892B8D
:1027D000E1F000910311109104110115110519F494
:1027E00010923D0C12C00730110510F007E010E008
:1027F0006091FF1070910011A8018DE39CE00E9490
:102800006491F801E35CF34F10828091481190913C
:1028100049110E94D14461E777E0CE0145960E94BC
:10282000AB5A6FEF70E1CE0145960E943359BC015F
:10283000CE0101960E94A35ACE0145960E94E1590D
:10284000BE016F5F7F4F89E39DE00E94C65A68EB2F
:102850007BE080E090E00E94965D6DE37CE0CE013D
:1028600045960E94AB5A61C069E777E0CE01459674
:102870000E94AB5ACE0145960E940F63811113C08E
:102880006EE777E0CE0101960E94AB5ACE01019629
:102890000E940F6311E0811101C010E0CE0101968A
:1028A0000E94E15901C011E0CE0145960E94E15914
:1028B000112309F444C064E070E0CE0101960E9447
:1028C0006644BE016F5F7F4F85EF9FE00E94A8596D
:1028D000CE0101960E94E15963E877E0CE0145966A
:1028E0000E94AB5A65EF7FE0CE0145960E943359B6
:1028F000BC01CE0101960E94A35ACE0145960E94CA
:10290000E159BE016F5F7F4F89E39DE00E94C65A87
:1029100068EB7BE080E090E00E94965DBE016F5F17
:102920007F4FCE0145960E94A35ACE0145960E9444
:10293000546FCE0145960E94E1590C948C1E6AE8B2
:1029400077E0CE0145960E94AB5ACE0145960E9493
:102950000F63811113C06FE877E0CE0101960E94EA
:10296000AB5ACE0101960E940F6311E0811101C0A4
:1029700010E0CE0101960E94E15901C011E0CE01A4
:1029800045960E94E159112399F145E050E064E039
:1029900070E0CE0101960E942444BE016F5F7F4F1C
:1029A00085EF9FE00E94A859CE0101960E94E1594F
:1029B00085EF9FE00E94474F7093980C6093970CAF
:1029C00063E170E1CE0101960E94A35ACE01019607
:1029D0000E94546FCE0101960E94E1591092491154
:1029E0001092481180E090E00E94D1440C94320B88
:1029F00064E977E0CE0145960E94AB5ACE01459638
:102A00000E940F63811113C069E977E0CE0101963E
:102A10000E94AB5ACE0101960E940F6311E0811112
:102A200001C010E0CE0101960E94E15901C011E001
:102A3000CE0145960E94E159112309F45EC046E09B
:102A400050E064E070E0CE0101960E942444BE0193
:102A50006F5F7F4F85EF9FE00E94A859CE010196DE
:102A60000E94E15985EF9FE00E94474F70939A0CB6
:102A70006093990C709355026093540263E170E186
:102A8000CE0101960E94A35ACE0101960E94546F76
:102A9000CE0101960E94E1591092491110924811FD
:102AA00080E090E00E94D144209154028091520233
:102AB0009091530280936610209367109C013327F6
:102AC000F901EB53F54FE491E0936810F901E158F7
:102AD000F54FE491E093691062E00E94355D80E378
:102AE00098EFAFEFBFEF80936A1090936B10A093B5
:102AF0006C10B0936D100C94320B6EE977E0CE0140
:102B000045960E94AB5ACE0145960E940F638111F3
:102B100013C065EA77E0CE0101960E94AB5ACE0160
:102B200001960E940F6311E0811101C010E0CE01F7
:102B300001960E94E15901C011E0CE0145960E9424
:102B4000E159112311F147E050E066E070E0CE0159
:102B500001960E942444BE016F5F7F4F85EF9FE086
:102B60000E94A859CE0101960E94E15985EF9FE08D
:102B70000E94474F672B21F410921F110C94821E64
:102B800081E080931F110C94821E6CEA77E0CE01E5
:102B900083960E94AB5ACE0183960E940F638111E7
:102BA0008FC76FEA77E0CE0145960E94AB5ACE01FF
:102BB00045960E940F63811113C062EB77E0CE014E
:102BC00001960E94AB5ACE0101960E940F6311E05C
:102BD000811101C010E0CE0101960E94E15901C0AF
:102BE00011E0CE0145960E94E159CE0183960E94E4
:102BF000E159111169C766EE77E0CE0101960E9496
:102C0000AB5ACE0101960E940F63182FCE01019698
:102C10000E94E159112309F46CC080911710909122
:102C20001810079710F40C947E1E66E070E0CE0139
:102C300001960E946644BE016F5F7F4F85EF9FE063
:102C40000E94A859CE0101960E94E1590E94E94EC6
:102C5000AB01BC0140930002509301026093020259
:102C60007093030221E0CE0145960E94155A65EB50
:102C700076E0CE0101960E94AB5ABE016B5E7F4F9B
:102C8000CE0101960E9433596EEA78E00E941C59E9
:102C9000BC018BEF9FE00E949359CE0101960E94E8
:102CA000E159CE0145960E94E1596BEF7FE0CE01DC
:102CB00001960E94A35ACE0101960E94FD75CE0195
:102CC00001960E94E1590E94B24928EE33E040E0AB
:102CD00050E00E946C8BCA01B9010E94128A609375
:102CE000BE0B7093BF0B8093C00B9093C10B0C94E1
:102CF0007E1E6DEE77E0CE0101960E94AB5ACE01AA
:102D000001960E940F63182FCE0101960E94E1598F
:102D1000112309F446C0809117109091181007975D
:102D200008F4ECC766E070E0CE0101960E946644AC
:102D3000BE016F5F7F4F85EF9FE00E94A859CE01D3
:102D400001960E94E1590E94E94EAB01BC014093FB
:102D50000C0250930D0260930E0270930F0221E05B
:102D6000CE0145960E94155A65EC76E0CE0101969B
:102D70000E94AB5ABE016B5E7F4FCE0101960E944E
:102D800033596EEA78E00E941C59BC018BEF9FE03A
:102D90000E949359CE0101960E94E159CE014596B9
:102DA00082C664EF77E0CE0145960E94AB5ACE0111
:102DB00045960E940F63811114C068EF77E0CE0141
:102DC00001960E94AB5ACE0101960E940F63FF2428
:102DD000F394811101C0F12CCE0101960E94E159BA
:102DE00002C0FF24F3948E010B5E1F4FC8010E94A6
:102DF000E159FF2009F455C08091CF049091D0048F
:102E00000E94C16860939502709396028093970226
:102E1000909398026093350C7093360C8093370C26
:102E20009093380C80E090E0A0E8BFE380939D028F
:102E300090939E02A0939F02B093A00280932D0CCA
:102E400090932E0CA0932F0CB093300C80911F11F7
:102E5000882381F06FEC73E083E79EE00E94D45AF0
:102E600060919502709196028091970290919802DC
:102E70000E94FE5F109249111092481180E090E08C
:102E80000E94D14440919502509196026091970220
:102E90007091980222E0C8010E94155A6CEF77E009
:102EA000EFC565E078E0C8010E94AB5AC8010E94F6
:102EB0000F63811114C06BE078E0CE0101960E948F
:102EC000AB5ACE0101960E940F63FF24F394811147
:102ED00001C0F12CCE0101960E94E15902C0FF24ED
:102EE000F394C8010E94E159FF2009F4B6C0809113
:102EF0001710909118100797D8F066E070E0CE0197
:102F000001960E946644BE016F5F7F4F85EF9FE090
:102F10000E94A859CE0101960E94E1590E94E94EF3
:102F200060938D0270938E0280938F029093900233
:102F30008091CD049091CE0499270E94CC56BC017B
:102F4000990F880B990B0E94148A2DE038E643E50F
:102F50005BE30E94738A6B017C012091280230910F
:102F6000290240912A0250912B020E940E8A1816C3
:102F70004CF06091100270911102809112029091B8
:102F800013021BC020913C0230913D0240913E0251
:102F900050913F02C701B6010E94538D87FF05C0C3
:102FA000C701B6010E948D4308C060912402709150
:102FB0002502809126029091270220E030E048EC23
:102FC00052E40E94738A6B017C0120E030E0A90189
:102FD0000E940E8A181634F0C12CD12CA8EAEA2ED1
:102FE000A1E4FA2EC0928D02D0928E02E0928F025E
:102FF000F0929002C092550CD092560CE092570C71
:10300000F092580C80911F11882381F06DEB73E0D2
:1030100083E79EE00E94D45A60918D0270918E02E7
:1030200080918F02909190020E94FE5F1092491150
:103030001092481180E090E00E94D14440918D02AE
:1030400050918E0260918F027091900222E0C8012F
:103050000E94155A61E178E013C56BE178E0C80180
:103060000E94AB5AC8010E940F63811114C060E234
:1030700078E0CE0101960E94AB5ACE0101960E94E3
:103080000F63FF24F394811101C0F12CCE0101964E
:103090000E94E15902C0FF24F394C8010E94E15943
:1030A000FF2009F492C08091171090911810069794
:1030B000E8F065E070E0CE0101960E946644BE0132
:1030C0006F5F7F4F85EF9FE00E94A859CE01019668
:1030D0000E94E1590E94E94E0E94948D609344023F
:1030E000709345028093460290934702809150026C
:1030F000909151020E94038520E030E048E051E4C5
:103100000E94648C60934C0270934D0280934E0237
:1031100090934F026093450C7093460C8093470C3C
:103120009093480C8091440290914502A0914602F0
:10313000B091470280934D0C90934E0CA0934F0C8E
:10314000B093500C80911F11882341F16CEA73E019
:1031500083E79EE00E94D45A2091440230914502B8
:10316000409146025091470260E070E080E291E4B5
:103170000E94128E41E050E00E94464265E278E0F3
:1031800083E79EE00E94C55B60914C0270914D0206
:1031900080914E0290914F020E94FE5F1092491161
:1031A0001092481180E090E00E94D14440914C027E
:1031B00050914D0260914E0270914F0223E0C80180
:1031C0000E94155A6CE278E0A9C067E378E0C80174
:1031D0000E94AB5AC8010E940F63811114C06CE3B6
:1031E00078E0CE0101960E94AB5ACE0101960E9472
:1031F0000F63FF24F394811101C0F12CCE010196DD
:103200000E94E15902C0FF24F394C8010E94E159D1
:10321000FF2009F491C08091171090911810069723
:10322000E8F065E070E0CE0101960E946644BE01C0
:103230006F5F7F4F85EF9FE00E94A859CE010196F6
:103240000E94E1590E94E94E0E94948D60934002D1
:103250007093410280934202909343028091500206
:10326000909151020E94038520E030E048E051E453
:103270000E94648C609348027093490280934A02D2
:1032800090934B026093490C70934A0C80934B0CC3
:1032900090934C0C209140023091410240914202A7
:1032A000509143022093510C3093520C4093530C95
:1032B0005093540C80911F118823D1F060E070E08E
:1032C00080E291E40E94128E41E050E00E9446426A
:1032D00065E278E083E79EE00E94C55B609148026A
:1032E0007091490280914A0290914B020E94FE5FC8
:1032F000109249111092481180E090E00E94D14450
:10330000409148025091490260914A0270914B02EB
:1033100023E0C8010E94155A61E478E0CE010196CD
:103320000E94AB5AB801CE0101960E94335965E361
:1033300078E00E941C59ADC36AE478E0C8010E949D
:10334000AB5AC8010E940F63811114C06EE478E08B
:10335000CE0101960E94AB5ACE0101960E940F63E6
:10336000FF24F394811101C0F12CCE0101960E943B
:10337000E15902C0FF24F394C8010E94E159FF20E3
:1033800009F46DC060E08091C9040E94355DF9E1E7
:10339000AF2EB12CC12CD12C76018091C9040E9492
:1033A000715DBC01990F880B990B0E94148A9B01D7
:1033B000AC01C701B6010E949E8B6B017C016AE0E3
:1033C00070E080E090E00E94965D61E0A61AB1088E
:1033D00021F720E030E040EA50E4C701B6010E9446
:1033E000738A20E030E040E85AE30E94738A20E0CC
:1033F00030E048EC51E40E94648C60938902709341
:103400008A0280938B0290938C0260936B0C709372
:103410006C0C80936D0C90936E0C1092491110926D
:10342000481180E090E00E94D1444091890250917F
:103430008A0260918B0270918C0222E0C8010E9486
:10344000155A6EE576E0CE0101960E94AB5AB8019E
:10345000CE0101960E9433596BE276E06ACF62E5B5
:1034600078E0C8010E94AB5AC8010E940F63811125
:1034700014C066E578E0CE0101960E94AB5ACE01F9
:1034800001960E940F63FF24F394811101C0F12C77
:10349000CE0101960E94E15902C0FF24F394C801B5
:1034A0000E94E159FF2009F435C146E050E064E094
:1034B00070E0CE0101960E942444BE016F5F7F4FF1
:1034C00085EF9FE00E94A859CE0101960E94E15924
:1034D00085EF9FE00E94474F4B015C011B0165E5B2
:1034E00076E0CE0101960E94AB5ACE0101960E9471
:1034F000F54EBC016F5F7F4FC8010E946644B80162
:1035000085EF9FE00E94A859C8010E94E159CE01B1
:1035100001960E94E159F090C7040E94E94E2B01E8
:103520003C01640171E0C71AD10880911F11882302
:10353000B9F06AE673E083E79EE00E94D45A4AE05D
:1035400050E0B40183E79EE00E949C5B6BE07AE070
:1035500083E79EE00E94C55BC301B2010E94FE5F4B
:103560006F2DC8010E944C4D18870F831D821E824B
:10357000198289E08A8381E08B838C831C8A1B8A71
:10358000CE0101960E94A84CCE0101960E943A4BB2
:10359000CE0101960E94CD61EE80F12C8BE0E81601
:1035A000F1041CF0EAE0EE2EF12CEBE58E1691040E
:1035B00008F44CC070E2A72E71E1B72E3501212C22
:1035C000312C2101C12CD12CCE14DF04B9F06C2D8B
:1035D000CE0101960E943A4C9B01AC01F30161932C
:1035E0007193819391933F01C201B1010E949E8B1F
:1035F0001B012C01FFEFCF1ADF0AE6CFB7010F2C1A
:10360000000C880B990B0E94148A9B01AC01C2012B
:10361000B1010E94648C2B013C01C12CD12CCE1431
:10362000DF0409F457C0F5012081318142815381C3
:10363000C301B2010E949D8BF50161937193819347
:1036400091935F01FFEFCF1ADF0AE9CF1214130441
:103650000CF5E214F30424F4670121E0C21AD10846
:103660006C2DCE0101960E943A4C9B01AC01C60123
:10367000880F991F880F991FBC01605E7E4E6B01F9
:10368000C301B2010E949D8BF60160837183828326
:10369000938320C02328F1F440E2A42E41E1B42E0C
:1036A000C12CD12CCE14DF04A9F06C2DCE010196D3
:1036B0000E943A4C9B01AC01C301B2010E949D8B58
:1036C000F50161937193819391935F01FFEFCF1A9D
:1036D000DF0AE8CFE0E2F1E1AFE6BCE041915191D1
:1036E000619171914D935D936D937D9321E1E834E8
:1036F000F207A1F7109249111092481180E090E072
:103700000E94D14464E070E0C8010E9466446AE50A
:1037100078E0B6C16BE778E0C8010E94AB5AC801F7
:103720000E940F63811114C06FE778E0CE0101960B
:103730000E94AB5ACE0101960E940F63FF24F394BE
:10374000811101C0F12CCE0101960E94E15902C005
:10375000FF24F394C8010E94E159FF2009F449C0F5
:103760008091CF049091D0040E94C168609391022F
:103770007093920280939302909394026093390C19
:1037800070933A0C80933B0C90933C0CC12C30E529
:10379000D32E33ECE32E37E4F32EC0929902D0926D
:1037A0009A02E0929B02F0929C02C092310CD0925D
:1037B000320CE092330CF092340C20911F11211145
:1037C0000E94FE5F109249111092481180E090E033
:1037D0000E94D144409191025091920260919302D3
:1037E0007091940222E0C8010E94155A63E878E0C3
:1037F00047C16EE878E0C8010E94AB5AC8010E9438
:103800000F63811114C062E978E0CE0101960E9435
:10381000AB5ACE0101960E940F63FF24F3948111ED
:1038200001C0F12CCE0101960E94E15902C0FF2493
:10383000F394C8010E94E159FF2009F474C08091FB
:103840001710909118100497D8F064E070E0CE0142
:1038500001960E946644BE016F5F7F4F85EF9FE037
:103860000E94A859CE0101960E94E1590E94E94E9A
:1038700060939D0270939E0280939F029093A0029A
:1038800060919D0270919E0280919F029091A00292
:1038900060932D0C70932E0C80932F0C9093300C12
:1038A00020911F11222321F042E050E00E94464265
:1038B0008091CF049091D0040E94C16860939502DA
:1038C0007093960280939702909398026093350CC0
:1038D0007093360C8093370C9093380C80911F11A5
:1038E000882381F062EA73E083E79EE00E94D45A65
:1038F0006091950270919602809197029091980242
:103900000E94FE5F109249111092481180E090E0F1
:103910000E94D14440919502509196026091970285
:1039200070919802A7C06EE978E0C8010E94AB5A76
:10393000C8010E940F63811114C062EA78E0CE01D1
:1039400001960E94AB5ACE0101960E940F63FF249C
:10395000F394811101C0F12CCE0101960E94E1592E
:1039600002C0FF24F394C8010E94E159FF2009F42A
:10397000C5C180911710909118100497D8F064E099
:1039800070E0CE0101960E946644BE016F5F7F4FDA
:1039900085EF9FE00E94A859CE0101960E94E1594F
:1039A0000E94E94E6093990270939A0280939B0261
:1039B00090939C028091990290919A02A0919B020F
:1039C000B0919C028093310C9093320CA093330CF5
:1039D000B093340C80911F11882391F069E873E053
:1039E00083E79EE00E94D45A6091990270919A02F6
:1039F00080919B0290919C0242E050E00E944642DE
:103A00008091CF049091D0040E94C168609391028C
:103A10007093920280939302909394026093390C76
:103A200070933A0C80933B0C90933C0C80911F1147
:103A3000882381F06FE773E083E79EE00E94D45A09
:103A40006091910270919202809193029091940200
:103A50000E94FE5F109249111092481180E090E0A0
:103A60000E94D14440919102509192026091930240
:103A70007091940222E0C8010E94155A66E978E02C
:103A8000CE0101960E94AB5AB801CE0101960E9468
:103A90003359BC018BEF9FE00E949359CE010196F0
:103AA0000E94E159C8010E94E1596BEF7FE0CE010D
:103AB00001960E94A35ACE0101960E94FD752CC169
:103AC000CE0183960E94E1590AE010E0C12CD12C6E
:103AD000760166246A9483E0782E6EE170E080E0DF
:103AE00090E00E94965D8091D1040E94715DB301C7
:103AF0000E94DF8E072E000C880B990B0E94148AFF
:103B000020E030E040EA50E40E94738A9B01AC015F
:103B1000C701B6010E949E8B6B017C010150110907
:103B2000E1F620E030E040E251E40E94648C6B0159
:103B30007C0165EB77E0CE0145960E94AB5ACE0141
:103B400045960E940F63811180C169EB77E0CE0139
:103B500001960E94AB5ACE0101960E940F6311E0BC
:103B6000811101C010E0CE0101960E94E159CE0101
:103B700045960E94E159112309F43FC020E030E04E
:103B800040E650E4C701B6010E94738A9B01AC0174
:103B900060E070E080E890E40E949D8BAB01BC0186
:103BA000409304025093050260930602709307024B
:103BB00022E0CE0101960E94155ABE016F5F7F4F31
:103BC0008BEF9FE00E94A859CE0101960E94E15917
:103BD0006DEB77E0CE0101960E94AB5A6BEF7FE070
:103BE000CE0101960E943359BC018BEF9FE00E94E9
:103BF0009359CE0101960E94E1596CEC77E0CE0119
:103C000045960E94AB5ACE0145960E940F638111E2
:103C10001EC161ED77E0CE0101960E94AB5ACE0144
:103C200001960E940F6311E0811101C010E0CE01E6
:103C300001960E94E159CE0145960E94E159112357
:103C400009F43FC020E030E040E650E4C701B6018F
:103C50000E94738A9B01AC0160E070E080E291E415
:103C60000E949D8BAB01BC01409308025093090256
:103C700060930A0270930B0222E0CE0101960E942B
:103C8000155ABE016F5F7F4F8BEF9FE00E94A859CE
:103C9000CE0101960E94E15966ED77E0CE010196D2
:103CA0000E94AB5A6BEF7FE0CE0101960E94335920
:103CB000BC018BEF9FE00E949359CE0101960E94B8
:103CC000E1596FEB7AE0CE0101960E94AB5A6BEF9F
:103CD0007FE0CE0101960E943359BC01CE0145968A
:103CE0000E94A35ACE0145960E94FD75CE014596CD
:103CF0000E94E159CE0101960E94E159BB2011F4C6
:103D00000C94320B63E170E1CE0101960E94A35A3C
:103D1000CE0101960E94546FCE0101960E94E15996
:103D20000C94320B6CEF7AE087E090E10E947E59B0
:103D300080911F11882379F066EA78E083E79EE09E
:103D40000E94C55B612F83E79EE00E94BF5A83E714
:103D50009EE00E94A25B812F0E9414760C94320B8D
:103D60000E94B24928EEC22E23E0D22EE12CF12C83
:103D7000A70196010E946C8BCA01B9010E94128AA8
:103D80002091BE0B3091BF0B4091C00B5091C10BE5
:103D90000E949D8B2091000230910102409102020D
:103DA000509103020E94538D181614F00C94F40BDA
:103DB0000E94B249A70196010E946C8BCA01B90109
:103DC0000E94128A6093BE0B7093BF0B8093C00B4E
:103DD0009093C10B8091DA0B9091DB0B59D064E189
:103DE00070E080E090E00E94965D0C94120C64E616
:103DF00070E080E090E00E94965D0E94B249CB01A5
:103E000068EE73E00E94DF8ECB0164E670E00E94F2
:103E1000DF8E8236910514F40C94DC0B80919D1199
:103E200081110C94DC0B87E090E10E94474F6130D8
:103E300071058105910511F00C94DC0B0E949B73B8
:103E40000C94DC0B10E00C942D0B11E090CE11E0E3
:103E5000F2CECE0183960E94E1590C94860DEA962B
:103E60000FB6F894DEBF0FBECDBFDF91CF911F918B
:103E70000F91FF90EF90DF90CF90BF90AF909F9009
:103E80008F907F906F905F904F903F902F9008950C
:103E90002F923F924F925F926F927F928F929F925A
:103EA000AF92BF92CF92DF92EF92FF920F931F9348
:103EB000CF93DF93CDB7DEB7C555D1090FB6F894D0
:103EC000DEBF0FBECDBF8C01E0901B11F0901C1126
:103ED00080911F11882349F063E776E083E79EE035
:103EE0000E94D45AC8010E948B5FC80105960597AD
:103EF00008F180911B1190911C118017910711F10D
:103F00000E94216D10931C1100931B110E944454B8
:103F10004AE0B801CE0101960E94705ABE016F5F5F
:103F20007F4F87E090E10E94A859CE0101960E9440
:103F3000E15908C00E3F2FEF1207B1F40E9453540D
:103F40000C942F346BE07AE0CE0101960E94AB5ABC
:103F50004AE050E06FEF7FEFCE0101960E94046EC1
:103F6000CE0101960E94E159F8017996E533F105F9
:103F700010F00C941F328827EE58FF4F8F4F0C948F
:103F8000F28E80919D11882309F45EC161E08091D9
:103F9000DD040E94355D60E08091DB040E94355DA8
:103FA0000E948C4760934A1170934B1180934C117F
:103FB00090934D1123E333E948E853E40E94648C65
:103FC00020E030E040E85FE30E949E8B0E94628E1A
:103FD00026E636EA45EA53E40E94738A60934E115E
:103FE00070934F1180935011909351110E940B5276
:103FF000AB01BC0123E0CE0180960E94155ABE01A0
:10400000605E7F4FCE0101960E94A35A6DE07BE077
:10401000CE0101960E941C59BC0185EF9FE00E94D1
:104020009359CE0101960E94E159CE0180960E94DB
:10403000E15967EF7AE0CE0101960E94AB5A65EF35
:104040007FE0CE0101960E943359BC018BEF9FE0C7
:104050000E949359CE0101960E94E1590E940B5291
:104060009B01AC0163966FAF639764963FAF649713
:1040700065964FAF659766965FAF66970E948D49CC
:104080002B013C016EE170E080E090E00E94965DC3
:104090000E940B526B017C010E948D494B015C0117
:1040A00084189508A608B70863962FAD63976496A1
:1040B0003FAD649765964FAD659766965FAD669721
:1040C00081ED881687E09806A104B1040CF43FC086
:1040D000C701B6010E949D8B6B017C0120E030E09E
:1040E000A9010E94538D18165CF426EA3BE944ECC2
:1040F0005BE3C701B6010E940E8A87FF0BC027C091
:1041000026EA3BE944EC5BEBC701B6010E94538D04
:104110001816ECF0C501B40128EE33E040E050E0A1
:104120000E94408BCA01B9010E94148A4B015C01B4
:1041300020E030E04AE754E4C701B6010E94738AE8
:10414000A50194010E94648CAB01BC0103C040E056
:1041500050E0BA0122E0CE0180960E94155ABE01BD
:10416000605E7F4FCE0101960E94A35A6CEA78E010
:10417000CE0101960E941C59BC018FEE9FE00E9467
:104180009359CE0101960E94E159CE0180960E947A
:10419000E15960EB78E0CE0101960E94AB5A6FEED8
:1041A0007FE0CE0101960E943359BC018BEF9FE066
:1041B0000E945259CE0101960E94E1596BE07AE0CB
:1041C000CE0101960E94AB5A6FEE7FE0CE010196C0
:1041D0000E943359BC0185EF9FE00E945259CE01E5
:1041E00001960E94E15964EB78E0CE0101960E94AD
:1041F000AB5A4AE050E060E070E0CE0101960E94C8
:10420000B66ECE0101960E94E15965EF7FE0CE01C6
:1042100001960E94A35A45E050E06FEF7FEFCE0178
:1042200001960E94856DCE0101960E94E1596BEBCB
:1042300078E08BEF9FE00E94445960E08091DD04BC
:104240000E94355D0C944D3260910C0270910D020C
:1042500080910E0290910F020E944D520C944D32AB
:10426000D090C7046CEF7AE0CE01805C9F4F0E9433
:10427000AB5A7E0190E2E90EF11C6D2DC7010E9440
:104280004C4DF886EF821D821E82198289E08A8356
:1042900081E08B838C831C8A1B8ACE0101960E944D
:1042A000A84CCE0101960E943A4BCE0101960E9485
:1042B000CD61EE80F12CA3E0EA16F10409F473C19C
:1042C0006EEC78E0CE01805C9F4F0E947E596CEFCF
:1042D0007AE08BEF9FE00E947E59BE01605C7F4FC9
:1042E000CE018E960E94A35A4AE050E060E070E052
:1042F000CE018E960E94B66ECE018E960E94E15936
:1043000061E080E00E943D4162EF78E0CE01805C98
:104310009F4F0E947E5980E2882E81E1982EAA2428
:10432000A394B12CC12CD12CCE14DF040CF0F1C01D
:104330006C2DCE0101960E943A4CF40121913191ED
:10434000419151914F010E949E8B2B013C0120E035
:1043500030E04CEF52EC0E940E8A87FF21C04AE009
:10436000B501CE018E960E94705A65EA75E0CE01C5
:10437000C4960E94AB5ABE01625D7F4FCE01C496C7
:104380000E94335968ED78E00E941C59BC018BEF04
:104390009FE00E945259CE01C4960E94E15945C047
:1043A00022E0B301A201CE018E960E94155A4AE086
:1043B000B501CE01C4960E94705A65EA75E0CE013F
:1043C000CA960E94AB5ABE016C5C7F4FCE01CA9662
:1043D0000E94335965E576E00E941C59BE01625D7A
:1043E0007F4F0E943359BC018FEE9FE00E9493598A
:1043F000CE01CA960E94E159CE01C4960E94E159AD
:10440000CE018E960E94E1596FEE7FE0CE018E962E
:104410000E94A35A6BE07AE0CE018E960E941C594E
:10442000BC018BEF9FE00E945259CE018E960E94F4
:10443000E159F1E0EF16F10461F4C114D10409F07F
:1044400061C06BEF7FE0CE01805C9F4F0E9493596B
:1044500059C022E0E216F10419F522E0B301A201ED
:10446000CE01C4960E94155ABE016C5C7F4FCE01EE
:104470008E960E94A35A6BE07AE0CE018E960E943F
:104480001C59BC01CE01805C9F4F0E945259CE0145
:104490008E960E94E159CE01C4960E94E15932C025
:1044A00083E0E816F10471F16FEE7FE0CE018E96A5
:1044B0000E94A35A44E150E06FEF7FEFCE018E9649
:1044C0000E94856DCE018E960E94E15967E17AE0E7
:1044D000CE018E960E94AB5ACE018E960E94456DFB
:1044E000CE018E960E94E1598091DA04882351F022
:1044F0008091D904882331F060ED77E080E090E08E
:104500000E94965D9FEFC91AD90AAFEFAA1ABA0A9C
:104510000BCFCE01805C9F4F0E94524F8BEF9FE0EC
:104520000E94524FE114F104A9F467EF73E08BEF9E
:104530009FE00E94585964EE78E0CE018E960E946A
:10454000AB5A4AE050E06FEF7FEFCE018E960E94AB
:10455000856DE7C0B4E0EB16F10414F00C946E32F4
:10456000BE01605C7F4FCE018E960E94A35A4AE046
:1045700050E06FEF7FEFCE018E960E94856DCE01E9
:104580008E960E94E15967E17AE0CE018E960E94F4
:10459000AB5ACE018E960E94456DCE018E960E943A
:1045A000E1590C946E326FEE78E0CE01805C9F4F43
:1045B0000E947E59BE01605C7F4FCE018E960E94A4
:1045C000A35A4AE050E060E070E0CE018E960E946F
:1045D000B66ECE018E960E94E1596CEF7AE08BEFB9
:1045E0009FE00E947E596BEF7FE0CE01805C9F4F81
:1045F0000E949359E12CF12C6E2DCE0101960E9460
:104600003A4C4B015C0122E0AB01BC01CE01E1144C
:10461000F10469F48E960E94155ABE01625D7F4FC7
:1046200085E091E10E94C65ACE018E961CC0C496C8
:104630000E94155ABE016C5C7F4FCE018E960E947F
:10464000A35A6BE07AE0CE018E960E941C59BC0101
:10465000CE01805C9F4F0E945259CE018E960E94DF
:10466000E159CE01C4960E94E15922E0B501A401AE
:10467000CE01C4960E94155ABE016C5C7F4FCE01DC
:104680008E960E94A35A6BE07AE0CE018E960E942D
:104690001C59BC018BEF9FE00E945259CE018E96AF
:1046A0000E94E159CE01C4960E94E159EFEFEE1A43
:1046B000FE0AF3E0EF16F10409F09ECFCE01805C14
:1046C0009F4F0E94524FBE01605C7F4FCE018E967D
:1046D0000E94A35A4AE050E06FEF7FEFCE018E9622
:1046E0000E94856DCE018E960E94E1590E94636DF5
:1046F0008BEF9FE00E94524F65EF78E0CE018E96DF
:104700000E94AB5A6BEF7FE0CE018E960E94335928
:104710006FEF78E00E941C59BC018BEF9FE00E9474
:104720009359CE018E960E94E159CE01805C9F4F35
:104730000C944B328091C9049091CA040E940B647E
:104740000C944D328091CD049091CE040E94B266BB
:104750000C944D3280915002909151020E947D67DD
:104760000C944D320E94B2492B013C0186ED9DE034
:104770000E94BC5C64E670E080E090E00E94965D80
:1047800040E855E260E070E086ED9DE00E947F7AAF
:1047900064E670E080E090E00E94965D63E374E080
:1047A00085EF9FE00E94585965EF7FE0CE010196AA
:1047B0000E94A35A42E350E06FEF7FEFCE010196D3
:1047C0000E94B66ECE0101960E94E15968E274E043
:1047D00085EF9FE00E94585965EF7FE0CE0101967A
:1047E0000E94A35A42E350E06FEF7FEFCE010196A3
:1047F0000E94856DCE0101960E94E15980911D11A4
:1048000090911E118D7F2B961FAE2B97A12CB12C52
:10481000C12CD12CE12CF12C019709F475C0CE01EB
:10482000809628969FAF8EAF2897DE015E962A96D7
:10483000BFAFAEAF2A970E94B249DC01CB01841909
:104840009509A609B709883B9B40A105B10508F069
:104850005BC086ED9DE00E946457892B09F44DC032
:104860008CED95E0A0E0B0E08093DA0D9093DB0D45
:10487000A093DC0DB093DD0D0E94724497FD06C03D
:1048800082349105C9F780E090E002C08FEF9FEF7E
:10489000892B99F5DE0111961D014D010E9472448C
:1048A00097FF06C089818D3441F520E030E00BC0D0
:1048B000D4018D934D012896EEADFFAD2897AE172C
:1048C000BF0761F7EFCFD1018D911D01280F311D79
:1048D0002A96EEADFFAD2A97AE17BF07A1F72E5B64
:1048E0003F4F8E8D90E0982F88274F8D840F911D1C
:1048F0002817390711F40C94763262E370E080E0F7
:1049000090E00E94965D97CF0E94B249DC01CB01F6
:1049100084199509A609B709883B9B40A105B105F3
:1049200028F42B962FAD2B972111C7C00E94216D23
:1049300065EF7FE0CE0180960E94A35A42E350E0EB
:1049400066E070E0CE0180960E94B66ECE01809641
:104950000E94E1592B962FAD2B97222311F40C9432
:10496000913282E090E090931E1180931D114AE0F5
:10497000B501CE0180960E94705A4AE0B601CE0180
:104980008E960E94705A4AE0B701CE01CA960E94E4
:10499000705ABE01665C7F4FCE01C4960E94A35A36
:1049A00064EE77E0CE01C4960E941C59BE01625DA0
:1049B0007F4F0E94335964EE77E00E941C59BE017C
:1049C000605E7F4F0E943359BC018BEF9FE00E94D5
:1049D0009359CE01C4960E94E159CE01CA960E9415
:1049E000E159CE018E960E94E159CE0180960E9437
:1049F000E1596BEF7FE0CE0180960E94A35A4AE016
:104A000050E06FEF7FEFCE0180960E94856DCE0162
:104A100080960E94E15962E179E085E091E10E948F
:104A2000C55B68E179E08BEF9FE00E947E594AE028
:104A3000B501CE0180960E94705A4AE0B601CE01BF
:104A40008E960E94705A4AE0B701CE01CA960E9423
:104A5000705ABE01665C7F4FCE01C4960E94A35A75
:104A60006BE07AE0CE01C4960E941C59BE01625DE3
:104A70007F4F0E9433596BE07AE00E941C59BE01BF
:104A8000605E7F4F0E94335962E179E00E941C59B9
:104A9000BC018BEF9FE00E945259CE01C4960E9448
:104AA000E159CE01CA960E94E159CE018E960E942C
:104AB000E159CE0180960E94E15962E370E080E006
:104AC00090E00E94965D86ED9DE00E94BC5C0C9497
:104AD000EF2DE090CF04F090D0046FE374E085EF09
:104AE0009FE00E9458590E94216D65EF7FE0CE0142
:104AF00001960E94A35A4AE050E06FEF7FEFCE018B
:104B000001960E94B66ECE0101960E94E159C7013E
:104B10000E94C16862966CAF7DAF8EAF9FAF629707
:104B20008090950290909602A0909702B090980283
:104B3000A50194016091910270919202809193027B
:104B4000909194020E949D8B2B013C0120E030E06B
:104B5000A9010E940E8A882309F45BC0C0909D02BF
:104B6000D0909E02E0909F02F090A00220E030E002
:104B7000A901C701B6010E940E8A18160CF049C09F
:104B80008091990290919A02A0919B02B0919C020F
:104B90002E968CAF9DAFAEAFBFAF2E979C01AD01EF
:104BA000C701B6010E940E8A882399F1A7019601D8
:104BB0002E966CAD7DAD8EAD9FAD2E970E94648C10
:104BC0000E949F8D2E966CAF7DAF8EAF9FAF2E97BC
:104BD000A501940162966CAD7DAD8EAD9FAD6297DF
:104BE0000E949D8BA30192010E94648C2E962CAD95
:104BF0003DAD4EAD5FAD2E970E94738A0E94D18C61
:104C00009B01AC01C701B6010E94738A6B017C0154
:104C100003C0C12CD12C760165EF7FE0CE01019657
:104C20000E94A35A4AE050E060E070E0CE01019695
:104C30000E94B66ECE0101960E94E15920E030E656
:104C40004AEE56E4C701B6010E94538D18163CF493
:104C500068E279E08BEF9FE00E947E5925C021E059
:104C6000B701A601CE0180960E94155A67E379E04C
:104C7000CE0101960E94AB5ABE01605E7F4FCE010D
:104C800001960E9433596BE379E00E941C59BC01E4
:104C90008BEF9FE00E949359CE0101960E94E1594B
:104CA000CE0180960E94E1596BEF7FE0CE01019624
:104CB0000E94A35A4AE050E06FEF7FEFCE010196C9
:104CC0000E94856DCE0101960E94E15964E670E074
:104CD00080E090E00E94965D80919D11882311F400
:104CE0000C944D3260E273E080E090E00C94C432AA
:104CF000E090D704F090D8040E94216DC7010E9473
:104D0000CC567C0162E370E080E090E00E94965D0A
:104D1000B701FF0C880B990B0E94148A20E030E049
:104D200040EA50E40E94738A20E030EC4FE754E4FC
:104D30000E94648CAB01BC0123E0CE0101960E946D
:104D4000155A68E17BE0CE0180960E94AB5ABE0105
:104D50006F5F7F4FCE0180960E9433596BE276E001
:104D60000E941C59BC018BEF9FE00E949359CE0119
:104D700080960E94E159CE0101960E94E1596FE3AD
:104D800079E085EF9FE00E947E5965EF7FE0CE01DC
:104D900001960E94A35A4AE050E068E070E0CE011C
:104DA00001960E94B66ECE0101960E94E1596BEF0A
:104DB0007FE0CE0101960E94A35A4AE050E06FEFD7
:104DC0007FEFCE0101960E94856DCE0101960E9473
:104DD000E15965EF7FE08BEF9FE00E9452597CCF55
:104DE0009091000C81E089278093000C80919D11A7
:104DF000882331F06BEF7FE089E39DE00E94B55B93
:104E000068EC70E080E090E00C94C43210929D1148
:104E10000C944D3281E080939D1167E070E18DE04C
:104E200090E10E94935980911B1190911C119093D5
:104E3000DB0B8093DA0B0C944D328091970C9091A0
:104E4000980C892B09F567E479E0CE0180960E94E1
:104E5000AB5A6FEF70E1CE0180960E943359BC01CE
:104E6000CE0101960E94A35A48EC50E06FEF7FEF0D
:104E7000CE0101960E94B66ECE0101960E94E159C4
:104E8000CE0180960E94E1598091970C9091980CE8
:104E9000019709F56BE479E0CE0180960E94AB5A48
:104EA0006FEF70E1CE0180960E943359BC01CE01B4
:104EB00001960E94A35A48EC50E06FEF7FEFCE01BD
:104EC00001960E94B66ECE0101960E94E159CE0174
:104ED00080960E94E15961E579E0CE0180960E94BA
:104EE000AB5A69EF70E1CE0180960E943359BC0144
:104EF000CE0101960E94A35A40ED57E06FEF7FEF7D
:104F0000CE0101960E94856DCE0101960E94E15965
:104F1000CE0180960E94E15980911D1190911E1141
:104F2000019719F465EA75E002C067E975E0CE0102
:104F300001960E949B5A48EC50E06FEF7FEFCE0144
:104F400001960E94046ECE0101960E94E15967E825
:104F500075E0CE0101960E949B5A40ED57E06FEF3D
:104F60007FEFCE0101960E94856DCE0101960E94D1
:104F7000E15967E775E0CE0101960E949B5A48EC23
:104F800050E06FEF7FEFCE0101960E94046ECE01DC
:104F900001960E94E1596AE675E0CE0101960E94F1
:104FA0009B5A40ED57E06FEF7FEFCE0101960E94D4
:104FB000856DCE0101960E94E1596DE575E0CE0147
:104FC00001960E949B5A48EC50E06FEF7FEFCE01B4
:104FD00001960E94046ECE0101960E94E15962E59D
:104FE00075E0CE0101960E949B5A40ED57E06FEFAD
:104FF0007FEFCE0101960E94856DCE0101960E9441
:10500000E15966E475E0CE0101960E949B5A48EC96
:1050100050E06FEF7FEFCE0101960E94046ECE014B
:1050200001960E94E15965E375E0CE0101960E9468
:105030009B5A40ED57E06FEF7FEFCE0101960E9443
:10504000856DCE0101960E94E15980911D119091CC
:105050001E11039719F46AE275E002C060E275E080
:10506000CE0101960E949B5A48EC50E06FEF7FEF13
:10507000CE0101960E94046ECE0101960E94E15974
:1050800065E175E0CE0101960E949B5A40ED57E024
:105090006FEF7FEFCE0101960E94856DCE010196E4
:1050A0000E94E15968E075E0CE0101960E949B5A8A
:1050B00048EC50E06FEF7FEFCE0101960E94046E46
:1050C000CE0101960E94E15969EF74E0CE0101968C
:1050D0000E949B5A40ED57E06FEF7FEFCE010196A3
:1050E0000E94856DCE0101960E94E1596EEE74E03A
:1050F000CE0101960E949B5A48EC50E06FEF7FEF83
:10510000CE0101960E94046ECE0101960E94E159E3
:1051100061EE74E0CE0101960E949B5A40ED57E08B
:105120006FEF7FEFCE0101960E94856DCE01019653
:105130000E94E15980911D1190911E11029719F45E
:1051400060ED74E002C060EC74E0CE0101960E9454
:105150009B5A48EC50E06FEF7FEFCE0101960E9422
:10516000046ECE0101960E94E15963EB74E0CE011A
:1051700001960E949B5A40ED57E06FEF7FEFCE0102
:1051800001960E94856DCE0101960E94E15967EA61
:1051900074E0CE0101960E949B5A48EC50E06FEFFC
:1051A0007FEFCE0101960E94046ECE0101960E940F
:1051B000E15967E974E0CE0101960E949B5A40EDE7
:1051C00057E06FEF7FEFCE0101960E94856DCE0113
:1051D00001960E94E1596CE874E0CE0101960E94AC
:1051E0009B5A48EC50E06FEF7FEFCE0101960E9492
:1051F000046ECE0101960E94E15962E874E0CE018E
:1052000001960E949B5A40ED57E06FEF7FEFCE0171
:1052100001960E94856DCE0101960E94E15962E7D8
:1052200074E0CE0101960E949B5A48EC50E06FEF6B
:105230007FEFCE0101960E94046ECE0101960E947E
:10524000E15965E674E0CE0101960E949B5A40ED5B
:1052500057E06FEF7FEFCE0101960E94856DCE0182
:1052600001960E94E15969E574E0CE0101960E9421
:105270009B5A48EC50E06FEF7FEFCE0101960E9401
:10528000046ECE0101960E94E15969E474E0CE01FA
:1052900001960E949B5A40ED57E00C94433286EDF4
:1052A0009DE00E94BC5C40E052EC61E070E086ED65
:1052B0009DE00E947F7A8CED95E0A0E0B0E08093C5
:1052C000DA0D9093DB0DA093DC0DB093DD0D64E659
:1052D00070E080E090E00E94965D66E579E08BEFFB
:1052E0009FE00E947E596BEF7FE0CE0101960E9405
:1052F000A35ACE0101960E94546FCE0101960E94DE
:10530000E15962E370E080E090E00E94965D6BEF0F
:105310007FE0CE0101960E94A35A42E350E06FEF76
:105320007FEFCE0101960E94B66ECE0101960E94DB
:10533000E15962E679E085EF9FE00E947E5965EFD2
:105340007FE0CE0101960E94A35A44E150E06FEF46
:105350007FEFCE0101960E94856DCE0101960E94DD
:10536000E15980911D1190911E11019739F484E04B
:1053700090E00E94D8656B017C0103C0C12CD12C48
:10538000760180911D1190911E11892B31F481E0DD
:1053900090E00E94D8656B017C0120E030E040EA9B
:1053A00051E4C701B6010E94538D181664F521E03F
:1053B000B701A601CE0101960E94155A69EA77E06D
:1053C000CE0180960E94AB5ABE016F5F7F4FCE0127
:1053D00080960E9433596EE679E00E941C59BC0108
:1053E0008BEF9FE00E949359CE0180960E94E15975
:1053F000CE0101960E94E15981E090E090931E1148
:1054000080931D1110C061E779E08BEF9FE00E944F
:105410007E5980911D1190911E11019721F41092D7
:105420001E1110921D116BEF7FE0CE0101960E94BC
:10543000A35A4AE050E060E070E0CE0101960E947D
:10544000B66ECE0101960E94E1596BEF7FE0CE016E
:1054500001960E94A35A6BE07AE0CE0101960E9469
:105460001C5965EF7FE00E943359BC018BEF9FE030
:105470000E949359CE0101960E94E15986ED9DE06C
:105480000E94BC5C29CC60E176E0CE0101960E94CE
:105490009B5A4AE050E06FEF7FEFCE0101960E94E9
:1054A000856DCE0101960E94E1590E94045FA12CF6
:1054B000B12C64E670E080E090E00E94965D0E946E
:1054C000045F6B017C019FEFA91AB90AA3E0AA1639
:1054D000B1047CF3A7019601C701B601BAE0AB168F
:1054E000B10414F00C94BD320E94A38E8111E1CF5F
:1054F00020E030E046E153E4C701B6010E940E8A85
:1055000087FD02C00C94C7320E94045F6093B21101
:105510007093B3118093B4119093B5110E94C05E43
:105520006093AE117093AF118093B0119093B1114D
:105530004091B2115091B3116091B4117091B511B5
:1055400021E0CE0101960E94155A62EF78E0CE016B
:1055500080960E94AB5ABE016F5F7F4FCE0180964E
:105560000E943359BC018BEF9FE00E949359CE01FA
:1055700080960E94E159CE0101960E94E159409126
:10558000AE115091AF116091B0117091B11121E045
:10559000CE0101960E94155A65EF79E0CE01809602
:1055A0000E94AB5ABE016F5F7F4FCE0180960E9472
:1055B0003359BC018BEF9FE00E945259CE01809677
:1055C0000E94E159CE0101960E94E15962E27BE01E
:1055D0008BEF9FE00E9444596CEF7AE0CE01019678
:1055E0000E94AB5A44E150E060E070E0CE010196C9
:1055F0000E94B66ECE0101960E94E1596091B211EF
:105600007091B3118091B4119091B5110E94FD8CED
:105610004AE0CE0101960E94705ABE016F5F7F4F33
:1056200085EF9FE00E94A859CE0101960E94E159A2
:1056300060E086E00E943D4165EF7FE085E091E11A
:105640000E94C65A6FED85E091E10E94BF5A63E85F
:1056500079E085E091E10E94C55B6091AE117091A7
:10566000AF118091B0119091B1110E94FD8C4AE070
:1056700050E085E091E10E949C5B62E27BE085E086
:1056800091E10E94C55B64E670E080E090E07CC739
:1056900080917602882309F400C76CEF7AE0CE018E
:1056A00001960E94AB5A4AE050E061E070E0CE0102
:1056B00001960E94B66ECE0101960E94E1590E94A9
:1056C000216D0E94B4452B013C010E948C474B0187
:1056D0005C016091A9027091AA028091AB02909145
:1056E000AC020E94148A9B01AC0163966FAF639772
:1056F00064963FAF649765964FAF659766965FAFC8
:1057000066970E94B4450E94148A63962FAD6397F2
:1057100064963FAD649765964FAD659766965FADAD
:1057200066970E94648C21E03EED42E45EE30E94B5
:10573000128E9B01AC0160E070E080E89FE30E9464
:105740009D8B20E03AE24DE257E40E94738A6B01A0
:105750007C01C301B2010E94148A20E030E048ECD1
:1057600052E40E94648CAB01BC0122E0CE010196A0
:105770000E94155ABE016F5F7F4F8FEE9FE00E941F
:10578000A859CE0101960E94E1596CE077E08FEEB6
:105790009FE00E9444596FEE7FE085EF9FE00E94FA
:1057A000935968E077E0CE0101960E94AB5A6FEE04
:1057B0007FE0CE0101960E943359BC018FEE9FE03D
:1057C0000E949359CE0101960E94E15962EF78E060
:1057D0008BEF9FE00E947E5921E0B501A401CE012C
:1057E00001960E94155ABE016F5F7F4F8BEF9FE0BD
:1057F0000E945259CE0101960E94E1596DE779E06D
:105800008BEF9FE00E94445921E0B701A601CE0131
:1058100080960E94155ABE01605E7F4FCE010196B0
:105820000E94A35A6DE07BE0CE0101960E941C59B4
:10583000BC018BEF9FE00E945259CE0101960E945D
:10584000E159CE0180960E94E1596FEE7FE0CE01D2
:1058500001960E94A35A6BE07AE0CE0101960E9465
:105860001C596BEF7FE00E943359BC018BEF9FE026
:105870000E949359CE0101960E94E15965EF7FE0A5
:10588000CE0101960E94A35A4AE050E060E070E029
:10589000CE0101960E94B66ECE0101960E94E1599A
:1058A00021E0B501A401CE0101960E94155ABE0166
:1058B0006F5F7F4F81E090E10E94A859CE01019671
:1058C0000E94E15961E070E1CE0101960E94A35A65
:1058D0004AE050E06FEF7FEFCE0101960E94856DA8
:1058E000CE0101960E94E15963E879E0CE0101966C
:1058F0000E94AB5ACE0101960E94456DCE010196E1
:105900000E94E15921E0B701A601CE0180960E94D4
:10591000155ABE01605E7F4FCE0101960E94A35AC8
:105920006DE07BE0CE0101960E941C59BC0181E034
:1059300090E10E949359CE0101960E94E159CE0157
:1059400080960E94E15961E070E1CE0101960E94CB
:10595000A35A4AE050E068EF7FEFCE0101960E9423
:10596000856DCE0101960E94E15980919D11882399
:1059700009F493C568E572E080E090E005C6809187
:105980009D11882331F0A2E04A2E512C612C712CFC
:1059900005C0FEE14F2E512C612C712C6EE176E09A
:1059A0008BEF9FE00E9458596BEF7FE0CE0101968C
:1059B0000E94A35A4AE050E06FEF7FEFCE010196BC
:1059C0000E94856DCE0101960E94E159812C912C97
:1059D0005401C12CD12C760183E20E94224187E040
:1059E00090E00E941D410E94C04066E970E080E0A6
:1059F00090E00E94965D83E20E94224180E290E066
:105A00000E941D410E94C04066E970E080E090E085
:105A10000E94965D62E070E083E290E00E9446455D
:105A200040E050E0BA018091ED0C90E02091EE0C46
:105A3000821B9109181619062CF580E19FE06596E6
:105A40004FAF659766965FAF669763966FAF639744
:105A500064967FAF64970E94F34F65964FAD65974C
:105A600066965FAD669763966FAD639764967FADFC
:105A70006497762F652F542F4427480F511D611DC1
:105A8000711DD1CFCB01BA010E94148A2AE939E9EC
:105A900049E95FE30E94648C0E94FD8CAB01BC016C
:105AA000C416D506E606F70614F46A017B012AE05F
:105AB000CE0180960E94445ABE01605E7F4FCE01A7
:105AC00001960E94A35A66E879E0CE0101960E94F1
:105AD0001C59BC0185EF9FE00E949359CE010196AD
:105AE0000E94E159CE0180960E94E15965EF7FE066
:105AF000CE0101960E94A35A4EE150E060E070E0B2
:105B0000CE0101960E94046ECE0101960E94E159D9
:105B1000EFEF8E1A9E0AAE0ABE0A481459046A04B0
:105B20007B040CF059CF2AE0B701A601CE01809684
:105B30000E94445ABE01605E7F4FCE0101960E94D2
:105B4000A35A66E879E0CE0101960E941C59BC0177
:105B500085EF9FE00E949359CE0101960E94E15982
:105B6000CE0180960E94E15965EF7FE0CE0101965B
:105B70000E94A35A4AE050E060E070E0CE01019636
:105B80000E94B66ECE0101960E94E1592AE0B7014B
:105B9000A601CE0101960E94445A6AE879E0CE013E
:105BA00080960E94AB5ABE016F5F7F4FCE018096F8
:105BB0000E9433596DE879E00E941C596BEF7FE039
:105BC0000E943359BC018BEF9FE00E949359CE0194
:105BD00080960E94E159CE0101960E94E15962E34C
:105BE00070E080E090E0D0C4E090D504F090D6045E
:105BF00081E08093DF0464E670E080E090E00E9442
:105C0000965D0E94216DC7010E94CC5660E074E051
:105C1000681B790B4AE0CE0101960E94705A62E936
:105C200079E0CE0180960E94AB5ABE016F5F7F4F34
:105C3000CE0180960E943359BC018BEF9FE00E94F9
:105C40009359CE0180960E94E159CE0101960E949F
:105C5000E15960E086E00E943D416EE276E0CE01CF
:105C600001960E949B5A42E350E068E070E0CE014A
:105C700001960E94B66ECE0101960E94E1596BEF2B
:105C80007FE0CE0101960E94A35A42E350E06FEFFD
:105C90007FEFCE0101960E94856DCE0101960E9494
:105CA000E15969E979E0C7C08091D3049091D404A7
:105CB0000E94CC567C019093DD0B8093DC0B62E359
:105CC00070E080E090E00E94965D4AE0B701CE016E
:105CD00001960E94705ABE016F5F7F4F8BEF9FE06D
:105CE0000E94A859CE0101960E94E15980915F104F
:105CF00090916010892B09F45DC06BE570E1CE01D5
:105D000080960E94A35ABE01605E7F4FCE0101962D
:105D10000E94A35A44E150E060E070E0CE01019699
:105D20000E94B66ECE0101960E94E15963EA79E0C5
:105D3000CE0101960E94AB5A6BEF7FE0CE01019637
:105D40000E943359BC0185EF9FE00E949359CE0118
:105D500001960E94E15965EF7FE0CE0101960E9415
:105D6000A35A44E150E06FEF7FEFCE0101960E940D
:105D7000856DCE0101960E94E159BE01605E7F4FA4
:105D8000CE0101960E94A35A6BE07AE0CE01019603
:105D90000E941C5965EF7FE00E943359BC018BEFD4
:105DA0009FE00E949359CE0101960E94E159CE01D5
:105DB000809652C06EEA79E085EF9FE00E947E599E
:105DC00065EF7FE0CE0101960E94A35A44E150E0C6
:105DD00060E070E0CE0101960E94B66ECE010196A1
:105DE0000E94E15962E979E0CE0101960E94AB5A26
:105DF0006BEF7FE0CE0101960E943359BC0185EF25
:105E00009FE00E949359CE0101960E94E15965EFEF
:105E10007FE0CE0101960E94A35A44E150E06FEF6B
:105E20007FEFCE0101960E94856DCE0101960E9402
:105E3000E15963EA79E0CE0101960E94AB5A6BEF1B
:105E40007FE0CE0101960E943359BC018BEF9FE0A9
:105E50000E949359CE0101960E94E1590C946C2640
:105E600080917602882309F418C380919D118823BC
:105E700029F082E090E00E94806F0FC3C0900C0276
:105E8000D0900D02E0900E02F0900F0220E030E082
:105E900040E450E4C701B6010E94538D18166CF41B
:105EA00020E030E04AE754E4C701B6010E94738A5B
:105EB0000E94FD8C6B017C0106C060E3C62E65E785
:105EC000D62EE12CF12C0E94216D60E080E00E9432
:105ED0003D4162EB79E085E091E10E94C55B61E0C4
:105EE00080E00E943D4163EC79E085E091E10E9411
:105EF000C55B64E670E080E090E00E94965D0E94E1
:105F0000B2496093D60B7093D70B8093D80B9093C4
:105F1000D90B0E94B2498090D60B9090D70BA090DD
:105F2000D80BB090D90BDC01CB0188199909AA09CB
:105F3000BB098C159D05AE05BF050CF0AEC283E014
:105F400090E00E94806F0E94B24964E170E080E0BE
:105F500090E00E94965DDDCF80919D11811102C07D
:105F60000E94216D86ED9DE00E94BC5C64E670E0BD
:105F700080E090E00E94965D61E576E085EF9FE02D
:105F80000E94585965EF7FE0CE0101960E94A35A06
:105F900044E150E060E070E0CE0101960E94B66EF0
:105FA000CE0101960E94E15962E476E085EF9FE020
:105FB0000E94585965EF7FE0CE0101960E94A35AD6
:105FC00044E150E06FEF7FEFCE0101960E94856DB6
:105FD000CE0101960E94E1598CE40E9483606B011E
:105FE0007C0154E0A52EB12CA7019601C701B60192
:105FF0000E94A38E882309F485C3F1E0AF1AB1088B
:1060000009F40EC364E670E080E090E00E94965DC3
:106010008CE40E9483606B017C01E6CF6DE576E045
:1060200085EF9FE00E94585965EF7FE0CE01019611
:106030000E94A35A4AE050E060E070E0CE01019671
:106040000E94B66ECE0101960E94E1598091D10462
:106050002B968FAF2B978091F80B81110DC00E946A
:10606000B2496093F40B7093F50B8093F60B909309
:10607000F70B81E08093F80B8091EC0B81110DC040
:106080000E94B2496093E80B7093E90B8093EA0B8E
:106090009093EB0B81E08093EC0B1092E70B109246
:1060A000E60B2090E60B3090E70BA8E22A163104AD
:1060B0000CF086C02B968FAD2B970E94715DF1017D
:1060C000EE0FFF1FE356F34F918380830E946D42D2
:1060D00020E030E040EA50E40E94738A20E030E0A3
:1060E00040E85AE30E94738A6B017C016093E20BE3
:1060F0007093E30B8093E40B9093E50B40900402C4
:10610000509005026090060270900702A301920170
:10611000609108027091090280910A0290910B022D
:106120000E949D8B9B01AC0160E070E080EC90E4EC
:106130000E949D8B4B015C0120E030E0A9010E9490
:106140000E8A20E030E040E650E4811105C0C7012E
:10615000B6010E94738A1EC0C701B6010E94738AED
:10616000A30192010E949E8B20E030E040E850E4C1
:106170000E949D8BA50194010E94648C20E030E078
:1061800040EC50E40E94738A20E030E040E850E4A4
:106190000E949E8B6093DE0B7093DF0B8093E00B6D
:1061A0009093E10B64E170E080E090E00E94965DE6
:1061B0009FEF291A390A3092E70B2092E60B71CF34
:1061C000C090DE0BD090DF0BE090E00BF090E10B85
:1061D00020E030E0A901C701B6010E94538D87FD80
:1061E0001EC022E0B701A601CE0101960E94155AF9
:1061F0006BEC79E0CE0180960E94AB5ABE016F5FD6
:106200007F4FCE0180960E943359BC018BEF9FE0F7
:106210000E949359CE0180960E94E15928C16FECEB
:1062200079E08BEF9FE00E947E5925C18091760234
:10623000882309F432C180919D11811127C0C0903B
:106240000C02D0900D02E0900E02F0900F0220E0C0
:1062500030E04AE754E4C701B6010E94738A0E9405
:10626000FD8C4B015C0120E030E040EA50E4C701C6
:10627000B6010E94738A20E030E040EA50E40E94B8
:106280009E8B0E94FD8CA501940108C021E030E0A6
:1062900040E050E06AE070E080E090E00E94E86852
:1062A000FCC08091970C9091980C892BF1F581E0BE
:1062B00090E09093980C8093970C6EED79E0CE016E
:1062C00001960E94AB5ACE0101960E94546FCE01F6
:1062D00001960E94E1596BE479E0CE0101960E949B
:1062E000AB5A6FEF70E1CE0101960E943359BC01A9
:1062F000CE0180960E94A35A48EC50E06FEF7FEFEA
:10630000CE0180960E94B66ECE0180960E94E15921
:10631000CE0101960E94E15989E39DE00E94BC5C98
:1063200040E052EC61E070E03BC01092980C10929B
:10633000970C67EE79E0CE0101960E94AB5ACE0130
:1063400001960E94546FCE0101960E94E15967E4C4
:1063500079E0CE0101960E94AB5A6FEF70E1CE0159
:1063600001960E943359BC01CE0180960E94A35A27
:1063700048EC50E06FEF7FEFCE0180960E94B66E42
:10638000CE0180960E94E159CE0101960E94E1590A
:1063900089E39DE00E94BC5C40E855E260E070E06B
:1063A00089E39DE00E947F7A109249111092481172
:1063B00080E090E00E94D14461E579E0CE01019651
:1063C0000E94AB5A69EF70E1CE0101960E943359E9
:1063D000BC01CE0180960E94A35A40ED57E06FEFBA
:1063E0007FEFCE0180960E94856DCE0180960E943F
:1063F000E1594FC080919B0C90919C0C892BA1F48A
:1064000081E090E090939C0C80939B0C8EED93E048
:1064100090934911809348110E94AA4468EC70E05F
:1064200080E090E00E94965DE0E0F0E0199535C0D4
:106430000E94A7620E94216D0E9444542EC0F092D7
:106440001C11E0921B1166E676E08BEF9FE00E9444
:1064500058596CEF7AE0CE0101960E94AB5A4AE09F
:1064600050E060E070E0CE0101960E94B66ECE0171
:1064700001960E94E1596BEF7FE0CE0101960E94E8
:10648000A35A4AE050E06FEF7FEFCE0101960E94E1
:10649000856DCE0101960E94E1598091FF0F909188
:1064A00000100097A1F0419720F4023011050CF084
:1064B000A4C06BEF7FE0CE0101960E94A35ACE01EB
:1064C00001960E94FD75CE0101960E94E15964E695
:1064D00070E080E090E00E94965DC1C16FEF78E0CF
:1064E0008BEF9FE00E9444590C949523EC80F12C93
:1064F000FE2CEE248D81E80EF11CCE80D12CDC2CFC
:10650000CC248F81C80ED11CA884B12CBA2CAA240B
:106510008985A80EB11C21E02B962FAF2B970C94E8
:106520007D246DE174E08BEF9FE00E9458596BEF82
:106530007FE0CE0180960E94A35A4AE050E060E0DE
:1065400070E0CE0180960E94856DCE0180960E94FB
:10655000E1596AE074E08BEF9FE00E945859809106
:106560001D1190911E11029711F00C945D2510924F
:106570001E1110921D110C945D250E94A38E88237C
:1065800011F40C94782A03C00E94965D86CFA7016F
:106590009601C701B6010E94A38E811115C062E069
:1065A00076E0CE0101960E949B5A4AE050E060E0FE
:1065B00070E0CE0101960E94B66ECE0101960E9457
:1065C000E1596FED75E014C064ED75E0CE01019600
:1065D0000E949B5A4AE050E060E070E0CE010196D4
:1065E0000E94B66ECE0101960E94E15964EB75E0FF
:1065F0008BEF9FE00E94585950CF6BEF7FE0CE01A8
:1066000001960E94A35A4AE050E06FEF7FEFCE015F
:1066100001960E94856DCE0101960E94E15949CFF5
:1066200067E376E085EF9FE00E94585965EF7FE0D1
:10663000CE0101960E94A35A4AE050E060E070E06B
:10664000CE0101960E94B66ECE0101960E94E159DC
:106650006BEF79E0CE0101960E94AB5A65EF7FE0C7
:10666000CE0101960E943359BC018BEF9FE00E943E
:106670009359CE0101960E94E15980911D1190918C
:106680001E11039751F510921E1110921D1125C075
:106690006CEF7AE081E090E10E947E5961E070E168
:1066A000CE0101960E94A35A6BE07AE0CE010196DA
:1066B0000E941C596BEF7FE00E943359BC018BEFA5
:1066C0009FE00E949359CE0101960E94E15983E018
:1066D00090E090931E1180931D1164E670E080E0BD
:1066E00090E00E94965D80919D11882331F060E2D8
:1066F00073E080E090E00E94965D89E39DE00E9457
:10670000F257CBCE21E0B701A601CE0101960E943F
:10671000155A6DE07AE0CE0180960E94AB5ABE0118
:106720006F5F7F4FCE0180960E943359BC018BEF83
:106730009FE00E949359CE0180960E94E159CE01BC
:1067400001960E94E1596BEF7FE0CE0101960E9415
:10675000A35A42E350E06FEF7FEFCE0101960E9413
:10676000856DCE0101960E94E1590E94636D66E13C
:106770007AE08BEF9FE00E94445986E60E94836096
:106780006B017C0184E0A82EB12CA7019601C70102
:10679000B6010E94A38E882389F021E0A21AB108D5
:1067A00009F476CF68EC70E080E090E00E94965D9E
:1067B00086E60E9483606B017C01E7CF21E0B70190
:1067C000A601CE0101960E94155A62EF78E0CE0133
:1067D00080960E94AB5ABE016F5F7F4FCE018096BC
:1067E0000E943359BC0181E090E10E949359CE018F
:1067F00080960E94E159CE0101960E94E1596BE01A
:106800007AE0CE0101960E94AB5A61E070E1CE01C0
:1068100001960E943359BC0185EF9FE00E94935975
:10682000CE0101960E94E15965EF7FE0CE0101960D
:106830000E94A35A4AE050E060E070E0CE01019669
:106840000E94046ECE0101960E94E1590E94636D80
:1068500066E17AE081E090E10E9444591FCFCB5A73
:10686000DF4F0FB6F894DEBF0FBECDBFDF91CF91E3
:106870001F910F91FF90EF90DF90CF90BF90AF905E
:106880009F908F907F906F905F904F903F902F9050
:1068900008952F923F924F925F926F927F928F92C4
:1068A0009F92AF92BF92CF92DF92EF92FF920F939F
:1068B0001F93CF93DF93CDB7DEB728970FB6F89429
:1068C000DEBF0FBECDBFFC0183E29FE093878287CE
:1068D0008091200F90E0958784878091ED0F90E064
:1068E0009787868780911C0F853009F0B7C3809108
:1068F000250F9091260F885891098D35910588F4C0
:106900008091200F843041F48091270F9091280FBF
:106910008097479708F407C28091200F843408F0CD
:10692000E8C18091200F8A3108F448C08091230F7C
:106930009091240F843F914050F4118610868FEF80
:106940009FEFDC0184839583A683B78351C0809138
:10695000250F9091260F85974B9780F519E2E12E30
:106960001FE0F12E82E090E040E050E0BA018C019F
:106970000F5F1F4F2091200F30E0021713076CF4B8
:10698000970122503109D9012D913C9127503109AD
:106990002730310508F40AC2C801019795958795FB
:1069A000918780870C971CF41186108607C044835A
:1069B00055836683778384E090E01CC18091200F2B
:1069C0008A3108F448C08091230F9091240F8032BF
:1069D000934008F4B2CF8091250F9091260FC6976F
:1069E000869708F403C237C0448355836683778350
:1069F0008BE090E0FFC0D7012D913C9125523109E9
:106A00002B31310508F004C2440F551F661F771F54
:106A100041600296B4E0EB0EF11C8C010F5F1F4F3A
:106A20002091200F30E00217130764F497012250E1
:106A30003109D9012D913C912C5031092B30310570
:106A4000D0F2C801019795958795918780870C971B
:106A50005CF6118610868091200F823208F44CC0BB
:106A60008091250F9091260F0697079708F044C054
:106A700049E2C42E4FE0D42E82E090E040E050E0A6
:106A8000BA018C010F5F1F4F2091200F30E00217D9
:106A900013070CF5D6011297ED90FC9011979D010C
:106AA000BEE1EB1AF108A7E1EA16F10408F0BEC155
:106AB000440F551F661F771F4160D6012D913C91F1
:106AC000B4E0CB0ED11C235031092530310510F430
:106AD0000296D7CFC80101979595879591878087B2
:106AE00040971CF41186108607C044835583668343
:106AF00077838CE090E07EC07F011C821B8281E066
:106B000090E09A8389838091200F8D3008F475C0BE
:106B100029E733E0AE014D5F5F4FBE016F5F7F4FEE
:106B2000CF010E940A79892B09F067C029E733E079
:106B3000AE014D5F5F4FBE016F5F7F4FC7010E9487
:106B40000A79019709F059C029E733E0AE014D5F9A
:106B50005F4FBE016F5F7F4FC7010E940A79892B8B
:106B600009F04BC0812C912C540100E010E0809181
:106B7000200F90E029813A81281739077CF529E711
:106B800033E0AE014D5F5F4FBE016F5F7F4FC701C6
:106B90000E940A796C0129E733E0AE014D5F5F4F37
:106BA000BE016F5F7F4FC7010E940A79E1E0CE16F8
:106BB000D10449F4892B09F5880C991CAA1CBB1C2B
:106BC000689480F808C0CD28C1F40197B1F4880C0E
:106BD000991CAA1CBB1C0F5F1F4FC9CFD701199668
:106BE0001C930E931897F70184829582A682B78230
:106BF00081E090E09183808329C21C821B8281E026
:106C000090E09A838983D7011C968D919C911D9762
:106C1000181619060CF061C01A96ED91FC911B979D
:106C200082E090E09A8389838281938189974E974D
:106C300008F053C083E090E09A8389838481958132
:106C40000B970A9708F049C02CEB31E0AE014D5F7D
:106C50005F4FBE016F5F7F4FC7010E940A79892B8A
:106C6000E1F52CEB31E0AE014D5F5F4FBE016F5F90
:106C70007F4FC7010E940A79019779F5412C512C69
:106C8000320100E010E029813A81D7011C968D91F4
:106C90009C911D97281739070CF010C12CEB31E09F
:106CA000AE014D5F5F4FBE016F5F7F4FC7010E9416
:106CB0000A795C010330110509F0C6C02CEB31E004
:106CC000AE014D5F5F4FBE016F5F7F4FC7010E94F6
:106CD0000A79A816B90609F4B7C0D7011A96ED913A
:106CE000FC911B9782819381C697869708F4F2C026
:106CF0003EC18091270F9091280F825491098E9761
:106D000008F00FCE20E030E0C12CD12C7601A90193
:106D1000475D504FDA014D915C914950510949301E
:106D2000510598F0FECD8091290F90912A0F099777
:106D3000099708F0F1CD118610868FEF9FEFDC01E7
:106D400084839583A683B7838CC1B901655D704F39
:106D5000DB014D915C914751510942315105C0F41D
:106D6000D701C601880F991FAA1FBB1F6C017D01A7
:106D70006894C0F82C5F3F4F2038310541F620E27F
:106D800030E031872087C482D582E682F78269C1EC
:106D9000DB014D915C91465051094730510508F097
:106DA000C0CDCC0CDD1CEE1CFF1CE4CFD7012D9117
:106DB0003C91235131092F30310550F4440F551FB8
:106DC000661F771F41600296B4E0EB0EF11CCFCD39
:106DD000D7012D913C912A5031092930310508F015
:106DE000EDCD440F551F661F771FEDCF8091270F04
:106DF0009091280FC697869708F02DCE8BE2E82E4B
:106E00008FE0F82E83E090E040E050E0BA0105CE3C
:106E1000D7012D913C912C5031092A30310508F0D1
:106E20001ACE440F551F661F771FF3CDD9012D9140
:106E30003C912C5031092B30310508F05DCE440FC8
:106E4000551F661F771F39CE2CEB31E0AE014D5F29
:106E50005F4FBE016F5F7F4FC7010E940A796C01CF
:106E60000330110579F42CEB31E0AE014D5F5F4F3B
:106E7000BE016F5F7F4FC7010E940A79C816D9060D
:106E800009F02BCFA114B10459F4CA94CD2809F00C
:106E900024CF440C551C661C771C689440F80BC02A
:106EA000AA94AB2809F019CFCD2809F016CF440CCD
:106EB000551C661C771C0F5F1F4FE5CE19961C935F
:106EC0000E931897F701448255826682778282E09A
:106ED00090E090CE848195814B97459708F047C00C
:106EE000DF0116966F0126ECC20ED11C20E030E0C7
:106EF00040E050E060E070E080E090E00D911C9197
:106F00001197095011090830110588F512960D9155
:106F10001C911397015111090D301105D8F401E0AE
:106F20000E94FA8E21601496AC15BD0539F7F70161
:106F3000248335834683578300E20E94158F228382
:106F4000338385E090E09183808380E390E09187B4
:106F500080877CC012960D911C91139704501109E3
:106F60000530110520F401E00E94FA8EDCCF8091FB
:106F7000200F893340F082819381895791098335AD
:106F8000910508F47CC18091200F823209F46CC015
:106F900082819381895791098335910508F4E6C16F
:106FA000828193818C549109C59708F064C08091C7
:106FB000200F843031F4848195818097479708F4BD
:106FC00034C28091200F843408F455C084819581A7
:106FD00089549109C39708F04EC09F012A5F3F4F23
:106FE000AF014A575F4F812C912C5401D9016D910B
:106FF0007C916950710969307105E8F5D9011296E3
:107000006D917C911397665171096131710508F09A
:1070100022C2D501C401880F991FAA1FBB1F4C01B2
:107020005D01689480F82C5F3F4F24173507F1F617
:1070300020E230E0F70131872087D70184829582F2
:10704000A682B78287E090E08D939C9381E090E0E8
:10705000BFC282E080931C0F1092200F80E090E06E
:10706000B7C283E090E0C6CD828193810A970997E9
:1070700008F460C18DCF8091200F863460F1828149
:1070800093810C970B9708F4F6C125C0D90112968D
:107090006D917C9113976E5171096731710508F0FC
:1070A0001EC2D501C401880F991FAA1FBB1F4C0126
:1070B0005D01689480F84E5F5F4F2C5F3F4F453411
:1070C000510509F4F3C1D9016D917C916C5071099E
:1070D0006B307105D8F28091200F883578F182816C
:1070E0009381855891098B35910508F408C226C013
:1070F000BC016F5F7F4FD8012D913C912750310922
:107100002730310508F00AC2440F551F416002962E
:107110000C5F1F4F2091200F30E02450310982175F
:1071200093070CF004C2980122503109D9012D9126
:107130003C912950310928303105D0F28091200F3F
:107140008032E1F48281938106970697B8F48481B6
:1071500095810997099790F49F012A5F3F4FAF01EE
:10716000425C5F4F812C912C5401D9016D917C912F
:10717000665071096630710508F4F3C1D7011C9699
:107180002D903C901D97B6E02B1631040CF461CF86
:107190008F010A5F1F4F73E0C72ED12CE5EC8E2EB6
:1071A000EDE99E2EECE1AE2EE1E8BE2EF801608105
:1071B000718134976080718080E090E00E94128A33
:1071C0006D837E838F839887B30180E090E00E9477
:1071D000128A2B013C012DEC3CEC4CE45FE30E9455
:1071E000738A9B01AC016D817E818F8198850E949D
:1071F0000E8A87FD19C02DEC3CEC4CE45FE36D81F9
:107200007E818F8198850E94738A9B01AC01C301A6
:10721000B2010E940E8AE82F880FFF0BEE27FF0FA6
:10722000EE1FFF27319602C0E0E0F0E0A5019401D7
:1072300063E971E080E091E00E94BC8E4F01FF0F96
:10724000AA08BB0886269726A826B926FFEFCF1ADC
:10725000DF0A0E5F1F4FC214D30409F0A7CFD70176
:1072600014968D929D92AD92BC92179780E290E019
:1072700019969C938E9318978FEF9FEFE5CE84819C
:107280009581CA97899708F07ECE9F012A5F3F4F6C
:10729000812C912C540143E050E0D9016D917C91F7
:1072A0006A5071096930710508F06DCED9011296E6
:1072B0006D917C911397665171096131710550F59B
:1072C000D501C401880F991FAA1FBB1F4C015D0186
:1072D000689480F84E5F5F4F2C5F3F4F4B335105F2
:1072E000E1F69F012A583F4FD9012D913C912A5038
:1072F00031092930310508F046CE2CE130E0F701A4
:1073000031872087D70184829582A682B7828AE05E
:1073100090E09ACED90112966D917C9113976650A8
:1073200071096730710508F02ECE880C991CAA1CD3
:10733000BB1CD0CF2091200FCF01820F911D820F57
:10734000911DDC0112978D919C910A97099708F085
:107350001FCEF701118610868FEF9FEFDC0184832B
:107360009583A683B78386E090E044CC8091200F7C
:10737000813208F415CE84819581CA97899708F0E7
:107380000FCE9F012A5F3F4F812C912C540143E087
:1073900050E0D9016D917C916A5071096930710595
:1073A00008F0FECDD90112966D917C91139766512C
:1073B00071096131710570F112966D917C9113978D
:1073C000665071096730710508F0EACD880C991C88
:1073D000AA1CBB1C4E5F5F4F2C5F3F4F43325105D1
:1073E000C1F69F012A5B3F4FD9012D913C912A5054
:1073F00031092930310508F0D3CD20E130E0F70123
:1074000031872087D70184829582A682B78286E061
:1074100090E01ACED501C401880F991FAA1FBB1F87
:107420004C015D01689480F8D5CF868197810997DA
:10743000099708F0C6CDD70119961C921E9218978D
:107440008FEF9FEFDC01F70184839583A683B783D9
:1074500087E090E0CFCBD90112966D917C91139784
:10746000665071096730710508F005CE880C991CCB
:10747000AA1CBB1CD8CD848195810997099708F077
:107480002ACE868197818C974F9708F024CE8085ED
:10749000918589974D9708F01ECE9F01265F3F4F3B
:1074A000812C912C540145E050E00DCE9F012657D0
:1074B0003F4FD9012D913C912C5031092B30310592
:1074C00008F009CE20E230E0F70131872087D701AC
:1074D00084829582A682B78288E090E0B5CDD901FA
:1074E00012966D917C9113976950710969307105FD
:1074F00008F0F1CD880C991CAA1CBB1CDCCD848142
:107500009581825491098E9708F018CE8F01045C02
:107510001F4F8DE190E040E050E0FCCDD8012D916F
:107520003C912851310922313105C0F0CB0101973E
:1075300095958795D70119969C938E9318978A975E
:107540000CF4FCCD052E000C660B770BF701448381
:1075500055836683778389E090E04CCB440F551FB9
:10756000D6CDD90112966D917C911397695171090D
:1075700063317105E8F4D501C401880F991FAA1F72
:10758000BB1F4C015D01689480F82C5F3F4F2417AE
:10759000350709F0EACD2EE030E0F701318720878A
:1075A000D70184829582A682B7828FE090E04CCD8D
:1075B000D90112966D917C911397695071096930C8
:1075C000710508F0DBCD880C991CAA1CBB1CDDCF13
:1075D00028960FB6F894DEBF0FBECDBFDF91CF91D6
:1075E0001F910F91FF90EF90DF90CF90BF90AF90E1
:1075F0009F908F907F906F905F904F903F902F90D3
:1076000008954F925F926F927F928F929F92AF9266
:10761000BF92DF92EF92FF920F931F93CF93DF936E
:10762000CDB7DEB7A9970FB6F894DEBF0FBECDBFBA
:10763000D82E882351F080911F11882331F06CEFF0
:107640007AE083E79EE00E94A55B21D760E08DE2AF
:107650000E94B95F60E18DE20E94B95F68E08DE24F
:107660000E94B95F4090751050907610609077102E
:107670007090781049825A826B827C828090791057
:1076800090907A10A0907B10B0907C108D829E829A
:10769000AF82B88680917D1090917E10A0917F106E
:1076A000B09180108EA39FA3A8A7B9A789879A87B6
:1076B000AB87BC87DD2099F180911F11882379F178
:1076C0007E019DE0E90EF11C67E57AE0C7010E94AA
:1076D0009B5AC7010E94546FC7010E94E1598E0155
:1076E0000F5F1F4FD8016D917D918D919D918D01FF
:1076F00046E050E0CBD66BE07AE083E79EE00E9464
:10770000C55B0E151F0571F76CEF7AE0C8010E948A
:10771000AB5AC8010E94546FC8010E94E15923E985
:1077200038E144E85FE3C301B2010E94738A2B0190
:107730003C016D877E878F87988B22E430E645E891
:107740005FE3C501B4010E94738A4B015C01698B40
:107750007A8B8B8B9C8B25E83BEE41E95FE36EA136
:107760007FA188A599A50E94738A6D8B7E8B8F8BD4
:10777000988F4092751050927610609277107092A8
:1077800078108092791090927A10A0927B10B0922B
:107790007C1060937D1070937E1080937F10909387
:1077A0008010DD2009F4A5C080911F11882309F401
:1077B000A0C07E01B9E1EB0EF11C6AE47AE0C701DA
:1077C0000E949B5AC7010E94546FC7010E94E15951
:1077D0008E01035F1F4FF801619171918191919129
:1077E0008F0142E050E052D66BE07AE083E79EE002
:1077F0000E94C55B0E151F0571F76CEF7AE0C8019A
:107800000E94AB5AC8010E94546FC8010E94E159FE
:1078100041E850E166E070E082E30E94505F8090B2
:107820008210912C982C882480918110882AA09015
:107830008410B12CBA2CAA2480918310A82AE0903D
:107840008610F12CFE2CEE2480918510E82A6DE341
:107850007AE083E79EE00E94D45A4AE050E0B40107
:1078600083E79EE00E949C5B6BE07AE083E79EE00A
:107870000E94C55B4AE050E0B50183E79EE00E94AC
:107880009C5B6BE07AE083E79EE00E94C55B4AE088
:1078900050E0B70183E79EE00E949C5B6CEF7AE0CA
:1078A00083E79EE00E94A55BC8010E940C6064E330
:1078B0007AE083E79EE00E94D45A7E01F5E2EF0E63
:1078C000F11CD8016D917D918D919D918D014AE0C2
:1078D00050E0DCD56BE07AE083E79EE00E94C55B78
:1078E0000E151F0571F76CEF7AE083E79EE00E94AA
:1078F000A55B61E08DE10E94B95FDD20B1F0809170
:107900001F11882391F060E27AE083E79EE00E94F5
:10791000D45AAE014B5D5F4F61E070E08DE10E9493
:10792000505F8DA190E00E948B5F62E08EE10E942B
:10793000B95F63E08FE10E94B95F64E080E20E947A
:10794000B95FDD2009F450C080911F11882309F42C
:107950004BC064E07AE083E79EE00E94D45AAE0117
:107960004B5D5F4F61E070E08EE10E94505FADA023
:10797000B12CAE014B5D5F4F61E070E08FE10E9482
:10798000505FEDA0F12CAE014B5D5F4F61E070E008
:1079900080E20E94505F0DA110E04AE050E0B50186
:1079A00083E79EE00E949C5B6BE07AE083E79EE0C9
:1079B0000E94C55B4AE050E0B70183E79EE00E9469
:1079C0009C5B6BE07AE083E79EE00E94C55B4AE047
:1079D00050E0B80183E79EE00E949C5B6CEF7AE088
:1079E00083E79EE00E94A55B65E081E20E94B95FAB
:1079F000DD20B1F080911F11882391F061EF79E0D3
:107A000083E79EE00E94D45AAE014B5D5F4F61E078
:107A100070E081E20E94505F8DA190E00E948B5F38
:107A200066E082E20E94B95FDD20B1F080911F1113
:107A3000882391F069ED79E083E79EE00E94D45AB3
:107A4000AE014B5D5F4F61E070E082E20E94505FEB
:107A50008DA190E00E948B5F67E083E20E94B95F96
:107A6000DD20B1F080911F11882391F063EC79E063
:107A700083E79EE00E94D45AAE014B5D5F4F61E008
:107A800070E083E20E94505F8DA190E00E948B5FC6
:107A900068E084E20E94B95FDD20B1F080911F119F
:107AA000882391F06BEA79E083E79EE00E94D45A44
:107AB000AE014B5D5F4F61E070E084E20E94505F79
:107AC0008DA190E00E948B5F69E085E20E94B95F22
:107AD000DD20B1F080911F11882391F061E979E0F8
:107AE00083E79EE00E94D45AAE014B5D5F4F61E098
:107AF00070E085E20E94505F8DA190E00E948B5F54
:107B00006AE086E20E94B95FDD20B1F080911F112A
:107B1000882391F06BE779E083E79EE00E94D45AD6
:107B2000AE014B5D5F4F61E070E086E20E94505F06
:107B30008DA190E00E948B5F6BE088E20E94B95FAC
:107B4000DD20B1F080911F11882391F062E679E089
:107B500083E79EE00E94D45AAE014B5D5F4F61E027
:107B600070E088E20E94505F8DA190E00E948B5FE0
:107B70006CE089E20E94B95FDD2009F479C0809150
:107B80001F11882309F474C06AE479E083E79EE05A
:107B90000E94D45AAE014B5D5F4F61E070E089E214
:107BA0000E94505F8DA190E00E948B5F63E379E0BB
:107BB00083E79EE00E94D45A66E070E087E20E946C
:107BC0009F5F90E00E948B5F6CE179E083E79EE02D
:107BD0000E94D45A65E070E087E20E949F5F90E0C7
:107BE0000E948B5F65E079E083E79EE00E94D45AB3
:107BF00064E070E087E20E949F5F90E00E948B5FEC
:107C00006CEE78E083E79EE00E94D45A62E070E078
:107C100087E20E949F5F90E00E948B5F63ED78E0B7
:107C200083E79EE00E94D45A61E070E087E20E9400
:107C30009F5F90E00E948B5F6AEB78E083E79EE0B5
:107C40000E94D45A60E070E087E20E949F5F90E05B
:107C50000E948B5F69EA78E083E79EE00E94D45A35
:107C600063E070E087E20E949F5F90E00E948B5F7C
:107C700041E067E070E087E20E94CE5F41E063E0B0
:107C800070E087E20E94CE5F41E063E070E08AE24C
:107C90000E94CE5FDD2091F080911F11882371F04A
:107CA00060E978E083E79EE00E94D45A63E070E0E8
:107CB0008AE20E949F5F90E00E948B5F40E063E059
:107CC00070E08AE20E94CE5FDD2091F080911F116A
:107CD000882371F066E778E083E79EE00E94D45A3B
:107CE00063E070E08AE20E949F5F90E00E948B5FF9
:107CF00041E062E070E08AE20E94CE5FDD2091F018
:107D000080911F11882371F06AE578E083E79EE097
:107D10000E94D45A62E070E08AE20E949F5F90E085
:107D20000E948B5F40E062E070E08AE20E94CE5FDA
:107D3000DD2091F080911F11882371F06DE378E0D0
:107D400083E79EE00E94D45A62E070E08AE20E94DB
:107D50009F5F90E00E948B5F41E061E070E08AE20B
:107D60000E94CE5FDD2091F080911F11882371F079
:107D700061E278E083E79EE00E94D45A61E070E01F
:107D80008AE20E949F5F90E00E948B5F40E061E08A
:107D900070E08AE20E94CE5FDD2091F080911F1199
:107DA000882371F064E078E083E79EE00E94D45A73
:107DB00061E070E08AE20E949F5F90E00E948B5F2A
:107DC00041E060E070E08AE20E94CE5FDD2091F049
:107DD00080911F11882371F068EE77E083E79EE0C1
:107DE0000E94D45A60E070E08AE20E949F5F90E0B7
:107DF0000E948B5F40E060E070E08AE20E94CE5F0C
:107E0000DD2091F080911F11882371F06BEC77E0F9
:107E100083E79EE00E94D45A60E070E08AE20E940C
:107E20009F5F90E00E948B5F41E066E070E087E238
:107E30000E94CE5F41E065E070E087E20E94CE5F85
:107E400041E064E070E087E20E94CE5F40E062E0E3
:107E500070E087E20E94CE5F40E061E070E087E280
:107E60000E94CE5F40E060E070E087E20E94CE5F5B
:107E7000DD2009F475C080911F11882309F470C0BA
:107E800063EB77E083E79EE00E94D45A66E070E0FF
:107E90008BE20E949F5F90E00E948B5F65E977E034
:107EA00083E79EE00E94D45A65E070E08BE20E9476
:107EB0009F5F90E00E948B5F67E777E083E79EE03B
:107EC0000E94D45A64E070E08BE20E949F5F90E0D1
:107ED0000E948B5F6EE577E083E79EE00E94D45AB4
:107EE00062E070E08BE20E949F5F90E00E948B5FF7
:107EF00065E477E083E79EE00E94D45A61E070E099
:107F00008BE20E949F5F90E00E948B5F6CE277E0C3
:107F100083E79EE00E94D45A60E070E08BE20E940A
:107F20009F5F90E00E948B5F69E177E083E79EE0CE
:107F30000E94D45A63E070E08BE20E949F5F90E061
:107F40000E948B5F64E077E083E79EE00E94D45A52
:107F500064E070E08CE20E949F5F90E00E948B5F83
:107F600040E064E070E08CE20E94CE5FAE014B5DC9
:107F70005F4F61E070E08CE20E94505F6DA1607F16
:107F800066608CE20E94B95FDD2009F465C08091D3
:107F90001F11882309F460C060EF76E083E79EE05C
:107FA0000E94D45AAE014B5D5F4F61E070E08CE2FD
:107FB0000E94505F6DA16F7070E066507109072ECE
:107FC000000C880B990B0E94148A9B01AC0160E0A5
:107FD00070E080E090E40E94128E20E030E048ECF7
:107FE00050E40E94738A0E94FE5F69ED76E083E7A9
:107FF0009EE00E94D45AAE014B5D5F4F61E070E09D
:1080000080E30E94505F4DA150E060E070E02AE004
:1080100083E79EE00E940D5B83E79EE00E94A25BE7
:1080200061EC76E083E79EE00E94D45A61E070E064
:1080300080E30E949F5F90E00E948B5F68EA76E099
:1080400083E79EE00E94D45A61E070E08FE20E94D4
:108050009F5F90E00E948B5F41E061E070E08FE203
:108060000E94CE5FDD2091F080911F11882371F076
:1080700060E976E083E79EE00E94D45A61E070E018
:108080008EE20E949F5F90E00E948B5F41E061E082
:1080900070E08EE20E94CE5F40E067E070E081E336
:1080A0000E94CE5FDD2009F455C080911F11882306
:1080B00009F450C06DE776E083E79EE00E94D45A51
:1080C00067E070E081E30E949F5F90E00E948B5F19
:1080D00069E17AE083E79EE00E94C55BAE014B5DFB
:1080E0005F4F61E070E080E00E94505F8DA10E94D0
:1080F000C34E6CEF7AE083E79EE00E94A55B0DE142
:1081000010E067E67AE083E79EE00E94C55B40E10D
:1081100050E0B80183E79EE00E949C5B69E278E052
:1081200083E79EE00E94C55BAE014B5D5F4F61E05F
:1081300070E0802F0E94505F8DA10E94C34E6CEFB3
:108140007AE083E79EE00E94A55B0F5F1F4F0A3332
:108150001105B9F6A9960FB6F894DEBF0FBECDBFD4
:10816000DF91CF911F910F91FF90EF90DF90BF9023
:10817000AF909F908F907F906F905F904F900895F9
:108180002091380D90911111213208F04AC0809150
:10819000150D8111FCCF32E03093150D31E0309395
:1081A000140D3FEF3093130D1092120D2093110D0B
:1081B000A8E1BDE041EF5CE0FA013E2F341B32172D
:1081C00018F43D913193F9CF1092F00C2091F00CFE
:1081D000990F922B9093F00C9091EF0C913061F4E9
:1081E0001092EF0C9091F00C9093BB009091BC001A
:1081F00093FDF8CF95EC01C095EE9093BC00909163
:10820000150D9230E1F39091130D9F3F79F080911D
:10821000130D803241F08091130D803331F084E0F2
:1082200005C081E003C082E001C083E01092170D19
:108230001092380D1092160D0895682F80E19FE07E
:108240000C943E5091E09093160D80931111109272
:10825000170D1092380D0895CF93C82F682F607FA7
:1082600085E091E10E94964D80E1C89FB001112404
:1082700085E091E1CF910C94964DCF93DF93CDB7EC
:10828000DEB728970FB6F894DEBF0FBECDBF98E0DB
:10829000E6EEF4E0DE01119601900D929A95E1F779
:1082A00090910E11961710F46FEF690FFE01319641
:1082B000E60FF11DE60FF11D9081890F8068289669
:1082C0000FB6F894DEBF0FBECDBFDF91CF91C4CF04
:1082D0004F925F926F927F928F929F92AF92BF92D6
:1082E000CF92DF92EF92FF926B017C01B42E9B0143
:1082F000AC010E94A38E882319F06EE27AE027C0B9
:1083000026013701E89477F82FEF3FEF4FE75FE75B
:10831000C301B2010E94A38E81110DC02FEF3FEF68
:108320004FE75FE7C301B2010E940E8A18161CF4E2
:1083300062E37AE00CC02FEF3FEF4FE75FE4C70145
:10834000B6010E94538D181694F466E37AE083E731
:108350009EE0FF90EF90DF90CF90BF90AF909F9006
:108360008F907F906F905F904F900C94F85A2FEF02
:108370003FEF4FE75FECC701B6010E940E8A87FD11
:10838000E4CF20E030E0A901C701B6010E940E8AC7
:1083900087FF0BC06DE283E79EE00E94BF5A4C014D
:1083A000F7FAF094F7F8F09402C0812C912CA12CEC
:1083B00060E070E080E09FE3AB1441F020E030E04B
:1083C00040E251E40E94648CA394F6CF9B01AC017F
:1083D000C701B6010E949E8B2B013C010E94028DB9
:1083E0006B017C010E94128A9B01AC01C301B201A6
:1083F0000E949D8B2B013C012AE0B701A60183E777
:108400009EE00E940D5B7C01E80CF91CBB2039F05A
:108410006EE283E79EE00E94BF5AE80EF91EDB2C55
:10842000DD2031F120E030E040E251E4C301B2014F
:108430000E94738A2B013C010E94028D4B01A12CEA
:10844000B12C2AE0B501A40183E79EE00E940D5BF8
:10845000E80EF91EC501B4010E94128A9B01AC010D
:10846000C301B2010E949D8B2B013C01DA94D8CF4D
:10847000C701FF90EF90DF90CF90BF90AF909F909B
:108480008F907F906F905F904F90089521CF1092C2
:10849000EE0C1092ED0C1092170D1092380D1092F8
:1084A000150D81E08093140D1092EF0C61E084E1D2
:1084B0000E94065D61E085E10E94065DE9EBF0E067
:1084C00080818E7F808380818D7F808388E480930C
:1084D000B80085E48093BC0008952F923F924F929C
:1084E0005F926F927F928F929F92AF92BF92CF9244
:1084F000DF92EF92FF920F931F93CF93DF93CDB74D
:10850000DEB728970FB6F894DEBF0FBECDBF4091FF
:108510009D0C50919E0CC0909F0CD090A00C4C15BF
:108520005D052CF03C2D2D2D6A01432F522FE1EAE1
:10853000FCE060E070E0CB01019111910417150798
:1085400054F44A01550FAA08BB08680D791D8A1D0D
:108550009B1DA80115C0C016D10654F40D2C000CAB
:10856000EE08FF086C0D7D1D8E1D9F1D680108C063
:10857000012E000C220B330B600F711F821F931F03
:108580002CE0ED3EF207C1F60E94148A20E030E0B4
:1085900048E152E40E94648C6B017C010DE91CE00F
:1085A000812C912C5401D8016D917D918D01072E64
:1085B000000C880B990B0E94148AA70196010E9457
:1085C0009D8B9B01AC010E94738A9B01AC01C5018C
:1085D000B4010E949E8B4B015C01BCE00D3E1B0769
:1085E00011F720E030E04CE152E40E94648C0E94DC
:1085F000628E4B015C0120E030E040E85FE30E94C6
:10860000538D18160CF06EC00DE91CE0212C312C96
:1086100019821A821B821C82F801819191918F012B
:108620009C01990F440B550B2D833E834F83588734
:10863000CA01B9010E94148AA70196010E949D8B6C
:108640002B013C0120E030E0A9010E94538D181657
:1086500024F077FA709477F87094A5019401C3011F
:10866000B2010E940E8A87FF13C089819A81AB8173
:10867000BC812D813E814F815885820F931FA41F9D
:10868000B51F89839A83AB83BC833FEF231A330AD8
:108690004CE00D3E140709F0BFCF20E030E040EC85
:1086A0005FE3C501B4010E94738A4B015C0155E090
:1086B000251631040CF4A8CF69817A818B819C81C5
:1086C0000E94148A6B017C01B101330C880B990B59
:1086D0000E94148A9B01AC01C701B6010E94648C00
:1086E0006B017C01C701B60128960FB6F894DEBF76
:1086F0000FBECDBFDF91CF911F910F91FF90EF90F3
:10870000DF90CF90BF90AF909F908F907F906F90B1
:108710005F904F903F902F9008954F925F926F928D
:108720007F928F929F92AF92BF92CF92DF92EF9201
:10873000FF920F931F93CF93DF9300D01F92CDB77B
:10874000DEB76B017C0111E0A12EB12C4501880C34
:10875000991C880C991CF401E85DFD4F4080518004
:1087600062807380A3019201C701B6010E94538DFC
:10877000181614F41F5FE8CFA3019201C701B601D8
:108780000E940E8A8401005F1D4F811106C0D8012E
:108790006D917D918D919C9142C0C5018150904C0D
:1087A000880F991F880F991FFC01E85DFD4F2081FC
:1087B00031814281538129833A834B835C83FC015D
:1087C000E05FFD4F80809180A280B380C701B60139
:1087D0000E949D8B6B017C01A5019401D8016D91D4
:1087E0007D918D919C910E949D8B9B01AC01C70155
:1087F000B6010E94738A6B017C0129813A814B8109
:108800005C81C301B2010E949D8B9B01AC01C70139
:10881000B6010E94648CA50194010E949E8B0F906A
:108820000F900F900F90DF91CF911F910F91FF90BC
:10883000EF90DF90CF90BF90AF909F908F907F9000
:108840006F905F904F900895DF92EF92FF920F9399
:108850001F93CF93DF937C018B01EA0146175707E3
:1088600020F4812F8A01C62FD82F6CEF7AE0C70140
:108870000E94AB5A80911710909118100817190791
:10888000E0F48C179D0708F4EC01E0911310F091CF
:108890001410EC0FFD1FD0801082609113107091A6
:1088A0001410600F711FC7010E947E59E0911310D0
:1088B000F0911410EC0FFD1FD082C701DF91CF9112
:1088C0001F910F91FF90EF90DF900895CF93DF936A
:1088D000EC014091171050911810B6DFCE01DF91D6
:1088E000CF9108950F931F933DD56093DE0D709344
:1088F000DF0D8093E00D9093E10DE091D60DF091A6
:10890000D70D0284F385E02D86ED9DE0199597FF44
:108910001EC028D50091DE0D1091DF0D2091E00DD5
:108920003091E10DDC01CB01801B910BA20BB30B4D
:108930000091DA0D1091DB0D2091DC0D3091DD0DF1
:1089400080179107A207B307C0F28FEF9FEF1F9127
:108950000F910895CF93DF931F92CDB7DEB760914B
:108960009B0C8EED93E069830E942A8B69816817C6
:1089700021F08EED93E00E94328B60919C0C8FED84
:1089800093E069830E942A8B6981681721F08FED3B
:1089900093E00E94328B8BE99CE00F90DF91CF91A6
:1089A0000895CF92DF92EF92FF920F931F93CF9390
:1089B000DF931F92CDB7DEB76C0101E21CE07C01B2
:1089C0008AE7E80EF11CF80161918F01C601698305
:1089D0000E942A8B6981681719F0C6010E94328BA8
:1089E000FFEFCF1ADF0ACE14DF0469F781E29CE0C3
:1089F0000F90DF91CF911F910F91FF90EF90DF903B
:108A0000CF9008959091150D9111FCCF91E0909326
:108A1000150D9093140D2FEF2093130D1092120D3E
:108A2000260F2093110D9093F00C9091F00C880F6D
:108A3000892B8093F00C8091EF0C813061F41092BF
:108A4000EF0C8091F00C8093BB008091BC0083FD03
:108A5000F8CF85EC01C085EE8093BC008091150DA8
:108A60008130E1F38091120D861710F46091120DA0
:108A7000A1EFBCE021E03CE0F9018E2F821B8617BC
:108A800018F48D918193F9CF862F0895613208F003
:108A900060E2B8DF1092EE0C8093ED0C08951F9306
:108AA000CF93DF931F92CDB7DEB7682F87E7698337
:108AB000C9DB698180E19FE00E943E5061DB87E76E
:108AC000C1DB61E070E087E790E0E0DF80E19FE0FC
:108AD0000E94F34F182F54DB812F0F90DF91CF911D
:108AE0001F9108950F931F93CF93DF931F92CDB7DC
:108AF000DEB7682F87E76983A5DB698180E19FE0A6
:108B00000E943E503DDB87E79DDB62E070E087E737
:108B100090E0BCDF80E19FE00E94F34F00E010E0B6
:108B2000182F80E19FE00E94F34F082B192B28DBC0
:108B3000C8010F90DF91CF911F910F91089587E7A2
:108B400081DB64EF80E19FE00E943E506EE280E1B5
:108B50009FE00E943E5014DB65E070E080E090E012
:108B60000E94965D86EFBECF3F924F925F926F92CA
:108B70007F928F929F92AF92BF92CF92DF92EF92AD
:108B8000FF920F931F93CF93DF93CDB7DEB7289754
:108B90000FB6F894DEBF0FBECDBFD1DF6C01E12C64
:108BA000F12C109119101295110F110F107C1C5CF3
:108BB00087E748DB64EF80E19FE00E943E50612F31
:108BC00080E19FE00E943E50DBDA80911910811114
:108BD00005C065E070E080E090E012C0813029F4CB
:108BE00068E070E080E090E00BC0823029F46EE035
:108BF00070E080E090E004C06AE170E080E090E026
:108C00000E94965D86EF6EDF4C01A12CB12CBA2C30
:108C1000A92C982C882488EF42DF882A30901910DC
:108C200080912E1090912F10A7019601281B390BCF
:108C300041095109A0912C10B0912D100E945C8B1C
:108C40006B017C01AFE0F594E794D794C794AA95A3
:108C5000D1F76091261070912710CB01770FAA0BE6
:108C6000BB0BBC01CD01BBE0660F771F881F991FAE
:108C7000BA95D1F720912810309129108901330F2E
:108C8000220B330BA90198012C0D3D1D4E1D5F1DBC
:108C90000E94408BC20ED31EE41EF51E20EAC21AAB
:108CA0002FE0D20AE108F108A7019601C701B60139
:108CB0000E94BC8E9B01AC011CE0559547953795F1
:108CC00027951A95D1F729833A834B835C830091CA
:108CD0001A1010911B10A0911E10B0911F10A70127
:108CE00096010E94668B2B013C018DE07594679480
:108CF000579447948A95D1F7A0912010B0912110F4
:108D000029813A814B815C810E94668BBB2797FD4C
:108D1000B095AB2F840D951DA61DB71D0296A11D04
:108D2000B11D32E0B595A795979587953A95D1F7FE
:108D30009C01AD0130584F4F5F4FA0912A10B09168
:108D40002B100E945C8B2B013C014FE076946794C2
:108D5000579447944A95D1F788E090E08319910998
:108D6000A501940104C056954795379527958A9596
:108D7000D2F72D833E834F8358874801110FAA08ED
:108D8000BB0852E0880C991CAA1CBB1C5A95D1F751
:108D9000A0912210B091231029813A814B815C81EE
:108DA0000E94668B9B01AC016BE05595479537950A
:108DB00027956A95D1F729833A834B835C83A091E9
:108DC0001C10B0911D10A70196010E94668BDC015A
:108DD000CB017BE0B595A795979587957A95D1F7C7
:108DE00029813A814B815C81820F931FA41FB51F9B
:108DF000880D991DAA1DBB1D032C04C0880F991F47
:108E0000AA1FBB1F0A94D2F7BC01CD016E5F7F4F32
:108E10008F4F9F4F24E030E040E050E00E94408BB5
:108E20008D819E81AF81B885821B930BA40BB50BFE
:108E30009C01AD0180E593ECA0E0B0E0BC01CD0168
:108E400004C096958795779567953A94D2F70E94D6
:108E5000BC8E97FD0BC0660F771F881F991FA3015B
:108E600092010E946C8B69017A010AC0A3019201F0
:108E70000E946C8B69017A01CC0CDD1CEE1CFF1C7E
:108E80009927F7FC9A958F2D7E2D6D2D9B01AC01B6
:108E90000E94BC8E9B01AC01AEEDBBE00E945C8BDE
:108EA0004C01BB2497FCB094AB2CA3E4B3EEA70118
:108EB00096010E94688BBB2797FDB095AB2F880D5C
:108EC000991DAA1DBB1D8153914FAF4FBF4F44E069
:108ED000B595A795979587954A95D1F7BC01CD0192
:108EE0006C0D7D1D8E1D9F1D28960FB6F894DEBF5C
:108EF0000FBECDBFDF91CF911F910F91FF90EF90EB
:108F0000DF90CF90BF90AF909F908F907F906F90A9
:108F10005F904F903F900895CF92DF92EF92FF9233
:108F20000F931F930CDEAC0160E070E0E9E1F0E12B
:108F3000858996899A01AB01281B390B4109510992
:108F4000A389B4890E945C8B6B017C018FE0F5944E
:108F5000E794D794C7948A95D1F765857685CB0138
:108F6000770FAA0BBB0BBC01CD012BE0660F771F5F
:108F7000881F991F2A95D1F7278530898901330FDA
:108F8000220B330BA90198012C0D3D1D4E1D5F1DB9
:108F90000E94408BD701C601820F931FA41FB51FEB
:108FA0000896A11DB11DBC01CD0134E095958795B2
:108FB000779567953A95D1F70E94148A20E030E0C2
:108FC00040E251E40E94648C1F910F91FF90EF905A
:108FD000DF90CF9008958F929F92AF92BF92CF92E1
:108FE000DF92EF92FF92CF93DF93A09168108823D6
:108FF00011F03A2F01C030E08091691090E0880FA5
:10900000991F8B59954FC0906E10D0906F10E090C3
:109010007010F090711040E050E0BA01FC01C59171
:10902000D49128812A2323130FC04A015B012FEF1B
:10903000821A920AA20AB20A4C155D056E057F05D6
:1090400038F4B501A401EACF342F252FCB0104C099
:1090500030E020E080E090E0632F722FDF91CF912D
:10906000FF90EF90DF90CF90BF90AF909F908F9048
:109070000895DC0180E0615090F09D919827E92FE0
:10908000EF70F0E0E55FF44F249192959F70E92F27
:10909000F0E0E55EF44FE4918E2F8227ECCF089547
:1090A0000F931F93CF93DF938C01EB0188E2FB01B9
:1090B00011928A95E9F74BE050E06AE37AE0CE013D
:1090C0000E9464911B8681E090E0A0E0B0E08C8774
:1090D0009D87AE87BF87F80185899689A789B08D5E
:1090E000888B998BAA8BBB8B82E090E0A0E0B0E0EC
:1090F0008C8B9D8BAE8BBF8B1CA21DA21EA21FA2B0
:1091000080E090E0A8E4B4E4888F998FAA8FBB8FA9
:1091100080E090E0A8E4B4EC8C8F9D8FAE8FBF8F81
:109120008DEC9CECACE4BEE388A399A3AAA3BBA3FB
:10913000DF91CF911F910F9108954F925F926F929F
:109140007F928F929F92AF92BF92CF92DF92EF92D7
:10915000FF920F931F93CF93DF938C01EB0184E277
:10916000FB0111928A95E9F78EE16CD883E090E0DB
:1091700064D806D866E08EE145DC1092EE0C809350
:10918000ED0C90E086309105ECF380E19FE02BD769
:10919000882E80E19FE027D7982E80E19FE023D79B
:1091A000682E80E19FE01FD7782E80E19FE01BD7DB
:1091B000482E80E19FE017D7582EB82CA12CB5017E
:1091C0006929072E000C880B990B0E94148A4B0109
:1091D0005C01F8016583768387839087D42CC12C4A
:1091E000B6016529072E000C880B990B0E94148A82
:1091F000F8016187728783879487F62CE12CB70189
:109200006729072E000C880B990B0E94148AF8011D
:10921000658776878787908B118A128A138A148ACA
:1092200084E290E0A0E0B0E088839983AA83BB83C6
:1092300085899689A789B08D8C839D83AE83BF83F2
:1092400082E090E0A0E0B0E088879987AA87BB879A
:10925000188A198A1A8A1B8AC0907202D0907302E7
:10926000E0907402F0907502A7019601C501B40167
:109270000E94648C20E030E048EC52E40E94738A43
:109280006C8B7D8B8E8B9F8BA7019601F80161857E
:109290007285838594850E94648C20E030E048ECE0
:1092A00052E40E94738A688F798F8A8F9B8F2091F6
:1092B0006E0230916F024091700250917102F8017C
:1092C00065857685878590890E94648C20E030E0F2
:1092D00048EC52E40E94738A6C8F7D8F8E8F9F8F33
:1092E00081E0DF91CF911F910F91FF90EF90DF9080
:1092F000CF90BF90AF909F908F907F906F905F9036
:109300004F900895862F0C94DE5C862F642F0C946A
:10931000065D862F642F0C94355D3FB7F8948091DD
:10932000171190911811A0911911B0911A1126B529
:10933000A89B05C02F3F19F00196A11DB11D3FBF8D
:10934000BA2FA92F982F8827820F911DA11DB11D1B
:10935000BC01CD0142E0660F771F881F991F4A9517
:10936000D1F708952FB7F8946091131170911411EB
:1093700080911511909116112FBF08951F920F9291
:109380000FB60F9211242F933F938F939F93AF9318
:10939000BF938091131190911411A0911511B09168
:1093A00016113091121123E0230F2D3720F401966E
:1093B000A11DB11D05C026E8230F0296A11DB11DF8
:1093C000209312118093131190931411A0931511EF
:1093D000B09316118091171190911811A091191145
:1093E000B0911A110196A11DB11D80931711909390
:1093F0001811A0931911B0931A11BF91AF919F91B9
:109400008F913F912F910F900FBE0F901F90189545
:10941000DF92EF92FF920F931F93CF93DF937C0124
:109420008B01D42EDC011696ED91FC9117971386D3
:1094300015861486DF011B9633961E92AE17BF0762
:10944000E1F7C0E0B801D70116968D919C9117976E
:109450000E943D61D82F811102C0D0E00DC0CD1116
:1094600007C067E0C80105DEF8019781891721F080
:10947000CF5FDC1690F3E6CF8D2FDF91CF911F9158
:109480000F91FF90EF90DF900895FC019081018093
:10949000F281E02DF8948181892B81832281892FAB
:1094A000809528232283A7E0B0E01197F1F721816E
:1094B00082238183A3E2B0E01197F1F78081789451
:1094C000EFECF0E03197F1F7982381E009F480E0C8
:1094D0000895FC0190810180F281E02D892F809513
:1094E00060FF12C0F8942281822382838181892BBC
:1094F0008183A3E2B0E01197F1F78281982B9283E8
:10950000789487ED90E011C0F894228182238283C1
:109510008181892B8183AFEFB0E01197F1F78281D0
:10952000982B928378948FE090E00197F1F708955B
:10953000CF92DF92EF92FF920F931F93CF93DF931F
:109540001F92CDB7DEB76C01E62E08E010E0FF24D5
:10955000F39461E08F2D8E2109F460E0C601498308
:10956000B8DFFF0C0150110949810115110589F778
:10957000411115C0F894D6011196ED91FC91129706
:1095800091818C918095892381831196ED91FC9135
:10959000129792818C9180958923828378940F9081
:1095A000DF91CF911F910F91FF90EF90DF90CF90BF
:1095B0000895CF92DF92EF92FF920F931F93CF9374
:1095C000DF931F92CDB7DEB78C01F62E40E065E544
:1095D0007983AEDFCF2C7981D72E760188E0E80E33
:1095E000F11CF60161916F0140E0C801A1DFCE14CA
:1095F000DF04B9F70F90DF91CF911F910F91FF908A
:10960000EF90DF90CF900895FC0190810180F2816E
:10961000E02DF8948181292F2095822381837894ED
:109620008DE743E050E0815021F1DA011197F1F725
:1096300030813923C1F3F89482818223828381812E
:10964000892B81837894ABE7B7E01197F1F7F89411
:10965000818128232183A3E1B1E01197F1F7808173
:10966000982381E009F080E07894E3E6F6E0319712
:10967000F1F708958F929F92AF92BF92CF92DF92AF
:10968000EF92FF920F931F93CF93DF93EC018E81A4
:109690009F81BADF40E06CEC8E819F8149DF488179
:1096A00064E48E819F8144DF8A81882309F43FC06E
:1096B000E981E950E33040F4F0E0EE0FFF1FEE5A8D
:1096C000FA4F0081118102C00EEE12E08B818823D7
:1096D000E1F08881811119C045DE4B015C01680110
:1096E000110FEE08FF088E819F81CFDE8130F9F0E7
:1096F00039DEDC01CB018C199D09AE09BF09881543
:109700009905AA05BB0578F312C0B801110F880BA3
:10971000990BDF91CF911F910F91FF90EF90DF9008
:10972000CF90BF90AF909F908F900C94965DDF91FB
:10973000CF911F910F91FF90EF90DF90CF90BF904E
:10974000AF909F908F9008954F925F926F927F920B
:109750008F929F92AF92BF92CF92DF92EF92FF9241
:109760000F931F93CF93DF931F921F92CDB7DEB756
:109770002C018A01FC018681978169837A8344DF09
:1097800069817A818823A1F1F2018681978111DFB5
:1097900040E06EEBF20186819781CADE78014801D4
:1097A000F9E08F0E911CF2016680778088E0A82E88
:1097B000B12CCC24C394D12CC30167DE8111DC28E9
:1097C000CC0CF1E0AF1AB108B9F7F701D1927F01E3
:1097D000E815F90541F7F2018681978115DF81309F
:1097E00039F468E0C80145DC91E0F8012085821376
:1097F00090E0892F0F900F90DF91CF911F910F91E3
:10980000FF90EF90DF90CF90BF90AF909F908F90A0
:109810007F906F905F904F900895CF93DF93CDB777
:10982000DEB729970FB6F894DEBF0FBECDBFAE01ED
:109830004F5F5F4F89DF882389F08D818F3361F01F
:1098400020F48F3159F489E00CC08F3519F08F372F
:1098500039F004C08BE005C08AE003C080E001C09D
:109860008CE029960FB6F894DEBF0FBECDBFDF9116
:10987000CF9108950F931F93CF93DF93CDB7DEB7AA
:1098800061970FB6F894DEBF0FBECDBF8C01462F97
:10989000BE01665F7F4FBCDD811105C060E070E0F6
:1098A0008EEF92EC4AC0AE014F5F5F4FBE01665F24
:1098B0007F4FC80149DF882359F1698148E0649FDF
:1098C000B00111248A81282F30E0322F2227330F54
:1098D000330F330F262B372B8A858031E1F46885CF
:1098E00070E08F81AB01481B5109CA019695982FF2
:1098F0008827979587950E94DF8E60517109207F98
:1099000053E0220F331F5A95E1F7620F731F04C013
:1099100060E874EE01C0B901613854EE75070CF4CB
:10992000BDCF072E000C880B990B0E94148A20E0F3
:1099300030E040E05CE30E94738A61960FB6F894D1
:10994000DEBF0FBECDBFDF91CF911F910F91089564
:10995000EF92FF920F931F93CF93DF93CDB7DEB7B4
:1099600028970FB6F894DEBF0FBECDBF8C01DC0187
:109970001696ED91FC911797138615861486DF01D4
:109980001B9633961E92AE17BF07E1F7F8011482BB
:109990001582EE24E394BE016F5F7F4FF80186814C
:1099A00097810E943D61882309F469C067E0CE0178
:1099B00001965FDB98858913EECFD8018C918111D8
:1099C00021C016968D919C9117971EDEBE016F5F88
:1099D0007F4FF80186819781ECDD40E064EBD80190
:1099E00016968D919C911797A3DDF801868197813A
:1099F0004CDDF82ED80116968D919C91179704DEB8
:109A0000FF20B1F1F801F18089818031A1F1BE011F
:109A10006F5F7F4FC80101DF8F1520F4D8011196C9
:109A20008C910AC08981803111F48CE005C0BE019F
:109A30006F5F7F4FC801F1DEF801818384818F5F02
:109A400084838981883261F030F4803149F0823238
:109A500009F0A1CF05C08B3319F0823409F09BCFF8
:109A6000D80115968C9115978F5F15968C9393CF8F
:109A7000D801EC92C7CFBCE0BF1580F2D6CF2896B4
:109A80000FB6F894DEBF0FBECDBFDF91CF911F910F
:109A90000F91FF90EF9008950F931F93CF93DF9353
:109AA000EC01162F60E0812F0E94355D612F70E080
:109AB000FB01EB53F54FE491E883FB01E158F54FCF
:109AC000E491F0E0EE0FFF1FEB59F54F8591949173
:109AD0009A8389831B861D861C86FE013B968E0118
:109AE0000D5F1F4F1292E017F107E1F7DF91CF9161
:109AF0001F910F9108950F931F93CF93DF931F92A0
:109B0000CDB7DEB78C01FC01848169830E942241BC
:109B1000F80183856981862B90E00E941D410F909A
:109B2000DF91CF911F910F910C94C0400F931F9321
:109B3000CF938C01C62FDFDF6C2F6460C801DBDFA1
:109B40006C2F6B7FC801D7DF83EC90E00197F1F7B2
:109B5000CF911F910F9108950F931F93CF938C0175
:109B6000C62F607F6160E2DF80E1C89FB0011124F1
:109B70006160C801DBDF81E090E0CF911F910F9120
:109B800008951F920F920FB60F9211240BB60F92E9
:109B90002F933F934F935F936F937F938F939F93F5
:109BA000AF93BF93EF93FF9380911D0F0E94DE5CF4
:109BB0002091210F3091220F2F5F3F4F3093220FC2
:109BC0002093210F9091200F953618F096E09093F6
:109BD0001C0F90911C0F9430C9F128F4923069F059
:109BE0009330D1F05EC0953009F451C0963009F041
:109BF00058C091E09093ED0F51C0811152C0209157
:109C0000210F3091220F2436310508F442C0109202
:109C1000ED0F1092200F1CC0813009F042C0E0917E
:109C2000200F91E09E0F9093200FF0E02091210FE4
:109C30003091220FEE0FFF1FE45EF04F3087278335
:109C40001092220F1092210F94E029C0811117C0A9
:109C5000E091200F91E09E0F9093200FF0E0209173
:109C6000210F3091220FEE0FFF1FE45EF04F30877F
:109C700027831092220F1092210F93E010C02091A1
:109C8000210F3091220F2536310558F007C0811180
:109C900008C01092220F1092210F03C095E09093FC
:109CA0001C0F90911F0F9923B9F081110AC0809168
:109CB0001E0F882321F080911E0F61E009C02F9AAA
:109CC0000BC080911E0F882331F080911E0F60E041
:109CD0000E94065D01C02F98FF91EF91BF91AF9157
:109CE0009F918F917F916F915F914F913F912F91B4
:109CF0000F900BBE0F900FBE0F901F901895CF9234
:109D0000DF92EF92FF92CF93DF93EC01072E000CCE
:109D1000880B990B0E94148A6B017C0120E030E0D3
:109D200040E45FE30E94738A20E030E048E452E4BC
:109D30000E94648C0E94FD8CC617D707D4F020E0E7
:109D400030E040EA5FE3C701B6010E94738A20E079
:109D500030E048E452E40E94648C20E030E040E8C7
:109D60005FE30E949E8B0E94FD8C21E06C177D07B3
:109D70000CF420E0822F90E0DF91CF91FF90EF90E4
:109D8000DF90CF9008950F931F93CF93DF93082F09
:109D90006FE679E083E79EE00E94C55BC7E0D0E014
:109DA00010E0B8010C2E02C0759567950A94E2F791
:109DB0006170772742E050E083E79EE00E949C5B61
:109DC000219778F7DF91CF911F910F9108950E940D
:109DD00042918091F50F9091F60F009711F00C943D
:109DE0005F8560E070E0CB010895AF92BF92CF92A3
:109DF000DF92EF92FF920F931F93CF93DF93209107
:109E0000171030911810FC01448155818901041B01
:109E1000150B4115510559F12115310541F1241753
:109E2000350728F10217130718F0890101501109AD
:109E30007C01A0901310B0901410C501DFEFCFEF9C
:109E40006501C00ED11EC816D906A0F0F7016081C9
:109E500071810E947391009769F09C012A193B0956
:109E60000217130710F0D22FC32F0196ECCF8FEFFC
:109E70009FEF02C08D2F9C2FDF91CF911F910F91EB
:109E8000FF90EF90DF90CF90BF90AF900895FC01CE
:109E900080819181009711F00C94628560E070E000
:109EA000CB010895AF92BF92CF92DF92EF92FF92D3
:109EB0000F931F93CF93DF93DC01CD90DC9011972C
:109EC000C114D10409F442C01496CD91DC911597C8
:109ED0002097E1F18C0156017501BFEFAB1ABB0A67
:109EE000F7018081082E000C990B0E94DE89892BD6
:109EF00099F72197CC0DDD1D8881082E000C990B58
:109F00000E94DE89892B91F4AE014F5F5F4F4E199D
:109F10005F09D80115965C934E931497CE14DF0415
:109F200050F4B701C6010E94469105C0CE15DF0569
:109F300058F32197E1CFD801ED91FC911197149638
:109F40008D919C911597E80FF91F1082DF91CF91A9
:109F50001F910F91FF90EF90DF90CF90BF90AF9047
:109F6000089585ED8093BC008091BC0084FDFCCFFA
:109F70001092150D089540917411262F30E0240F92
:109F8000311D21323105DCF42091150D2430C9F446
:109F9000FC0180E090E0861758F430917411219113
:109FA000DC01AE5ABE4EA30FB11D2C930196F3CF28
:109FB00080917411680F6093741180E0089581E0BE
:109FC000089582E008950895E091EE0C8091ED0CE3
:109FD000E81730F4F0E0EF5FF34F808190E00895F0
:109FE0008FEF9FEF08959091EE0C8091ED0C9817F4
:109FF00050F4E92FF0E0EF5FF34F208130E09F5FF6
:10A000009093EE0C02C02FEF3FEFC90108958091AD
:10A01000ED0C90E02091EE0C821B91090895CF92F7
:10A02000DF92EF92FF920F931F93CF93DF937C0108
:10A03000262F972F8A018091160D882391F0C62F25
:10A04000D72F6E01C40ED51ECC15DD0569F06991C0
:10A05000D701ED91FC910190F081E02DC701199598
:10A06000F3CF642F822F87DFC801DF91CF911F913B
:10A070000F91FF90EF90DF90CF900895CF93DF93F3
:10A080001F92CDB7DEB769832091160D2223D1F040
:10A090002091380D203240F021E030E0FC01338384
:10A0A000228380E090E014C08091170DE82FF0E04B
:10A0B000E85EF24F998190838F5F8093170D8093B4
:10A0C000380D04C061E0CE01019655DF81E090E0DB
:10A0D0000F90DF91CF910895089580E090E008956A
:10A0E0000C94C68F0F931F93CF93C091DD0460E053
:10A0F0008C2F0E94065D83E090E00197F1F761E00C
:10A100008C2F0E94065D83E290E00197F1F760E0FA
:10A110008C2F0E94065D8091DB049091DC049927CE
:10A12000FC01EB53F54F6491FC01E158F54FE491CC
:10A13000F0E0EE0FFF1FEB59F54F8591949100E48D
:10A1400012E42FE030E0462F0E94E67A6115710597
:10A150008105910549F0DC01CB010196A11DB11DDE
:10A16000BC01CD019F7003C060E070E0CB010E9494
:10A17000128A20E030E048EC52E40E94648C209186
:10A180004E1130914F1140915011509151110E9438
:10A19000738A20E030E44CE156E40E94648C20E0B5
:10A1A00030E040E05FE30E94738ACF911F910F91EE
:10A1B00008951F920F920FB60F9211240BB60F92B3
:10A1C0002F933F934F935F936F937F938F939F93BF
:10A1D000AF93BF93EF93FF938091B900887F803650
:10A1E00009F49CC068F5883209F45BC090F48031B2
:10A1F00009F454C038F4882309F4F6C0883009F40F
:10A200004DC0F5C0883109F44CC0803209F45DC0FE
:10A21000EEC0803409F468C048F4803309F455C0B6
:10A22000883309F0E4C08093130DD8C0803509F459
:10A230004FC0883509F45DC0883409F0D8C0D6C055
:10A24000883909F4C7C0A8F4883709F467C038F41E
:10A25000883609F463C0803709F460C0C8C0883804
:10A2600009F4B8C0803909F45FC0803809F0BFC074
:10A270005BC0803B09F486C038F4803A09F466C0BC
:10A28000883A09F47FC0B3C0803C09F4A7C0883C79
:10A2900009F4A4C0883B09F48AC0A9C08091F00CDD
:10A2A00010C09091120D8091110D981770F5E091EA
:10A2B000120D81E08E0F8093120DF0E0EF50F34FFE
:10A2C00080818093BB0085EC86C08093130D8EC087
:10A2D000E091120D81E08E0F8093120D8091BB00F2
:10A2E000F0E0EF50F34F80839091120D8091110DAB
:10A2F0006EC0E091120D81E08E0F8093120D80915F
:10A30000BB00F0E0EF50F34F80838091140D81117A
:10A310006DC081E08093EF0C84EA61C083E080939C
:10A32000150D10929811CFCF80919811803208F0BE
:10A3300051C0E091981181E08E0F80939811809127
:10A34000BB00F0E0E858FE4E8083BDCF85EC8093E3
:10A35000BC001092150D80919811803230F4E0917C
:10A360009811F0E0E858FE4E10826091981170E06C
:10A37000E0917611F091771188E791E119951092AB
:10A38000981135C084E08093150D109275111092CC
:10A390007411E0917211F0917311199580917411FB
:10A3A000811105C081E08093741110925211E091E7
:10A3B000751181E08E0F80937511F0E0EE5AFE4E1C
:10A3C00080818093BB0090917511809174119817D2
:10A3D00008F479CF85E88093BC0009C085EC8093B0
:10A3E000BC001092150D03C01092130DBADDFF9141
:10A3F000EF91BF91AF919F918F917F916F915F91FD
:10A400004F913F912F910F900BBE0F900FBE0F9069
:10A410001F9018950895CF92DF92EF92FF9262DE1F
:10A420006B017C0120E030E040E050E40E94538D5D
:10A4300018161CF457DE6B017C0120E030E040E090
:10A4400050E4C701B6010E94538D18161CF44ADE71
:10A450006B017C0120E030E040E050E4C701B60130
:10A460000E94538D18161CF43DDE6B017C0120E028
:10A4700030E040E050E4C701B6010E94538D181649
:10A480002CF4FF90EF90DF90CF902CCEC701B60157
:10A49000FF90EF90DF90CF9008954F925F926F9270
:10A4A0007F928F929F92AF92BF92CF92DF92EF9264
:10A4B000FF92CF93DF93CDB7DEB768970FB6F894CE
:10A4C000DEBF0FBECDBF6B017C010E94B249698B1C
:10A4D0007A8B8B8B9C8B61E08091DD040E94355DD3
:10A4E00060E08091DB040E94355D0E948C476093A0
:10A4F0004A1170934B1180934C1190934D1123E3AB
:10A5000033E948E853E40E94648C20E030E040E8FE
:10A510005FE30E949E8B0E94628E26E636EA45EA41
:10A5200053E40E94738A60934E1170934F1180938D
:10A530005011909351116FDF6D877E878F87988BB5
:10A540000E948D494B015C016AE070E080E090E080
:10A550000E94965D69EE7BE08BEF9FE0A9D620E03C
:10A5600030E04AE754E4C701B6010E94738A6D8B5C
:10A570007E8B8F8B988F412C512C3201C12CD12C8A
:10A580007601C701B6010E94148A2D893E894F8940
:10A59000588D0E940E8A87FF5DC10E94B2492989A9
:10A5A0003A894B895C89621B730B840B950B0E9463
:10A5B000128A20E030E04AE754E40E94648CAB0148
:10A5C000BC0123E0CE01019630D7BE016F5F7F4F03
:10A5D00085EF9FE0BDD6CE010196F3D61CDF6B015F
:10A5E0007C010E948D499B01AC01281939094A0957
:10A5F0005B0949015A0131ED831637E09306A10446
:10A60000B1040CF441C020E030E0A901C701B6015B
:10A610000E94538D18165CF426EA3BE944EC5BE398
:10A62000C701B6010E940E8A87FF0BC02DC026EA23
:10A630003BE944EC5BEBC701B6010E94538D181651
:10A640001CF1C501B40128EE33E040E050E00E9467
:10A65000408BCA01B9010E94148A4B015C012D850F
:10A660003E854F855889C701B6010E949D8B20E029
:10A6700030E04AE754E40E94738AA50194010E94E5
:10A68000648C4B015C0103C0812C912C540165EF5B
:10A690007FE0CE01019657D76EEA78E0CE010196B1
:10A6A000CBD5BC0185EF9FE03ED6CE01019689D681
:10A6B00023E0B701A601CE010196B7D6BE016F5FB8
:10A6C0007F4FCE0107963FD763EF7AE0CE01079622
:10A6D000B3D5BC018FEE9FE026D6CE01079671D68A
:10A6E000CE0101966ED622E0B501A401CE010796F7
:10A6F0009CD66BE37BE0CE0101962DD765EF7FE022
:10A70000CE010196B0D566EF7AE096D56FEE7FE088
:10A71000AAD561EB78E090D5BE01695F7F4FA3D5E4
:10A720006CEA78E089D5BC018BEF9FE0BBD5CE0108
:10A73000019647D6CE01079644D620E030E0A90125
:10A74000C501B4010E94538D87FD05C06BE07AE01E
:10A750008FEE9FE099D522E0B501A401CE010196CC
:10A7600064D6BE016F5F7F4FCE010796ECD66CEAD0
:10A7700078E0CE01079660D5BC018FEE9FE092D5C0
:10A78000CE0107961ED6CE0101961BD66BEF7FE059
:10A79000CE010196D8D6CE0101960E94FD75CE015C
:10A7A00001960FD6C301B20125E030E040E050E051
:10A7B0000E94408B672B682B692B01F564EB78E0D6
:10A7C000CE010196C8D645E050E060E070E0CE01D1
:10A7D00001960E94B66ECE010196F3D56FEE7FE032
:10A7E000CE010196B0D645E050E06FEF7FEFCE018D
:10A7F00001960E94856DCE010196E3D56CEF7AE05B
:10A800008BEF9FE07BD565E070E080E090E00E94F8
:10A81000965D0E94B2496B017C0129893A894B8976
:10A820005C89C21AD30AE40AF50AF5DD6D877E87D2
:10A830008F87988B0E948D494B015C016AE070E024
:10A8400080E090E00E94965D3FEF431A530A630A4E
:10A85000730A97CE60E08091DD040E94355D6896B2
:10A860000FB6F894DEBF0FBECDBFDF91CF91FF9042
:10A87000EF90DF90CF90BF90AF909F908F907F90A0
:10A880006F905F904F90089581E08093D9048091FC
:10A89000DA04882339F088E08093101160E085E0C5
:10A8A00091E129C908958091DA0481110FC081E0F6
:10A8B0008093DA048093D90480910B11982F9460CF
:10A8C00090930B118C600E942C4117C08091D90489
:10A8D000882399F01092101160E085E091E10BD986
:10A8E0001092D90480910B118B7F80930B1188609B
:10A8F0000E942C411092DA040895C6CF2F923F9205
:10A900004F925F926F927F928F929F92AF92BF927F
:10A91000CF92DF92EF92FF920F931F93CF93DF932B
:10A92000CDB7DEB764970FB6F894DEBF0FBECDBFCC
:10A930007C0186ED9DE00E94BC5C40E855E260E051
:10A9400070E086ED9DE00E947F7A64E670E080E032
:10A9500090E00E94965D8CED95E0A0E0B0E08093E1
:10A96000DA0D9093DB0DA093DC0DB093DD0D64E662
:10A9700070E080E090E00E94965D8FEF898381E037
:10A980008A8386E88B831C821D821E821F82188622
:10A9900089E78987C701880F991F9C8B8B8B212C96
:10A9A000312CC12CD12C812C912C5401CE14DF04DC
:10A9B00044F086ED9DE0E0D7C114D10489F1760121
:10A9C0002FC08B899C89281639069CF786ED9DE05F
:10A9D0004AD2089744F049E050E0BE016F5F7F4FD4
:10A9E00086ED9DE0FCD165E070E080E090E00E94A3
:10A9F000965D00E010E0412C512C320186ED9DE087
:10AA000063D2892B31F484E0481651046104710447
:10AA10001CF4023011057CF19FEF291A390AC6CFC8
:10AA2000C501B4010E94148A4B015C01B701FF0CFF
:10AA3000880B990B0E94148A9B01AC01C501B401DB
:10AA40000E94648C64960FB6F894DEBF0FBECDBF33
:10AA5000DF91CF911F910F91FF90EF90DF90CF90FA
:10AA6000BF90AF909F908F907F906F905F904F902E
:10AA70003F902F90089586ED9DE026D2892B61F0BE
:10AA800086ED9DE0FFD1EAE0F0E0EC0FFD1FE00F66
:10AA9000F11F80830F5F1F4F65E070E080E090E062
:10AAA0000E94965D02301105C1F59A85898198133F
:10AAB00034C09B858B81981330C086ED9DE004D215
:10AAC000892B31F494E0491651046104710484F433
:10AAD0000930110581F086ED9DE0D4D1EAE0F0E087
:10AAE000EC0FFD1FE00FF11F80830F5F1F4FE5CFBD
:10AAF000043011057CF02D858C8590E0982F8827F7
:10AB0000820F911D092E000CAA0BBB0B880E991EFB
:10AB1000AA1EBB1E8FEFC81AD80A9FEF491A590AFE
:10AB2000690A790A6BCF2F923F924F925F927F9280
:10AB30008F929F92AF92BF92CF92DF92EF92FF924D
:10AB40000F931F93CF93DF9300D01F92CDB7DEB743
:10AB50006C0188E595E09C838B83E9E7F2E0FA835A
:10AB6000E9830BE51CE0EE24E394F12C9DE3292E10
:10AB7000312C2EE3422E512C30E1A32EB12C41E199
:10AB8000842E912C57E1752E809177029091780256
:10AB90008E159F050CF4EAC0F1E0CF16D10431F414
:10ABA000F80180819181E981FA8109C0F2E0CF1634
:10ABB000D10439F4E981FA8180819181F80191838E
:10ABC0008083E981FA8180819181009749F4EB814A
:10ABD000FC81828193819093D8048093D70427C00D
:10ABE0008130910549F4EB81FC81828193819093BE
:10ABF0005302809352021BC08230910549F4EB81CD
:10AC0000FC81828193819093D6048093D5040FC0F8
:10AC1000039769F4EB81FC81828193819093D40442
:10AC20008093D3046CEF7AE08BE590E167D3E98100
:10AC3000FA8181919191FA83E9838430910549F4F5
:10AC4000EB81FC81228133813093D2042093D104A3
:10AC500030C08530910549F4EB81FC81228133813C
:10AC60003093D0042093CF0424C08630910549F45A
:10AC7000EB81FC8122813381309351022093500279
:10AC800024C08730910549F4EB81FC812281338116
:10AC90003093CE042093CD0424C08A30910549F42A
:10ACA000EB81FC81228133813093CC042093CB044F
:10ACB0003AC08531910549F4EB81FC8122813381D1
:10ACC0003093CA042093C9042EC08631910549F4FB
:10ACD000EB81FC81228133813093C8042093C70427
:10ACE00022C087319105F9F4EB81FC812281338107
:10ACF000A901475051094230510540F4B092DE0499
:10AD0000A092DD049092DC048092DB04255031098E
:10AD10002230310540F43092DE042092DD0450925E
:10AD2000DC044092DB049C012B5031092A303105B0
:10AD300090F4EB81FC81228133813093D404209301
:10AD4000D304789EB001799E700D11246A547D4F12
:10AD50008BE590E1D3D2FFEFEF1AFF0A8B819C8144
:10AD600002969C838B830E5F1F4F0ECF0F900F9028
:10AD70000F900F90DF91CF911F910F91FF90EF9067
:10AD8000DF90CF90BF90AF909F908F907F905F901B
:10AD90004F903F902F900895FF920F931F93CF9362
:10ADA000DF93F82E0AE010E0C0E0D0E08F2D99D6B6
:10ADB000C80FD91F65E070E080E090E0B7D6015081
:10ADC0001109A1F7CE016AE070E00E94CB8ECB01A1
:10ADD000DF91CF911F910F91FF9008950895CF9229
:10ADE000DF92EF92FF920F931F93CF93DF936C014B
:10ADF0007A018B01C0E0D0E0CE15DF0589F0D801E3
:10AE00006D918D01D601ED91FC910190F081E02DC5
:10AE1000C6011995892B11F47E0102C02196ECCF51
:10AE2000C701DF91CF911F910F91FF90EF90DF90BD
:10AE3000CF900895FC01A089B1898C91A689B7892A
:10AE400082FD0FC09C91818D8F5F8F73228D821741
:10AE500049F0218DDF01A20FB11D5D969C93818F7A
:10AE600008958C910895FC01538D448D252F30E079
:10AE7000842F90E0821B930B541710F0CF96089507
:10AE800001970895FC01918D828D981761F0828D54
:10AE9000DF01A80FB11D5D968C91928D9F5F9F730E
:10AEA000928F90E008958FEF9FEF0895FC01918DB0
:10AEB000828D981731F0828DE80FF11D858D90E01D
:10AEC00008958FEF9FEF0895FC01918D228D892FBA
:10AED00090E0805C9F4F821B91098F7399270895A2
:10AEE00089E39DE0F1DF21E0892B09F420E0822F46
:10AEF000089586ED9DE0E8DF21E0892B09F420E04C
:10AF0000822F089583E79EE0DFDF21E0892B09F49B
:10AF100020E0822F0895FC01848DDF01A80FB11D70
:10AF2000A35ABF4F2C91848D90E001968F7399277F
:10AF3000848FA689B7892C93A089B1898C9180646C
:10AF40008C93938D848D981306C00288F389E02D2D
:10AF500080818F7D80830895EF92FF920F931F93DE
:10AF6000CF93DF93EC0181E0888F9B8D8C8D9813BC
:10AF700005C0E889F989808185FD23C0F62E0B8DF7
:10AF800010E00F5F1F4F0F731127E02E8C8DE8121A
:10AF90000BC00FB607FCFACFE889F989808185FFDD
:10AFA000F5CFCE01B8DFF2CF8B8DFE01E80FF11D9A
:10AFB000E35AFF4FF0820B8FEA89FB898081806220
:10AFC00007C0EE89FF896083E889F9898081806400
:10AFD000808381E090E0DF91CF911F910F91FF90EE
:10AFE000EF900895CF93DF93EC01888D8823C1F013
:10AFF000EA89FB89808185FD05C0A889B9898C9182
:10B0000086FD0EC00FB607FCF5CF808185FFF2CF1D
:10B01000A889B9898C9185FFEDCFCE017CDFE8CF7F
:10B02000DF91CF91089580E090E0892B19F06ADFDD
:10B0300081111BC080E090E0892B41F080E090E01E
:10B04000892B21F00E940000811112C080E090E065
:10B05000892B19F04EDF81110EC080E090E0892B22
:10B0600079F03EDF81110AC008950E940000E2CF0E
:10B070000E940000EBCF0E940000EFCF0C94000074
:10B08000089590E0FC013197E231F10508F04EC0DF
:10B090008827E955FF4F8F4F0C94F28E80918000E6
:10B0A0008F7703C0809180008F7D8093800008950A
:10B0B00080918000877FF9CF84B58F7702C084B5F7
:10B0C0008F7D84BD08958091B0008F7703C08091FB
:10B0D000B0008F7D8093B0000895809190008F77AD
:10B0E00007C0809190008F7D03C080919000877F82
:10B0F0008093900008958091A0008F7707C0809181
:10B10000A0008F7D03C08091A000877F8093A00066
:10B110000895809120018F7707C0809120018F7D55
:10B1200003C080912001877F809320010895CF93F1
:10B13000DF93EC0188819981009711F00E94C68FFE
:10B14000198218821D821C821B821A82DF91CF9184
:10B1500008950F931F93CF93DF93EC01888199811A
:10B16000009729F02A813B812617370788F48B0145
:10B170006F5F7F4F0E945E90009761F09983888394
:10B180001B830A832C813D81232B11F4FC01108247
:10B1900081E001C080E0DF91CF911F910F91089570
:10B1A000EF92FF920F931F93CF93DF93EC017B01FC
:10B1B0008A01BA01CEDF811103C0CE01B8DF07C01A
:10B1C0001D830C83B701888199810E944F91CE0124
:10B1D000DF91CF911F910F91FF90EF900895EF9223
:10B1E000FF920F931F93CF93DF93FC01248135814E
:10B1F0006115710511F480E018C041155105A1F0E9
:10B200007B01EC018A01020F131FB801A2DF882322
:10B2100091F3288139818C819D81B701820F931F21
:10B220000E944F911D830C8381E0DF91CF911F918C
:10B230000F91FF90EF900895CF93DF93EC0161158C
:10B24000710559F0FB0101900020E9F73197AF013A
:10B25000461B570BC4DF811102C0CE0168DFCE014F
:10B26000DF91CF910895CF93DF93EC01FB014481EF
:10B27000558160817181B3DF811102C0CE0157DF3A
:10B28000CE01DF91CF9108956115710549F0FB0161
:10B2900001900020E9F73197AF01461B570B9FCF74
:10B2A00080E00895FB01448155816081718197CFD1
:10B2B000EF92FF920F931F93CF93DF93EC018B01DB
:10B2C0006115710549F0CB010E948F857C01BC019D
:10B2D000CE013FDF811103C0CE0129DF07C0FD820F
:10B2E000EC82B801888199810E948885CE01DF9126
:10B2F000CF911F910F91FF90EF900895CF93DF931F
:10B30000EC016115710551F0FB0101900020E9F796
:10B310003197AF01461B570B43DF01C008DFCE0159
:10B32000DF91CF910895CF93DF93EC01FB01861756
:10B33000970751F0608171816115710521F0448199
:10B3400055812EDF01C0F3DECE01DF91CF9108954C
:10B350000F931F93CF93DF938C01EB01FC0180814E
:10B3600091810097B1F0688179816115710579F05B
:10B37000428153812C813D814217530740F00E9446
:10B380004F918C819D81F8019583848313C00E9425
:10B39000C68F88819981F801918380838A819B81FE
:10B3A000938382838C819D81958384831982188203
:10B3B0001B821A821D821C82DF91CF911F910F91F7
:10B3C0000895FC01808191810C94C68FEF92FF92C9
:10B3D0000F931F93CF93DF93CDB7DEB7A1970FB62F
:10B3E000F894DEBF0FBECDBF7C01CB01BA01F701DF
:10B3F00011821082138212821582148242E0420F5F
:10B400008E010F5F1F4F0E944085BC01C70176DF90
:10B41000A1960FB6F894DEBF0FBECDBFDF91CF91DE
:10B420001F910F91FF90EF900895EF92FF920F936D
:10B430001F93CF93DF93CDB7DEB7A1970FB6F894E4
:10B44000DEBF0FBECDBF7C01CB01BA01F701118277
:10B450001082138212821582148242E0420F8E0102
:10B460000F5F1F4F0E944085BC01C70147DFA196B7
:10B470000FB6F894DEBF0FBECDBFDF91CF911F9105
:10B480000F91FF90EF9008950F931F93CF93DF9349
:10B49000CDB7DEB7A2970FB6F894DEBF0FBECDBF13
:10B4A0008C01CB01BA01F801118210821382128241
:10B4B0001582148230E0AE014F5F5F4F0E94AC8571
:10B4C000BE016F5F7F4FC80119DFA2960FB6F894D7
:10B4D000DEBF0FBECDBFDF91CF911F910F910895B9
:10B4E0000F931F93CF93DF93CDB7DEB762970FB65D
:10B4F000F894DEBF0FBECDBF8C01CB01F8011182E5
:10B500001082138212821582148250E0BE016F5F96
:10B510007F4F0E949885BE016F5F7F4FC801EEDEAE
:10B5200062960FB6F894DEBF0FBECDBFDF91CF910C
:10B530001F910F910895FC011182108213821282D3
:10B5400015821482B5CEFC01118210821382128200
:10B5500015821482E8CEFC011182108213821282BD
:10B56000158214826115710549F0FB0101900020DC
:10B57000E9F73197AF01461B570B12CE0895DC0156
:10B58000ED91FC910190F081E02D1994DC01ED9199
:10B59000FC91DB0114964D915C9115976D917C9116
:10B5A0000280F381E02D1994EF92FF920F931F9385
:10B5B000CF93DF938C017B01C0E0D0E0F701EC0F6B
:10B5C000FD1F6491662361F0D801ED91FC9101901B
:10B5D000F081E02DC8011995892B11F02196EECF4D
:10B5E000CE01DF91CF911F910F91FF90EF900895C1
:10B5F0006115710579F0FB0101900020E9F73197A1
:10B60000AF01461B570BDC01ED91FC910280F381E9
:10B61000E02D199480E090E008954F925F926F9230
:10B620007F92EF92FF920F931F93CF93DF93CDB74B
:10B63000DEB7A1970FB6F894DEBF0FBECDBF7C0179
:10B64000FA01CB0119A2223008F42AE08E010F5D25
:10B650001F4F422E512C612C712CBF01A30192016E
:10B660000E946C8BF901CA01015011096A3014F46F
:10B67000605D01C0695CD8016C93232B242B252BC2
:10B6800061F7B801C701B4DFA1960FB6F894DEBF29
:10B690000FBECDBFDF91CF911F910F91FF90EF9023
:10B6A0007F906F905F904F900895CF92DF92EF92CE
:10B6B000FF920F931F93CF93DF93EC016A017B01FD
:10B6C0002115310579F4E881F9810190F081E02DAF
:10B6D000642FDF91CF911F910F91FF90EF90DF903A
:10B6E000CF9019942A303105D9F477FF18C06DE254
:10B6F00046DF8C0144275527BA014C195D096E09B4
:10B700007F092AE0CE0189DF800F911FDF91CF9161
:10B710001F910F91FF90EF90DF90CF9008952AE056
:10B72000B701A601CE01DF91CF911F910F91FF903C
:10B73000EF90DF90CF9071CF9A01AB01770F660B3E
:10B74000770BB3CF6AEF7AE053CF0F931F93CF936A
:10B75000DF93EC014DDF8C01CE01F4DF800F911FF0
:10B76000DF91CF911F910F9108950F931F93CF9366
:10B77000DF93EC010BDF8C01CE01E4DF800F911F22
:10B78000DF91CF911F910F91089532CF1F920F92A9
:10B790000FB60F9211240BB60F922F933F934F9336
:10B7A0005F936F937F938F939F93AF93BF93EF9329
:10B7B000FF9389E39DE0AFDBFF91EF91BF91AF91E4
:10B7C0009F918F917F916F915F914F913F912F91B9
:10B7D0000F900BBE0F900FBE0F901F9018951F92E9
:10B7E0000F920FB60F9211240BB60F922F933F9327
:10B7F0004F935F936F937F938F939F93AF93BF9379
:10B80000EF93FF9389E39DE015DBFF91EF91BF91EB
:10B81000AF919F918F917F916F915F914F913F91E8
:10B820002F910F900BBE0F900FBE0F901F90189589
:10B830001F920F920FB60F9211240BB60F922F93F7
:10B840003F934F935F936F937F938F939F93AF93A8
:10B85000BF93EF93FF9386ED9DE05DDBFF91EF914A
:10B86000BF91AF919F918F917F916F915F914F9118
:10B870003F912F910F900BBE0F900FBE0F901F9016
:10B8800018951F920F920FB60F9211240BB60F92BC
:10B890002F933F934F935F936F937F938F939F93D8
:10B8A000AF93BF93EF93FF9386ED9DE0C3DAFF91D3
:10B8B000EF91BF91AF919F918F917F916F915F9128
:10B8C0004F913F912F910F900BBE0F900FBE0F9095
:10B8D0001F9018951F920F920FB60F9211240BB65E
:10B8E0000F922F933F934F935F936F937F938F9319
:10B8F0009F93AF93BF93EF93FF9383E79EE00BDBA0
:10B90000FF91EF91BF91AF919F918F917F916F9137
:10B910005F914F913F912F910F900BBE0F900FBEF3
:10B920000F901F9018951F920F920FB60F9211242F
:10B930000BB60F922F933F934F935F936F937F9329
:10B940008F939F93AF93BF93EF93FF9383E79EE013
:10B9500071DAFF91EF91BF91AF919F918F917F919C
:10B960006F915F914F913F912F910F900BBE0F9070
:10B970000FBE0F901F901895CF93DF93EC01E881D5
:10B98000F9810680F781E02D1995EA89FB8980818C
:10B990008F7E8083EA89FB898081877F8083EA8923
:10B9A000FB8980818F778083EA89FB8980818F7D05
:10B9B00080838A8D898FDF91CF910895CF93DF9314
:10B9C000282F30E0F901E55CF34F8491F901EB5346
:10B9D000F54FD491F901E158F54FC491CC2389F08A
:10B9E00081114FDBEC2FF0E0EE0FFF1FEB59F54F0D
:10B9F000A591B491EC91ED2381E090E021F480E0F9
:10BA000002C080E090E0DF91CF9108951F93CF9323
:10BA1000DF93282F30E0F901E55CF34F8491F901C1
:10BA2000EB53F54FD491F901E158F54FC491CC2374
:10BA3000C1F0162F811125DBEC2FF0E0EE0FFF1F78
:10BA4000EF5DF34FA591B4918FB7F894111105C034
:10BA50009C91ED2FE095E92302C0EC91ED2BEC9346
:10BA60008FBFDF91CF911F910895CF93DF9390E027
:10BA7000FC01EB53F54F2491FC01E158F54F849103
:10BA8000882361F190E0880F991FFC01E95FF34F73
:10BA9000C591D491FC01EF5DF34FA591B491611173
:10BAA00009C09FB7F8948881209582238883EC9100
:10BAB0002E230BC0623061F49FB7F8943881822F37
:10BAC000809583238883EC912E2B2C939FBF06C0F7
:10BAD0008FB7F894E8812E2B28838FBFDF91CF9109
:10BAE0000895863308F0865390917B00282F2870A4
:10BAF000977F922B90937B0087702091DF0490E4D6
:10BB0000299F90011124822B80937C0080917A00E0
:10BB1000806480937A0080917A0086FDFCCF8091CA
:10BB200078002091790090E0922B08958F929F9257
:10BB3000AF92BF92CF92DF92EF92FF926B017C01A6
:10BB40000E948D494B015C01C114D104E104F10450
:10BB5000F1F00E948D49DC01CB0188199909AA09ED
:10BB6000BB09883E9340A105B10570F321E0C21ADC
:10BB7000D108E108F10888EE880E83E0981EA11C28
:10BB8000B11CC114D104E104F10419F7DDCFFF9019
:10BB9000EF90DF90CF90BF90AF909F908F900895DF
:10BBA000CF92DF92EF92FF920F931F93CF93DF9389
:10BBB000CDB7DEB7C054D1400FB6F894DEBF0FBE8C
:10BBC000CDBF0E94B24900916A1010916B10209174
:10BBD0006C1030916D106B017C01C01AD10AE20A21
:10BBE000F30A40EDC41647E0D406E104F10418F46A
:10BBF00080917210B5C060936A1070936B1080933F
:10BC00006C1090936D101092651010926410109249
:10BC10006310109262101092611061E080916610C2
:10BC2000F5DE6AEF70E080E090E080DF61E0809117
:10BC300066101BDF60E080916610E8DE64E170E072
:10BC400080E090E073DFF89461E080916610DEDEC2
:10BC50008BE990E00197F1F762E08091661005DFD3
:10BC600083E290E00197F1F780E00E94EB47672BB9
:10BC7000682B692B21F41092721078943EC081E0F9
:10BC80000E94EB47672B682B692BA9F38E010F5F8E
:10BC90001F4F6E018FEBC81A8EEFD80A780180E033
:10BCA0000E94EB47F701608371838283938381E075
:10BCB0000E94EB47F7016483758386839783F8E0DE
:10BCC000EF0EF11CEC14FD0451F7789420E030E005
:10BCD000F8014081518162817381C480D580E68002
:10BCE000F780411551056105710529F0C114D10492
:10BCF000E104F10421F41092721080E031C0F901E6
:10BD000083E0F595E7958A95E1F7EF59FF4E80813D
:10BD1000880F4C155D056E057F0508F481608083F2
:10BD20002F5F3F4F085F1F4F2832310589F6209162
:10BD3000651030E0409161108091621090E0840FB6
:10BD4000911D40916310840F911D40916410840FE8
:10BD5000911D99272817390771F681E08093721099
:10BD6000C05CDE4F0FB6F894DEBF0FBECDBFDF91D3
:10BD7000CF911F910F91FF90EF90DF90CF9008959A
:10BD8000CF92DF92EF92FF920BDF8823A1F1809197
:10BD900067108B3041F178F18551823060F5609108
:10BDA000611070E080E090E00E94128A20E030E0B4
:10BDB00040E853E40E94738A6B017C018091621019
:10BDC000682F70E080E090E00E94148A9B01AC0133
:10BDD000C701B6010E949E8B2DEC3CEC4CEC5DE360
:10BDE0000E94738A0CC06091611070E080E090E066
:10BDF0000E94128A04C060E070E080EC9FE7FF9030
:10BE0000EF90DF90CF900895CF92DF92EF92FF9264
:10BE1000CF93C6DE8823D1F1809167108B3029F053
:10BE2000A8F18551823048F031C06091631070E014
:10BE300080E090E00E94128A2DC0C09163106C2FA8
:10BE40006F7770E080E090E00E94148A20E030E09C
:10BE500040E853E40E94738A6B017C018091641076
:10BE6000682F70E080E090E00E94148A9B01AC0192
:10BE7000C701B6010E949E8B2DEC3CEC4CEC5DE3BF
:10BE80000E94738AC7FF06C0905804C060E070E04B
:10BE900080EC9FE7CF91FF90EF90DF90CF900895D7
:10BEA000EF92FF920F931F93CF93DF93C82F8B01D5
:10BEB0007A0183E50E9422416C2F80E19FE00E947D
:10BEC0003E500E94C04083E50E942241B80183E5B4
:10BED00090E00E944645E701CE018E199F093091FE
:10BEE000ED0C2091EE0C321731F080E19FE00E94C2
:10BEF000F34F8993F1CF8017910729F010927310B7
:10BF000081E080937410DF91CF911F910F91FF908A
:10BF1000EF900C94C040CF93DF93AC01990F660B68
:10BF2000770B2AE030E083E79EE0BFDBEC0183E79C
:10BF30009EE008DC8C0F9D1FDF91CF9108951F9329
:10BF4000CF93DF931F92CDB7DEB7162FAE014F5FB1
:10BF50005F4F61E070E0A4DF898190E002C09595B9
:10BF600087951A95E2F781700F90DF91CF911F911D
:10BF70000895CF93DF93D82FC62F83E50E942241E7
:10BF80006D2F80E19FE00E943E506C2F80E19FE08A
:10BF90000E943E50DF91CF910C94C040FF920F93CE
:10BFA0001F93CF93DF931F92CDB7DEB7182F062FC5
:10BFB000F42EAE014F5F5F4F61E070E071DF898169
:10BFC000FF2049F041E050E001C0440F0A95EAF734
:10BFD000482B498309C021E030E001C0220F0A95B7
:10BFE000EAF72095282329836981812FC2DF0F90EA
:10BFF000DF91CF911F910F91FF900895CF93DF9321
:10C0000042E00E946841EC0183E79EE09BDB8C0FDD
:10C010009D1FDF91CF910895AF92BF92CF92DF9293
:10C02000EF92FF921F93CF93DF93CDB7DEB72A979E
:10C030000FB6F894DEBF0FBECDBF182F41E850E118
:10C0400066E070E082E39F832BDF2091821030E076
:10C05000322F222780918110282B3A832983209127
:10C06000841030E0322F222780918310282B3C83CC
:10C070002B832091861030E0322F2227809185106B
:10C08000282B3E832D839E012F5F3F4F590155E79B
:10C09000C52E50E1D52EE12E9F81F92EF50161913B
:10C0A00071915F01F60121913191419151916F019F
:10C0B000072E000C880B990B2F83388749875A87E6
:10C0C0000E94148A2F81388549855A850E94738A77
:10C0D000F70161937193819391937F01F1E8CF16FA
:10C0E000F0E1DF06D9F62A960FB6F894DEBF0FBE50
:10C0F000CDBFDF91CF911F91FF90EF90DF90CF9058
:10C10000BF90AF9008953F924F925F926F927F924F
:10C110008F929F92AF92BF92CF92DF92EF92FF9257
:10C120000F931F93CF93DF9300D01F921F92CDB731
:10C13000DEB7982E0E94B2492B013C0120ED420E41
:10C1400027E0521E611C711C60E08091F6105EDCDD
:10C1500035E0832ECE0101966C01AA24A394B12C64
:10C1600055E0352E380EF601282D11922A95E9F763
:10C17000860127E0E22EF12C8091F7101FDC019759
:10C1800039F40E94B2496415750586059705A0F338
:10C190008091F71013DC892B39F40E94B2496415A1
:10C1A000750586059705A0F38091F81007DC892BAB
:10C1B00051F0F8012081C5010E2C01C0880F0A94AE
:10C1C000EAF7822B8083F1E0EF1AF108A8F60F5FFF
:10C1D0001F4F3012CECF0E94B249641575058605F7
:10C1E000970548F061E08091F61010DC60E070E0A7
:10C1F00080EC9FE72BC089818911B5CF9B818A8113
:10C20000980F990D8C818913AECF8D818D3009F0F7
:10C21000AACF61E08091F610F9DB6A818B8170E032
:10C22000762F6627680F711D072E000C880B990B5F
:10C230000E94148A20E030E040E85DE30E94738AA7
:10C2400023E333E948E853E40E949D8B0F900F905D
:10C250000F900F900F90DF91CF911F910F91FF9052
:10C26000EF90DF90CF90BF90AF909F908F907F9096
:10C270006F905F904F903F900895AF92BF92CF9292
:10C28000DF92EF92FF920F931F93CF93DF931F9252
:10C29000CDB7DEB75C01D62EE72EFC018585811176
:10C2A00005C0C5010E94044B811106C0F50113862B
:10C2B0001586148680E065C040E060EFC5010E94ED
:10C2C000984A01E0F12CC12C11E0C5010E94454AB9
:10C2D000682FC50169830E94454A6981613019F45C
:10C2E0008130B9F433C04F2D50E068131BC0F50105
:10C2F0008385181730F4E40FF51F8381802349F4F8
:10C3000002C0181731F060E0193058F4F5011487B5
:10C3100008C0F501EF0DF11D8381802B838361E05F
:10C3200009C0C12EF501E40FF51F9381802F809580
:10C3300089238383C5010E94694A1F5F000F11F49E
:10C34000F39401E0F7E0FF1508F0BFCF113408F4D3
:10C35000ADCFF501C386C11002C081E08587F5012C
:10C360008381882309F4A2CFD5011396ED2DFE2DEC
:10C370009501255F3F4F8D918193A217B307D9F7A0
:10C3800081E00F90DF91CF911F910F91FF90EF907F
:10C39000DF90CF90BF90AF9008959F92AF92BF92E1
:10C3A000CF92DF92EF92FF920F931F93CF93DF9381
:10C3B000CDB7DEB761970FB6F894DEBF0FBECDBF25
:10C3C0008C018CE0F8018183C12CD12C2FE5E22E69
:10C3D0003FE7B32E4FE1A42E5FE3952EF801848151
:10C3E00090E0C816D9060CF0A0C04C2DBE01665FC7
:10C3F0007F4FC8010E94084AF8018181893038F0D6
:10C40000F82EFCE0F81728F49CE0F92E02C089E031
:10C41000F82E8A85803139F0BE01665F7F4FC801F2
:10C420000E940D4C01C08CE08F1509F47AC0AE015A
:10C430004F5F5F4FBE01665F7F4FC8010E94A44BF4
:10C44000882309F46EC08A85803109F46AC08BE0C4
:10C45000F81651F0ECE0FE1629F0FAE0FF1206C0E3
:10C460009D8205C0BD8203C0ED8201C0AD82F8018E
:10C47000868197810E94044BBE01665F7F4FF80161
:10C48000868197810E94D94A40E06EE4F801868156
:10C4900097810E94984A40E06B81F80186819781DC
:10C4A0000E94984A40E06C81F801868197810E9441
:10C4B000984A8A85803139F040E06D81F8018681A3
:10C4C00097810E94984AF801868197810E94044BC7
:10C4D000BE01665F7F4FF801868197810E94D94A2D
:10C4E000F801408168E4868197810E94984A64E15E
:10C4F00070E080E090E01ADBF8018081882329F069
:10C500006AE070E080E090E011DBF80186819781BD
:10C510000E94044BF8018181F81608F4F82EF80106
:10C52000F182FFEFCF1ADF0A59CF61960FB6F89468
:10C53000DEBF0FBECDBFDF91CF911F910F91FF9056
:10C54000EF90DF90CF90BF90AF909F900895CF93E2
:10C55000DF930E94474210920A1180910E1182309F
:10C5600018F098E090930A1190910F11992339F0E7
:10C57000813029F480910A11846080930A1162E36A
:10C5800070E080E090E0D2DA6091101185E091E1F6
:10C590000E947B4D68EE73E080E090E0C7DA60E3D4
:10C5A00085E091E10E94964DCBE4D6E4CE0101975F
:10C5B000F1F760E385E091E10E94964D2197F1F754
:10C5C00060E385E091E10E94964D83E592E001975A
:10C5D000F1F760E285E091E10E94964D80910A11A9
:10C5E00080620E942C4184E080930B118CE00E94B9
:10C5F0002C4181E00E942C41CBE3DFE1CE01019789
:10C60000F1F782E080930C1186E00E942C4182E0D9
:10C610000E942C412197F1F7DF91CF910895FC0101
:10C6200044815581809117109091181084179507B7
:10C6300080F08091131090911410009751F0608158
:10C6400071816115710529F00E94569121E0892BB5
:10C6500009F020E0822F0895FF920F931F93CF934C
:10C66000DF93CDB7DEB72B970FB6F894DEBF0FBEC2
:10C67000CDBF86ED9DE080D940E855E260E070E0F6
:10C6800086ED9DE00E947F7A64E670E080E090E0B5
:10C690004DDA8CED95E0A0E0B0E08093DA0D909358
:10C6A000DB0DA093DC0DB093DD0D64E670E080E05F
:10C6B00090E03CDA8FEF898381E08A8386E88B8380
:10C6C0001C821D821E821F82188689E7898786ED5B
:10C6D0009DE00E94F25762E370E080E090E026DA8D
:10C6E00086ED9DE00E94335708974CF049E050E0FA
:10C6F000BE016F5F7F4F86ED9DE00E94EF5662E3C3
:10C7000070E080E090E012DA86ED9DE00E946457D0
:10C71000892B01F186ED9DE00E943357089784F440
:10C7200065E070E080E090E001DA00E010E0F12CDC
:10C7300086ED9DE00E94645702301105A4F50CC0FF
:10C7400049E050E0BE016F5F7F4F86ED9DE00E94A3
:10C75000EF56E6CFF12C27C086ED9DE00E9464578E
:10C76000892B99F465E070E080E090E0DFD9023039
:10C770001105F1F69A8589819813DACF9B858B8113
:10C780009813D6CFFF24F394D3CF86ED9DE00E947B
:10C790004257EAE0F0E0EC0FFD1FE00FF11F80834D
:10C7A0000F5F1F4FDFCF62E370E080E090E0BED903
:10C7B00086ED9DE0E1D88F2D2B960FB6F894DEBF65
:10C7C0000FBECDBFDF91CF911F910F91FF900895C4
:10C7D00096E0899FD0011124A957BF4E90967C9373
:10C7E0006E935F9791E091969C9391979091F3103F
:10C7F000E091F410F091F510992339F0309751F051
:10C80000811108C08091A31004C0309719F05C9684
:10C810008C91199408952F923F924F925F926F924C
:10C820007F928F929F92AF92BF92CF92DF92EF92C0
:10C83000FF920F931F93CF93DF93CDB7DEB763972C
:10C840000FB6F894DEBF0FBECDBF8B8B60E00DD965
:10C8500080919D11882329F082E090E0A0E0B0E073
:10C8600004C08FE090E0A0E0B0E08F87988BA98BA8
:10C87000BA8B6DEF7AE08BEF9FE00E947E596BEFF1
:10C880007FE0CE0101960E94A35A4AE050E06FEF8C
:10C890007FEFCE0101960E94B66ECE0101960E94F6
:10C8A000E159C12CD12C7601312C1D861E86212CFC
:10C8B00002E310E0412C512C32018B8912D9092E50
:10C8C000000CAA0BBB0B480E591E6A1E7B1E65E0AE
:10C8D00070E080E090E02AD90150110971F7809052
:10C8E000890290908A02A0908B02B0908C02C301C2
:10C8F000B2010E94148A20E030E040EA50E40E9435
:10C90000738A20E030E040E85AE30E94738A20E016
:10C9100030E048E452E40E94648CA50194010E9436
:10C920009D8B20E030E040E751E40E94738A2B01A8
:10C930003C01A50194016AE979E989E390E40E9448
:10C940009D8B9B01AC01C301B2010E94648C20E06D
:10C9500030E0A9010E949E8B20E030E040E251E4EB
:10C960000E94738A5B018C01232D3D854E85522DDB
:10C970000E94538D181624F43A2CBD860E87212E62
:10C9800020E030E0A901B501C8010E940E8A87FFAE
:10C9900004C0A12CB12C00E010E022E0A501B801F8
:10C9A000CE0101960E94155ABE016F5F7F4FCE01E6
:10C9B00007960E94A35A6AE07BE0CE0107960E9488
:10C9C0001C59BC0185EF9FE00E949359CE01079648
:10C9D0000E94E159CE0101960E94E15965EF7FE086
:10C9E000CE0101960E94A35A4AE050E060E070E058
:10C9F000CE0101960E94856DCE0101960E94E159FB
:10CA00000E94B2494090991150909A1160909B11E8
:10CA100070909C11930182010C591F4F2F4F3F4F73
:10CA2000061717072807390708F4C0C00E94B24943
:10CA30000E94128A4B015C01C301B2010E94148A58
:10CA400020E030E048EC51E40E949E8B9B01AC0159
:10CA5000C501B4010E940E8A87FDA8C06CE370E096
:10CA600080E090E063D89FEFC91AD90AE90AF90A71
:10CA70008F859889A989BA898C159D05AE05BF0552
:10CA80000CF016CF64E670E080E090E04FD8D9D784
:10CA900064E670E080E090E049D86FE07BE085EFED
:10CAA0009FE00E947E5965EF7FE0CE0101960E94D3
:10CAB000A35A44E150E060E070E0CE0101960E948C
:10CAC000B66ECE0101960E94E15922E0432D5D85AC
:10CAD0006E85722DCE0101960E94155ABE016F5FC0
:10CAE0007F4FCE0107960E94A35A6AE07BE0CE01F9
:10CAF00007960E941C59BC0185EF9FE00E94935944
:10CB0000CE0107960E94E159CE0101960E94E1599B
:10CB100065EF7FE0CE0101960E94A35A42E350E008
:10CB20006FEF7FEFCE010196F0D7CE0101960E9404
:10CB3000E159DDD762E370E080E090E00E94965D0D
:10CB400067E17BE0CE0101960E94AB5A65EF7FE082
:10CB5000CE0101960E9433596BE17BE00E941C5983
:10CB60006BEF7FE00E943359BC018BEF9FE00E9486
:10CB70009359CE0101960E94E15963960FB6F8943D
:10CB8000DEBF0FBECDBFDF91CF911F910F91FF9000
:10CB9000EF90DF90CF90BF90AF909F908F907F905D
:10CBA0006F905F904F903F902F900895A0D756CFF1
:10CBB0002F923F924F925F926F927F928F929F92AD
:10CBC000AF92BF92CF92DF92EF92FF920F931F939B
:10CBD000CF93DF93CDB7DEB72B970FB6F894DEBFB8
:10CBE0000FBECDBF7C018BEB8F838AEA888781E003
:10CBF000898784E68E9D90018F9D300D11243B879F
:10CC00002A87C12CD12C212C312C812C912C540120
:10CC10002E143F048CF1C501B4010E94148A20E057
:10CC200030E040E251E40E94648C4B015C01B701AA
:10CC3000FF0C880B990B0E94148A9B01AC01C50163
:10CC4000B4010E94648C2B960FB6F894DEBF0FBE21
:10CC5000CDBFDF91CF911F910F91FF90EF90DF90AB
:10CC6000CF90BF90AF909F908F907F906F905F908C
:10CC70004F903F902F9008952A853B85C216D3068A
:10CC800054F6C6016AE070E00E94DF8E892B49F4F9
:10CC900043E050E0BE01695F7F4F86ED9DE00E945A
:10CCA000EF5665E070E080E090E00E94965D3FEF17
:10CCB000C31AD30A00E010E0412C512C320186ED5A
:10CCC0009DE00E946457892B39F424E042165104F8
:10CCD000610471040CF09CCF063011050CF098CF64
:10CCE00086ED9DE00E946457892B69F086ED9DE0FA
:10CCF0000E944257E1E0F0E0EC0FFD1FE00FF11F52
:10CD000080830F5F1F4F65E070E080E090E00E943D
:10CD1000965D0630110501F599818F8198131CC02D
:10CD20009A818885981318C09B818985981314C0AF
:10CD30002C818D8190E0A0E0B0E0BA2FA92F982F30
:10CD40008827820F911DA11DB11D880E991EAA1E54
:10CD5000BB1E8FEF281A380A9FEF491A590A690A31
:10CD6000790AADCFCF92DF92EF92FF92CF93DF930C
:10CD7000CDB7DEB72C970FB6F894DEBF0FBECDBF90
:10CD800099270E94CC56BC01990F880B990B0E94E1
:10CD9000148A2DE038E643E55BE30E94738A6B0159
:10CDA0007C01209128023091290240912A02509161
:10CDB0002B020E940E8A18164CF06091100270919E
:10CDC000110280911202909113021BC020913C022B
:10CDD00030913D0240913E0250913F02C701B601A1
:10CDE0000E94538D87FF05C0C701B6010E948D4385
:10CDF00008C06091240270912502809126029091D2
:10CE0000270220E030E048EC52E40E94738A20E0E0
:10CE100030E048EA51E40E94738A20918D023091FB
:10CE20008E0240918F02509190020E94648C6B019F
:10CE30007C0169EE7CE085EF9FE00E94585965EF28
:10CE40007FE0CE0101960E94A35A42E350E060E0E9
:10CE500070E0CE0101968AD7CE0101960E94E15979
:10CE600022E0B701A601CE0107960E94155A65E29D
:10CE70007BE0CE0101960E94AB5ABE01695F7F4FF5
:10CE8000CE0101960E9433596FE17BE00E941C594C
:10CE9000BC018BEF9FE00E949359CE0101960E9446
:10CEA000E159CE0107960E94E1596BEF7FE0CE0178
:10CEB00001960E94A35A42E350E06FEF7FEFCE014C
:10CEC000019623D6CE0101960E94E15980919D11D1
:10CED000882331F060E273E080E090E00E94965D8C
:10CEE0002C960FB6F894DEBF0FBECDBFDF91CF9169
:10CEF000FF90EF90DF90CF900895CF92DF92EF9266
:10CF0000FF920F931F93CF93DF93CDB7DEB72C978C
:10CF10000FB6F894DEBF0FBECDBF93D56FED7CE0AA
:10CF20008BEF9FE00E9458596BEF7FE0CE01019696
:10CF30000E94A35A4AE050E060E070E0CE01019602
:10CF400015D7CE0101960E94E15966ED7CE085EF90
:10CF50009FE00E94585965EF7FE0CE0101960E9444
:10CF6000A35A44E150E06FEF7FEFCE010196CDD59B
:10CF7000CE0101960E94E15980911D1190911E11E0
:10CF80008430910541F468DB811117C010921E11A5
:10CF900010921D1112C0892B81F45EDB882339F0B9
:10CFA00084E090E090931E1180931D1106C054DB25
:10CFB0008111F6CF51DB8111F3CF80911D1190913A
:10CFC0001E11049769F16AEC7CE08BEF9FE00E94F0
:10CFD00058596BEF7FE0CE0101960E94A35A4AE0B8
:10CFE00050E060E070E0CE010196C0D6CE0101961F
:10CFF0000E94E1596BEF7FE0CE0101960E94A35A97
:10D000006BE07AE0CE0101960E941C5965EF7FE04B
:10D010000E943359BC018BEF9FE00E94935994C04A
:10D020008AE090E00E947E546B017C0120E030E0B9
:10D03000A9010E940E8A181634F08AE090E00E943E
:10D040007E546B017C010BE010E020E030E041EE0B
:10D0500053E4C701B6010E940E8A181684F420E03A
:10D0600030E0A901C701B6010E940E8A1816BCF073
:10D070006CEB7CE08BEF9FE00E94585941C001505F
:10D08000110969F368EC70E080E090E00E94965D21
:10D0900083E090E00E947E546B017C01D6CF20E0BB
:10D0A00030E048EC52E4C701B6010E940E8A87FFC7
:10D0B00002C021E001C020E0B701A601CE01079621
:10D0C0000E94155A64E27BE0CE0101960E94AB5AA1
:10D0D000BE01695F7F4FCE0101960E94335969E21C
:10D0E0007BE00E941C59BC018BEF9FE00E9493598A
:10D0F000CE0101960E94E159CE0107960E94E159A6
:10D100006BEF7FE0CE0101960E94A35A42E350E00C
:10D110006FEF7FEFCE010196F8D4CE0101960E9409
:10D12000E15963EB7CE085EF9FE00E94585965EF81
:10D130007FE0CE0101960E94A35A42E350E060E0F6
:10D1400070E0CE01019612D6CE0101960E94E159FF
:10D1500080919D11882331F060E273E080E090E0DF
:10D160000E94965D2C960FB6F894DEBF0FBECDBF21
:10D17000DF91CF911F910F91FF90EF90DF90CF90B3
:10D1800008951F93CF93DF93182FCDE9DCE0812F13
:10D190000E94715D899399936CE370E080E090E068
:10D1A0000E94965D8CE0CD3ED80789F70E946D42C3
:10D1B00020E030E040EA50E40E94738A20E030E052
:10D1C00040E85AE30E94738ADF91CF911F9108953E
:10D1D0002F923F924F925F926F927F928F929F9287
:10D1E000AF92BF92CF92DF92EF92FF920F931F9375
:10D1F000CF93DF93CDB7DEB7C954D1090FB6F894FA
:10D20000DEBF0FBECDBF2B013C0127962FAF279766
:10D2100028963FAF289729964FAF29972A965FAF58
:10D220002A970E94B24922966CAF7DAF8EAF9FAF16
:10D23000229727962FAD279728963FAD28972996B6
:10D240004FAD29972A965FAD2A9780E9481681E06D
:10D2500058066104710434F060E9462E5524539455
:10D26000612C712C203197E23907410551052CF4CE
:10D270002DA73EA74FA758AB0AC090E1C92E97E251
:10D28000D92EE12CF12CCDA6DEA6EFA6F8AA80912E
:10D290009D11882321F02DA73EA74FA758AB2296BA
:10D2A0006CAD7DAD8EAD9FAD229728EE33E040E0B2
:10D2B00050E00E94408B26962CAF3DAF4EAF5FAF43
:10D2C000269721E02DAB19A61AA61BA61CA68E0137
:10D2D000035F1F4FCC24DD247601C418D508E6086F
:10D2E000F708C9AADAAAEBAAFCAAC9A4DAA4EBA493
:10D2F000FCA42DA53EA54FA558A9C216D306E40649
:10D30000F5060CF02CC369A57AA58BA59CA50E94F7
:10D31000148A20E030E04AE754E40E94648CAB01B8
:10D32000BC0123E0C8010E94155AB80185EF9FE0B7
:10D330000E94A859C8010E94E1592DA53EA54FA5FC
:10D3400058A92A3031054105510594F42AE0269662
:10D350004CAD5DAD6EAD7FAD2697C8010E94445ABD
:10D36000B80185EF9FE00E94A859C8010E94E159C9
:10D37000CE0101960E940C606DE27BE08BEF9FE096
:10D380000E947E59AE014F5F5F4F1A01C12CD12C14
:10D390007601D1018D909D90AD90BD901D01A501AC
:10D3A0009401C501B4010E94738A9B01AC01C701BD
:10D3B000B6010E949E8B6B017C0123E0B501A401A4
:10D3C000C8010E94E659B801CE0143960E94A35AB3
:10D3D0006BE07AE0CE0143960E941C59BC018BEFB2
:10D3E0009FE00E945259CE0143960E94E159C80124
:10D3F0000E94E1592016310661F6C701B6010E946C
:10D40000628E6B017C01BDE24B16B1E05B066104EC
:10D4100071042CF016D360E080E00E943D4123E0CF
:10D42000B701A601CE0143960E94155A6AE37BE03C
:10D43000C8010E94AB5A65EF7FE0C8010E943359D2
:10D440006DE37BE00E941C59BE016D5E7F4F0E9420
:10D45000335962E47BE00E941C59BC018BEF9FE0D2
:10D460000E945259C8010E94E159CE0143960E9480
:10D47000E1592DEC3CEC4CE45FE3C701B6010E949E
:10D48000538D29813A814B815C812DA33EA34FA30B
:10D4900058A718160CF0A8C12AE939E949E95FE351
:10D4A000C701B6010E940E8A87FF9EC1CDA8CC207D
:10D4B00009F49AC189849A84AB84BC8420E030E06A
:10D4C000A901C501B4010E940E8ACD80DE80EF80E3
:10D4D000F884882309F12DA13EA14FA158A5CA01C6
:10D4E000B9010E94738A6EAB7FAB88AF99AFA70179
:10D4F0009601C701B6010E94738A9B01AC016EA917
:10D500007FA988AD99AD0E949E8B0E94628EA50175
:10D5100094010E94118C04C06BED7FE089EC9FE3C5
:10D5200020EE3EE245E652E40E94738A6EAB7FAB8A
:10D5300088AF99AF20E030E0A901C701B6010E9491
:10D540000E8A882309F12DA13EA14FA158A5CA0139
:10D55000B9010E94738A6AAF7BAF8CAF9DAFA50102
:10D560009401C501B4010E94738A9B01AC016AADAC
:10D570007BAD8CAD9DAD0E949E8B0E94628EA701FB
:10D5800096010E94118C04C06BED7FE089EC9FE353
:10D5900020EE3EE245E652E40E94738A6AAF7BAF1A
:10D5A0008CAF9DAF20E030E0A9016DA17EA18FA1DD
:10D5B00098A50E940E8A8823F9F0A5019401C5015F
:10D5C000B4010E94738A4B015C01A7019601C70157
:10D5D000B6010E94738A9B01AC01C501B4010E948F
:10D5E0009E8B0E94628E2DA13EA14FA158A50E9444
:10D5F000118C6B017C0108C08BEDC82E8FE0D82EFA
:10D6000089ECE82E8FE3F82E6BE37BE0C8010E94E3
:10D61000AB5A65EF7FE0C8010E94335965E47BE0B7
:10D620000E941C59BC018BEF9FE00E949359C801D6
:10D630000E94E1596BE37BE0C8010E94AB5A65EFA1
:10D640007FE0C8010E9433596FE57BE00E941C59BE
:10D65000BC0185EF9FE00E949359C8010E94E159E7
:10D6600021E04EA95FA968AD79ADCE014F960E9429
:10D67000155A21E04AAD5BAD6CAD7DADCE0149964A
:10D680000E94155A20EE3EE245E652E4C701B6017B
:10D690000E94738AAB01BC0121E0C8010E94155AA7
:10D6A000B801CE0143960E94A35A6BE07AE0CE0106
:10D6B00043960E941C59BE01675E7F4F0E943359FA
:10D6C0006BE07AE00E941C59BE01615E7F4F0E94B0
:10D6D0003359BC018FEE9FE00E949359CE014396CF
:10D6E0000E94E159C8010E94E159CE0149960E9469
:10D6F000E159CE014F960E94E1592DE2421621E0F8
:10D7000052066104710474F469A57AA58BA59CA5E1
:10D7100025E030E040E050E00E94408B672B682B12
:10D72000692BA1F565EF7FE0C8010E94A35A45E08F
:10D7300050E06FEF7FEFC80167D2C8010E94E15946
:10D7400068E67BE0C8010E94AB5A45E050E061EF1B
:10D750007FEFC8010BD3C8010E94E1596CEF7AE05A
:10D76000C8010E94AB5AC80190D1C8010E94E1597A
:10D770006FEE7FE0C8010E94A35A45E050E060E0F0
:10D7800070E0C801C2D1C8010E94E1596FEE7FE08C
:10D790008BEF9FE00E9452593FE143165104610410
:10D7A000710434F4C9A4DAA4EBA4FCA4F7FC11C0FE
:10D7B0006BEF7FE0C8010E94A35AC8010E94FD756B
:10D7C000C8010E94E1596CEF7AE08BEF9FE00E9464
:10D7D0007E59B201C30177FE04C069A97AA98BA959
:10D7E0009CA90E94965DA8C023E04DA15EA16FA1F7
:10D7F00078A5CE0143960E94155A6BE37BE0C801E1
:10D800000E94AB5A65EF7FE0C8010E9433596AE677
:10D810007BE00E941C59BE016D5E7F4F0E94335910
:10D8200063E47BE00E941C59BC0185EF9FE00E94ED
:10D830009359C8010E94E159CE0143960E94E159D3
:10D8400049855A856B857C8523E0CE0149960E94E7
:10D85000E6594D815E816F81788523E0C8010E9481
:10D86000E659B801CE0143960E94A35A6FE67BE0C9
:10D87000CE0143960E941C59BE01675E7F4F0E94F5
:10D88000335963E47BE00E941C59BC018FEE9FE09A
:10D890000E949359CE0143960E94E159C8010E940B
:10D8A000E159CE0149960E94E1592DE2421621E04C
:10D8B00052066104710474F469A57AA58BA59CA530
:10D8C00025E030E040E050E00E94408B672B682B61
:10D8D000692BE1F465EF7FE0C8010E94A35A4AE09A
:10D8E00050E06FEF7FEFC8018FD1C8010E94E1596E
:10D8F0006FEE7FE0C8010E94A35A4AE050E060E06A
:10D9000070E0C80102D1C8010E94E1596BEF7FE0CD
:10D91000C8010E94A35AC8010E94FD75C8010E9457
:10D92000E1596CEF7AE08BEF9FE00E947E59C301D2
:10D93000B2010E94965D1DAA0E94B2496B017C0152
:10D9400022962CAD3DAD4EAD5FAD2297C21AD30AE3
:10D95000E40AF50AC9A6DAA6EBA6FCA6C6CC65EFD2
:10D960007FE0CE010D960E94A35A4AE050E06FEF8F
:10D970007FEFCE010D96FAD1CE010D960E94E159AE
:10D98000CDA8CC2099F168E67BE0CE010D960E94EF
:10D99000AB5A45E050E061EF7FEFCE010D96E6D146
:10D9A000CE010D960E94E15980919D11882389F046
:10D9B00061E87CE0CE010D960E949B5A45E050E064
:10D9C00060E070E0CE010D96D1D1CE010D960E949F
:10D9D000E1596CEF7AE0CE010D960E94AB5ACE0170
:10D9E0000D9653D0CE010D960E94E1596FEE7FE067
:10D9F000CE010D960E94A35A4AE050E06FEF7FEFF0
:10DA0000CE010D9682D0CE010D960E94E159C75BE2
:10DA1000DF4F0FB6F894DEBF0FBECDBFDF91CF91C1
:10DA20001F910F91FF90EF90DF90CF90BF90AF903C
:10DA30009F908F907F906F905F904F903F902F902E
:10DA400008958091DA048823F9F08091D90488231D
:10DA5000D9F081E00E942C418BE39FE10197F1F71F
:10DA600060E080E00E943D4165E47DE085E091E179
:10DA70000E94D45A61E080E00E943D4165E37DE070
:10DA800085E091E10C94D45A0895CF93DF932091CF
:10DA9000DA042223A9F02091D904222389F0EC0191
:10DAA0006FED85E091E10E94BF5A8C819D81892BA9
:10DAB00039F0BE0185E091E1DF91CF910C94C65A17
:10DAC000DF91CF9108958091DA04882379F08091D5
:10DAD000D904882359F06FED85E091E10E94BF5A87
:10DAE00067E17AE085E091E10C94C55B089580914F
:10DAF000DA04882349F08091D904882329F060E072
:10DB000085E091E10C94AC4D08958F929F92AF9275
:10DB1000BF92EF92FF920F931F93CF93DF937C01FD
:10DB2000EB018A018091DA04882309F462C08091B4
:10DB3000D904882309F45DC077FF18C0C095D0953B
:10DB400061E08C2F0E943D41B70185E091E10E9488
:10DB5000C65A64E27DE085E091E10E94D45AF70163
:10DB6000848161E08C0F0E943D4133C00E94B24924
:10DB70008090991190909A11A0909B11B0909C1157
:10DB800024E6820E911CA11CB11C86169706A806DD
:10DB9000B90678F561E08C2F0E943D41B70185E020
:10DBA00091E10E94C65A63E17DE085E091E10E9427
:10DBB000D45AF701848161E08C0F0E943D410E949C
:10DBC000B2496093991170939A1180939B1190932D
:10DBD0009C11B801110F880B990BDF91CF911F9108
:10DBE0000F91FF90EF90BF90AF909F908F900C940B
:10DBF000965DDF91CF911F910F91FF90EF90BF90B5
:10DC0000AF909F908F900895AF92BF92CF92DF9286
:10DC1000EF92FF920F931F93CF93DF93CDB7DEB7B1
:10DC200062970FB6F894DEBF0FBECDBF2091DA0425
:10DC3000222309F48AC02091D904222309F485C043
:10DC40006A017B015C010E94B2490091AA11109106
:10DC5000AB112091AC113091AD110C591F4F2F4FCA
:10DC60003F4F061717072807390708F06EC0F7FE61
:10DC700008C087010095109560E0802F0E943D410B
:10DC800043C060E080E00E943D410E94B24928EE1E
:10DC900033E040E050E00E94408BBA01A9012AE045
:10DCA000CE0101960E94445ABE016F5F7F4FCE01A4
:10DCB00007960E94A35A6CE776E0CE0107960E9471
:10DCC0001C59BC01CE010D960E94A35ACE010796A5
:10DCD0000E94E159CE0101960E94E159BE01635FA5
:10DCE0007F4F85E091E10E94C65A09891A89E114A3
:10DCF000F10431F00E0D1F1D60E0802F0E943D41A8
:10DD0000CE010D960E94E159B50185E091E10E9496
:10DD1000C65A62E07DE085E091E10E94D45AF501A7
:10DD2000848160E0800F0E943D410E94B24960936F
:10DD3000AA117093AB118093AC119093AD11B60101
:10DD4000DD0C880B990B0E94965D62960FB6F894D5
:10DD5000DEBF0FBECDBFDF91CF911F910F91FF901E
:10DD6000EF90DF90CF90BF90AF900895BF92CF9289
:10DD7000DF92EF92FF920F931F93CF93DF93CDB774
:10DD8000DEB762970FB6F894DEBF0FBECDBF6C0151
:10DD90008B017A018091DA04882309F475C080919F
:10DDA000D904882309F470C077FF07C00095109547
:10DDB00060E0802F0E943D4146C060E080E00E940C
:10DDC0003D410E94B24928EE33E040E050E00E941D
:10DDD000408BBA01A9012AE0CE0101960E94445A63
:10DDE000BE016F5F7F4FCE0107960E94A35A6CE77A
:10DDF00076E0CE0107960E941C59BC01CE010D961B
:10DE00000E94A35ACE0107960E94E159CE010196C5
:10DE10000E94E159BE01635F7F4F85E091E10E945E
:10DE2000C65AB98860E08B2D0E943D41011511054D
:10DE300011F40B2D04C060E0802F0E943D41CE0103
:10DE40000D960E94E159B60185E091E10E94C65A03
:10DE500061EF7CE085E091E10E94D45AF601848173
:10DE600060E0800F0E943D410E94B2496093AA1178
:10DE70007093AB118093AC119093AD11B701FF0C6F
:10DE8000880B990B0E94965D62960FB6F894DEBFE0
:10DE90000FBECDBFDF91CF911F910F91FF90EF90FB
:10DEA000DF90CF90BF9008950F931F93CF93DF9390
:10DEB00000D000D0CDB7DEB720911F112223A9F0EA
:10DEC0008C016FEB7AE0CE0101960E94AB5AB8014B
:10DED000CE0101960E943359BC0183E79EE00E9467
:10DEE000B55BCE0101960E94E15926960FB6F894D3
:10DEF000DEBF0FBECDBFDF91CF911F910F9108956F
:10DF00004F925F926F927F928F929F92AF92BF9249
:10DF1000CF92DF92EF92FF920F931F93CF93DF93F5
:10DF2000CDB7DEB7CA54D1090FB6F894DEBF0FBE25
:10DF3000CDBF8C016CEF7AE0CE018B960E94AB5A7C
:10DF40006CEF7AE0CE0185960E94AB5ABE016F5FFE
:10DF50007F4F80E390E10E949D488D889E88AF8826
:10DF6000B88C498C5A8C6B8C7C8C8D8D9E8DAF8D32
:10DF7000B8A127968CAF9DAFAEAFBFAF2797C801B2
:10DF80000197039708F0D4C1A3019201C501B40120
:10DF900090580E94118C2BED3FE049EC5FE30E940A
:10DFA0009E8B2091A5023091A6024091A70250912C
:10DFB000A8020E949E8B6B017C0120E030E0A90149
:10DFC0000E940E8A87FD09C0C092A611D092A711A7
:10DFD000E092A811F092A91110C02BED3FE049EC9E
:10DFE00050E4C701B6010E949E8B6093A611709306
:10DFF000A7118093A8119093A911C090A611D09059
:10E00000A711E090A811F090A9112BED3FE049EC89
:10E0100050E4C701B6010E94538D181684F42BED0D
:10E020003FE049EC50E4C701B6010E949D8B60932C
:10E03000A6117093A7118093A8119093A91120E0C5
:10E0400030E044E353E46091A6117091A7118091F0
:10E05000A8119091A9110E94738A2BED3FE049E429
:10E0600050E40E94648C6093A2117093A31180937A
:10E07000A4119093A5110E94FD8C4AE0CE01C79691
:10E080000E94705A62E77BE0CE01C1960E94AB5AB3
:10E09000BE01695C7F4FCE01C1960E9433596CE787
:10E0A0007BE00E941C59BC0181E090E10E949359E1
:10E0B000CE01C1960E94E159CE01C7960E94E15956
:10E0C000C090A211D090A311E090A411F090A511DE
:10E0D00020E030E044EB52E4C701B6010E940E8A12
:10E0E000181694F020E030E040E05FE3C701B6018D
:10E0F0000E949E8B0E94FD8C4AE0CE01C7960E9432
:10E10000705A63E87BE023C020E030E044E353E44E
:10E11000C701B6010E940E8A1816A4F1A701960144
:10E1200060E070E884E393E40E949D8B6093A21109
:10E130007093A3118093A4119093A5110E94FD8C5C
:10E140004AE0CE01C7960E94705A66E87BE0CE0195
:10E15000C1960E94AB5ABE01695C7F4FCE01C19649
:10E160000E943359BC01CE018B960E949359CE0177
:10E17000C1960E94E159CE01C7960E94E15967E716
:10E1800077E063C020E030E047E853E4C701B60120
:10E190000E940E8A181604F120E030E044E353E4B4
:10E1A000C701B6010E949D8B20E030E040E05FE3B4
:10E1B0000E949E8B6093A2117093A3118093A4116F
:10E1C0009093A5110E94FD8C4AE0CE01C7960E9453
:10E1D000705A66E87BE01FC0A701960160E070E01E
:10E1E00084EB93E40E949D8B20E030E040E05FE30D
:10E1F0000E949E8B6093A2117093A3118093A4112F
:10E200009093A5110E94FD8C4AE0CE01C7960E9412
:10E21000705A63E87BE0CE01C1960E94AB5ABE0102
:10E22000695C7F4FCE01C1960E943359BC01CE017B
:10E230008B960E949359CE01C1960E94E159CE015E
:10E24000C7960E94E15969E87BE0CE0185960E945D
:10E250007E59BE01655D7F4FCE01C1960E94A35AD3
:10E260004AE050E060E070E0CE01C1967FDDCE0173
:10E27000C1960E94E1590E94B2492091AA113091A1
:10E28000AB114091AC115091AD1169017A01A4E636
:10E29000CA0ED11CE11CF11CC616D706E806F90609
:10E2A00008F434C228962FAF289729963FAF2997B4
:10E2B0002A964FAF2A972B965FAF2B970E94B249B1
:10E2C0000E94128A6B017C0128962FAD289729960F
:10E2D0003FAD29972A964FAD2A972B965FAD2B9786
:10E2E000CA01B9010E94148A20E030E048EC51E4F0
:10E2F0000E949E8B9B01AC01C701B6010E940E8A51
:10E3000087FD04C26BE07AE0CE01C1960E94AB5A51
:10E31000BE016B5D7F4FCE01C1960E943359BC0197
:10E32000CE018B960E945259CE01C1960E94E159AE
:10E33000C8010297029708F0C3C120E030E040E234
:10E3400051E4C501B4010E94738A6B017C0120E095
:10E3500030E040E251E4C301B2010E94738A4B01F4
:10E360005C0120E030E040E251E427966CAD7DADE9
:10E370008EAD9FAD27970E94738A2B013C010E94AE
:10E38000B2492091D60B3091D70B4091D80B5091C8
:10E39000D90B621B730B840B950B0E94128A20E031
:10E3A00030E04AE754E40E94648CAB01BC0123E0F6
:10E3B000CE01C7960E94155A6BE37BE0CE01C19651
:10E3C0000E94AB5ABE01695C7F4FCE01C1960E948C
:10E3D00033596CE776E00E941C59BC018FEE9FE038
:10E3E0000E949359CE01C1960E94E159CE01C79671
:10E3F0000E94E1596FEE7FE0CE01C1960E94A35AC0
:10E4000061E070E1CE01C1960E943359BE01655DA5
:10E410007F4F0E943359BC01CE018B960E949359C5
:10E42000CE01C1960E94E1596BE87BE08BEF9FE043
:10E430000E947E5921E0B701A601CE01C1960E943B
:10E44000155ABE016F5C7F4F8BEF9FE00E945259BF
:10E45000CE01C1960E94E15921E0B301A201CE0193
:10E46000CD960E94155A21E0B501A401CE01C796B0
:10E470000E94155A6BE07AE0CE01C1960E94AB5A19
:10E48000BE01695C7F4FCE01C1960E9433596BE09B
:10E490007AE00E941C59BE01635C7F4F0E94335991
:10E4A00066E97BE00E941C59BC018BEF9FE00E9453
:10E4B0005259CE01C1960E94E159CE01C7960E94E1
:10E4C000E159CE01CD960E94E159A7019601C701FD
:10E4D000B6010E94738A6B017C01A5019401C501FC
:10E4E000B4010E94738A9B01AC01C701B6010E946E
:10E4F0009E8B6B017C01A3019201C301B2010E94BA
:10E50000738A9B01AC01C701B6010E949E8B0E94D9
:10E51000628E6B017C0160939E1170939F118093BA
:10E52000A0119093A1116AE97BE08BEF9FE00E941C
:10E53000445921E0B701A601CE01C1960E94155AA7
:10E54000BE016F5C7F4FCE01C7960E94A35A68EA56
:10E550007BE0CE01C7960E941C59BC0181E090E18E
:10E560000E949359CE01C7960E94E159CE01C196EF
:10E570000E94E15961E070E18BEF9FE00E945259E7
:10E58000C0909E11D0909F11E090A011F090A11129
:10E5900020E030E04AE754E4C701B6010E94538D01
:10E5A00087FD29C020E030E04AE754E4C701B60106
:10E5B0000E94648CAB01BC0123E0CE01C1960E9495
:10E5C000E659BE016F5C7F4FCE01C7960E94A35AE9
:10E5D00069EA7BE0CE01C7960E941C59BC0181E02C
:10E5E00090E10E949359CE01C7960E94E159CE0155
:10E5F000C1960E94E15920E030E64AE656E4609177
:10E600009E1170919F118091A0119091A1110E9473
:10E610000E8ABE01655D7F4F87FF4EC0CE01C19659
:10E620000E94A35A6AE37BE0CE01C1960E941C5966
:10E630006BEF7FE00E943359BC018BEF9FE00E949B
:10E640009359CE01C1960E94E1590330110599F406
:10E650006BEF7FE0CE01C1960E94A35ACE01C19616
:10E66000CCD2CE01C1960E94E1596CEF7AE08BEFDB
:10E670009FE00E947E596EE97BE0CE01C1960E9428
:10E68000AB5A61E070E1CE01C1960E943359BC01E2
:10E69000CE01C7960E94A35A4AE050E06FEF7FEF89
:10E6A000CE01C79632DACE01C7960E94E159CE015B
:10E6B000C1960E94E15904C08BEF9FE00E949359DC
:10E6C0006AE070E080E090E00E94965DCE01859661
:10E6D0000E94E159CE018B960E94E159C65BDF4F43
:10E6E0000FB6F894DEBF0FBECDBFDF91CF911F9163
:10E6F0000F91FF90EF90DF90CF90BF90AF909F90E1
:10E700008F907F906F905F904F9008956CEF7AE0BC
:10E71000CE01C1960E94AB5ACE01C196B6D9CE01A8
:10E72000C1960E94E159BE016B5D7F4F85E091E18A
:10E730000E94C65AE7CDCF92DF92EF92FF920F93DD
:10E740001F93CF93DF93CDB7DEB72C970FB6F89416
:10E75000DEBF0FBECDBF68E17EE0CE0101960E9414
:10E760009B5A4CE251E06FEF7FEFCE010196CDD97D
:10E77000CE0101960E94E1590E94045F00E010E082
:10E7800064E670E080E090E00E94965D0E94045F85
:10E790006B017C010F5F1F4F033011058CF39B0150
:10E7A000AC010A3011057CF40E94A38E8111E8CFE0
:10E7B00020E030E046E153E4C701B6010E940E8A32
:10E7C00087FDCEC004C00E94A38E882389F339D967
:10E7D0006EE170E080E090E00E94965D0E948C47C0
:10E7E0006B017C0164E670E080E090E00E94965D41
:10E7F00062EF78E08BEF9FE00E947E5921E0B70145
:10E80000A601CE0101960E94155ABE016F5F7F4F8F
:10E810008BEF9FE00E945259CE0101960E94E15970
:10E820006BEF7FE0CE0101960E94A35A4AE050E0D0
:10E8300060E070E0CE01019699DACE0101960E9467
:10E84000E15941D966E17AE08BEF9FE00E9444599B
:10E85000C092B211D092B311E092B411F092B511FE
:10E8600020E030E040EF51E4C701B6010E94538D33
:10E8700087FD03C06EEA7DE052C020E030E040ED4D
:10E8800051E4C701B6010E94538D87FD1EC06EE999
:10E890007DE0CE0101960E949B5A4AE050E06FEF66
:10E8A0007FEFCE01019631D9CE0101960E94E15948
:10E8B0008091AD02882331F06CED75E080E090E04E
:10E8C0000E94965D6EE87DE02AC020E030E040EBDB
:10E8D00051E4C701B6010E94538D87FD03C060E873
:10E8E0007DE01DC061E77DE0CE0101960E949B5A4C
:10E8F0004AE050E06FEF7FEFCE01019606D9CE01DE
:10E9000001960E94E1598091AD02882331F06CEDAF
:10E9100075E080E090E00E94965D63E67DE0CE01C8
:10E9200001960E949B5A4AE050E06FEF7FEFCE01C4
:10E930000196EBD8CE0101960E94E1596CE271E09C
:10E9400080E090E00E94965D8091AD02882309F4FA
:10E9500045C168EE73E080E090E00E94965D3EC1A4
:10E960000E94045F6B017C016093B2117093B3113C
:10E970008093B4119093B5110E94C05E6093AE1164
:10E980007093AF118093B0119093B11121E0B70152
:10E99000A601CE0107960E94155A62EF78E0CE01DB
:10E9A00001960E94AB5ABE01695F7F4FCE0101966E
:10E9B0000E943359BC018BEF9FE00E949359CE0116
:10E9C00001960E94E159CE0107960E94E1594091BB
:10E9D000AE115091AF116091B0117091B11121E061
:10E9E000CE0107960E94155A65EF79E0CE01019697
:10E9F0000E94AB5ABE01695F7F4FCE0101960E9413
:10EA00003359BC018BEF9FE00E945259CE01019611
:10EA10000E94E159CE0107960E94E15962E27BE033
:10EA20008BEF9FE00E9444596CEF7AE0CE01019693
:10EA30000E94AB5A44E150E060E070E0CE010196E4
:10EA400095D9CE0101960E94E1596091B211709161
:10EA5000B3118091B4119091B5110E94FD8C4AE0E0
:10EA6000CE0101960E94705ABE016F5F7F4F85EF05
:10EA70009FE00E94A859CE0101960E94E15960E0F2
:10EA800086E00E943D4165EF7FE085E091E10E94D4
:10EA9000C65A6FED85E091E10E94BF5A63E879E0C4
:10EAA00085E091E10E94C55B6091AE117091AF115C
:10EAB0008091B0119091B1110E94FD8C4AE050E01C
:10EAC00085E091E10E949C5B62E27BE085E091E160
:10EAD0000E94C55B64E670E080E090E00E94965D75
:10EAE000C090B211D090B311E090B411F090B51174
:10EAF00020E030E040EF51E4C701B6010E94538DA1
:10EB000087FD03C069E07EE054C020E030E040EDC6
:10EB100051E4C701B6010E94538D87FD1FC069EF04
:10EB20007DE0CE0101960E949B5A4AE050E06FEFD3
:10EB30007FEFCE0101960E94856DCE0101960E9465
:10EB4000E1598091AD02882331F06CED75E080E0F1
:10EB500090E00E94965D69EE7DE02BC020E030E001
:10EB600040EB51E4C701B6010E94538D87FD03C0FD
:10EB70006BED7DE01EC06CEC7DE0CE0101960E9445
:10EB80009B5A4AE050E06FEF7FEFCE0101960E9462
:10EB9000856DCE0101960E94E1598091AD028823D6
:10EBA00031F06CED75E080E090E00E94965D6EEBD8
:10EBB0007DE0CE0101960E949B5A4AE050E06FEF43
:10EBC0007FEFCE0101960E94856DCE0101960E94D5
:10EBD000E15962E370E080E090E0BFCE2C960FB682
:10EBE000F894DEBF0FBECDBFDF91CF911F910F9183
:10EBF000FF90EF90DF90CF900895CF93DF93FC01CB
:10EC000024813581232B69F0EC01BC0183E79EE070
:10EC10000E94B55BBE0189E39DE0DF91CF910C942A
:10EC2000B55BDF91CF910895CF92DF92EF92FF9283
:10EC30000F931F93CF93DF93CDB7DEB728970FB60F
:10EC4000F894DEBF0FBECDBF823409F441C0CCF4CE
:10EC5000803309F45DC07CF4833209F450C08A32F9
:10EC600009F076C067E875E083E190E10E947E5983
:10EC70008FEF9FEF6AC0813309F459C08134E9F006
:10EC800067C08136D1F02CF4833469F1843439F0D3
:10EC90005FC0833641F1E4F0843609F059C08091B9
:10ECA0000B1090910C10892B09F4F7C087E090E1CC
:10ECB0000E94474F97FF74C0F0C06EE775E083E194
:10ECC00090E10E947E5980911B1190911C113DC0D2
:10ECD0006BE775E083E190E10E947E5910929D11EF
:10ECE0008CEF9FEF32C061E875E083E190E10E9414
:10ECF0007E5981E080939D118DEF9FEF26C064E8DF
:10ED000075E083E190E10E947E598EEF9FEF1DC078
:10ED100065E775E087E090E10E947E5965E775E060
:10ED200083E190E10E947E5980E090E00EC068E8A7
:10ED300075E087E090E10E947E5968E875E083E124
:10ED400090E10E947E5981E090E00E94481FACC093
:10ED50001A8219821C821B821E821D828F83188652
:10ED6000BE01695F7F4FCE0101960E947E59BE01B0
:10ED70006F5F7F4F87E090E10E94A859CE01019616
:10ED80000E94E15987E090E10E94474FCB010E9429
:10ED9000481F64E670E080E090E00E94965D84C0C9
:10EDA00080911F11882361F06CE57DE083E79EE090
:10EDB0000E94D45A67E070E183E79EE00E94B55B51
:10EDC00087E090E10E94474F0AEF1FEF2FEF3FEFE0
:10EDD00068017901C61AD70AE80AF90AB701A6013B
:10EDE0002AE0CE0101960E94445ABE016F5F7F4F18
:10EDF00087E090E10E94A859CE0101960E94E15956
:10EE000087E090E146C08FEFE81AF80A89EEE8162D
:10EE100083E0F80609F446C06EE170E080E090E01F
:10EE20000E94965DAED0182F112369F31033D4F1F0
:10EE30006AE270E0611B710917FD73954AE0CE012B
:10EE400001960E94705ABE016F5F7F4F83E190E18F
:10EE50000E94A859CE0101960E94E15963E170E138
:10EE600087E090E10E94935980911F11882379F0E7
:10EE700065E57DE083E79EE00E94D45A612F83E739
:10EE80009EE00E94BF5A83E79EE00E94A25B83E15E
:10EE900090E10E94474FCB0158CF73D0182FE12C3F
:10EEA000F12CC2CF1451C4CF28960FB6F894DEBF10
:10EEB0000FBECDBFDF91CF911F910F91FF90EF90CB
:10EEC000DF90CF9008950F931F93CF93DF93C82FB8
:10EED000D62F86E0C89FF0011124E957FF4E11A2FA
:10EEE000878D90A181309105F1F01CF4892B49F0B8
:10EEF00043C082309105A9F10397F1F560E070E01D
:10EF000034C06623C9F161E070E08C2F0E94E86391
:10EF10000E94B2496093DF107093E0108093E1107B
:10EF20009093E21029C00E94B2490091DF10109125
:10EF3000E0102091E1103091E210AB01BC01401BC8
:10EF4000510B620B730B8091F1109091F210A0E0C5
:10EF5000B0E084179507A607B70718F462E070E0E1
:10EF600004C0D11109C063E070E08C2FDF91CF9114
:10EF70001F910F910C94E863DF91CF911F910F9136
:10EF800008956F927F928F929F92AF92BF92CF928D
:10EF9000DF92EF92FF920F931F93CF93DF9381E065
:10EFA0008093F3100E94B2490091E3101091E41095
:10EFB0002091E5103091E610AB01BC01401B510BD4
:10EFC000620B730B8091EF109091F010A0E0B0E015
:10EFD00084179507A607B70708F00AC1C0E080911B
:10EFE000ED10C81760F4E091E910F091EA10EC0F11
:10EFF000F11D62E080810E94355DCF5FF0CF712C02
:10F00000812C912C540183948091EE10781608F095
:10F010005FC0072D10E0E091EB10F091EC10E00FD5
:10F02000F11F61E080810E94355DE091EB10F0916D
:10F03000EC10E00FF11F60E080810E94065DD501B9
:10F04000C401072C04C0880F991FAA1FBB1F0A9474
:10F05000D2F76C017C01E094F094612C8091ED106A
:10F060006816F8F4C62DD0E0E091E910F091EA10AE
:10F07000EC0FFD1F80810E94DE5C2496CC0FDD1F0B
:10F08000C957DF4E892B29F4888199818C299D29C4
:10F0900004C0888199818E219F21998388836394FC
:10F0A000DDCFE091EB10F091EC10E00FF11F61E08B
:10F0B00080810E94065D8091EB109091EC10FC0124
:10F0C000E00FF11F60E080810E94355D73949CCF5A
:10F0D000E3EAF0E18FEF9FEF23813481232B21F4CA
:10F0E0001082928381831582369620E1EF3DF207EC
:10F0F00099F710E096E0F92E8091ED10181708F0BE
:10F1000051C000E0C12FD0E0CC0FDD1FC157DF4E52
:10F110002091EE10021708F043C068817981002E1B
:10F1200002C0769567950A94E2F761707727129F7F
:10F1300090011124200F311DE091E710F091E810AB
:10F14000E20FF31F4081E7E8F0E180E0A58DB68D86
:10F15000A217B30711F461701AC08F5F36968A3018
:10F16000A9F7672BD9F0E3EAF0E180E090E0508165
:10F1700051110FC0F89EF001F99EF00D1124E957CE
:10F18000FF4E448F368F258F10A2178E61E09BDED5
:10F1900005C0019636968A30910549F70F5FB8CFC2
:10F1A0001F5FAACF80E090E0C0E0FC01E957FF4E6E
:10F1B00021A12111C1E006968C339105B1F70E947F
:10F1C000B2496093E3107093E4108093E51090933C
:10F1D000E610CC2369F08091A810882349F0809133
:10F1E000A6109091A710019719F48091A31003C065
:10F1F0001092F31080E0DF91CF911F910F91FF905B
:10F20000EF90DF90CF90BF90AF909F908F907F90C6
:10F210006F9008958F929F92AF92BF92CF92DF929C
:10F22000EF92FF920F931F93CF93DF93DB01CD916A
:10F23000DC91DC011C96ED91FC911D97CE17DF0748
:10F240000CF04AC0FE01EE0FFF1F1A968D919C91A3
:10F250001B97E80FF91F80809180C170DD27B1E016
:10F26000CB27209719F404E610E002C00CE91FEF49
:10F2700079015A016B01020F131FB801C4010E94EA
:10F280007F4E892B99F40E0D1F1DB801C4010E94F9
:10F290007F4E892B71F4B8016E0D7F1DC4010E9451
:10F2A0007F4E892BE1F023E030E005C021E030E023
:10F2B00002C022E030E0F501808191810196821741
:10F2C000930734F011821082F601808191810196BA
:10F2D00091838083CE0105C081E090E002C08FEF72
:10F2E0009FEFDF91CF911F910F91FF90EF90DF90F3
:10F2F000CF90BF90AF909F908F9008951F93CF9322
:10F30000DF93CDB7DEB7A8970FB6F894DEBF0FBE78
:10F31000CDBF182F0E9447428EE10E94224162E039
:10F3200080E19FE00E943E5060E080E19FE00E940B
:10F330003E500E94C0408EE10E94224161E080E187
:10F340009FE00E943E5060E280E19FE00E943E50BC
:10F350000E94C04080E290E090933410809333107C
:10F3600080E090E8A9E8B4E480937202909373027D
:10F37000A0937402B093750280E090E0A5E7B4E436
:10F3800080936E0290936F02A0937002B09371020B
:10F39000BE016F5F7F4F80E390E10E9450481123D0
:10F3A00009F49CC080911F11882309F497C06CEA6E
:10F3B0007EE083E79EE00E94D45A83E79EE00E94AD
:10F3C000A25B6CE97EE083E79EE00E94D45ABE0116
:10F3D0006F5F7F4F83E79EE00E94A55B6CE87EE055
:10F3E00083E79EE00E94D45A4D855E856F857889BB
:10F3F0002AE030E083E79EE00E94555B83E79EE0D1
:10F400000E94A25B6CE77EE083E79EE00E94D45AF4
:10F4100049895A896B897C892AE030E083E79EE03C
:10F420000E94555B83E79EE00E94A25B6CE67EE053
:10F4300083E79EE00E94D45A20E030E040E251E4AD
:10F44000698D7A8D8B8D9C8D0E94738A42E050E08D
:10F450000E94464267EA7BE083E79EE00E94A55B4C
:10F460006CE57EE083E79EE00E94D45A20E030E025
:10F4700040E251E46D8D7E8D8F8D98A10E94738A3C
:10F4800042E050E00E94464267EA7BE083E79EE06C
:10F490000E94A55B6CE47EE083E79EE00E94D45A64
:10F4A00020E030E040E251E469A17AA18BA19CA167
:10F4B0000E94738A42E050E00E94464267EA7BE085
:10F4C00083E79EE00E94A55B66E27EE083E79EE024
:10F4D0000E94D45A83E79EE00E94A25B64EF71E031
:10F4E00080E090E00E94965DA8960FB6F894DEBF8B
:10F4F0000FBECDBFDF91CF911F9108950895CF9298
:10F50000DF92EF92FF920F931F93CF93DF93EC0163
:10F510006A017B01E889F98982E080834115514EB7
:10F5200061057105B1F060E079E08DE390E0A7013D
:10F5300096010E946C8B89019A01015011092109E1
:10F5400031093695279517950795980101151041B2
:10F55000A8F0E889F989108260E874E88EE190E00B
:10F56000A70196010E946C8BDA01C9010197A109DC
:10F57000B109B695A795979587959C01EC85FD8572
:10F580003083EE85FF852083188EEC89FD8986E027
:10F590008083EA89FB89808180618083EA89FB8995
:10F5A000808188608083EA89FB898081806880838C
:10F5B000EA89FB8980818F7D8083DF91CF911F91C4
:10F5C0000F91FF90EF90DF90CF900895CF92DF9250
:10F5D000EF92FF920F931F93E82FF92F05C0015070
:10F5E00011092109310961F1908196239417B9F32A
:10F5F00005C0015011092109310911F190819623AB
:10F600009413F7CFC12CD12CE12CF12C0AC08FEF31
:10F61000C81AD80AE80AF80A0C151D052E053F0578
:10F6200079F080818623841791F36C2D7D2D8E2DAA
:10F630009F2D1F910F91FF90EF90DF90CF90089535
:10F6400060E070E080E090E01F910F91FF90EF90FC
:10F65000DF90CF9008958F929F92AF92BF92CF92FA
:10F66000DF92EF92FF9210923C0D10923B0D88EECC
:10F6700093E0A0E0B0E080933D0D90933E0DA09309
:10F680003F0DB093400D22EF34E030933A0D2093BC
:10F69000390D45E351E05093460D4093450D44E349
:10F6A00051E05093480D4093470D40E351E0509393
:10F6B0004A0D4093490D41E351E050934C0D409366
:10F6C0004B0D42E351E050934E0D40934D0D46E3F8
:10F6D00051E05093500D40934F0D1092520D1092E7
:10F6E000530D1092540D1092550D1092D90D109289
:10F6F000D80D8093DA0D9093DB0DA093DC0DB093C1
:10F70000DD0D3093D70D2093D60D45ED50E050938D
:10F71000E30D4093E20D44ED50E05093E50D40932E
:10F72000E40D40ED50E05093E70D4093E60D41EDC0
:10F7300050E05093E90D4093E80D42ED50E05093B6
:10F74000EB0D4093EA0D46ED50E05093ED0D4093E4
:10F75000EC0D1092EF0D1092F00D1092F10D109231
:10F76000F20D1092760E1092750E8093770E909394
:10F77000780EA093790EB0937A0E3093740E209386
:10F78000730E25EC30E03093800E20937F0E24EC36
:10F7900030E03093820E2093810E20EC30E03093E5
:10F7A000840E2093830E21EC30E03093860E20935C
:10F7B000850E22EC30E03093880E2093870E26ECE5
:10F7C00030E030938A0E2093890E10928C0E1092A6
:10F7D0008D0E10928E0E10928F0E1092130F1092AB
:10F7E000120F8093140F9093150FA093160FB093E0
:10F7F000170F84E095E09093110F8093100F1092F3
:10F8000008111092071180E295E090930611809301
:10F8100005111092091184E180930D1184E0809309
:10F820000E1110920F1188E08093101160E27AE0BF
:10F830008FEF90E10E94AB5A66E27AE089EF90E1A7
:10F840000E94AB5A88E18093F61081E18093F71013
:10F8500080E18093F81061E088E10E94355D61E00D
:10F860008091F6100E94065D60E08091F7100E9482
:10F87000355D60E08091F8100E94355D61E0809117
:10F88000F7100E94065D61E08091F8100E94065D0D
:10F8900061E08091F6100E94065D1092891010922E
:10F8A0008D1010928C1010928E1086E195E090933E
:10F8B00088108093871080E090E0FC01E957FF4EAC
:10F8C000148E10A2178E11A206968C339105A9F7FB
:10F8D0008AE592E09093EA108093E91086E592E041
:10F8E0009093EC108093EB1084E08093ED10809364
:10F8F000EE108EE592E09093E8108093E7108AE096
:10F9000090E09093F0108093EF1084EF91E090934B
:10F91000F2108093F1101092F5101092F4101092E2
:10F92000E3101092E4101092E5101092E61010927D
:10F93000F31081E0809373101092741083EC9BEAB3
:10F94000A6E7BBE38093751090937610A093771091
:10F95000B093781088ED9BE6A6E7BBE3809379101F
:10F9600090937A10A0937B10B0937C1082EF94EE6A
:10F97000A4E6BBE380937D1090937E10A0937F104C
:10F98000B0938010209154028091520290915302C2
:10F9900080936610209367109927FC01EB53F54F75
:10F9A000E491E0936810FC01E158F54FE491E09395
:10F9B000691080E89EE3A0E0B0E080936E10909321
:10F9C0006F10A0937010B09371106CEF7AE08BE51C
:10F9D00090E10E94AB5A8091500290915102909315
:10F9E0005A108093591080904C0290904D02A09034
:10F9F0004E02B0904F02209148023091490240914E
:10FA00004A0250914B02C501B4010E949D8B6B01CB
:10FA10007C0160935510709356108093571090930B
:10FA20005810609144027091450280914602909175
:10FA300047026093491070934A1080934B10909343
:10FA40004C1080924D1090924E10A0924F10B09298
:10FA50005010209140023091410240914202509159
:10FA600043020E949D8B9B01AC01C701B6010E941D
:10FA7000648C609351107093521080935310909344
:10FA8000541086E495E090933110809330108FEFFE
:10FA90009FEFDC018093451090934610A093471090
:10FAA000B09348106CEF7AE083E190E10E94AB5A8A
:10FAB0006CEF7AE08DE090E10E94AB5A6CEF7AE057
:10FAC00087E090E10E94AB5A6CEF7AE081E090E130
:10FAD0000E94AB5A6CEF7AE08BEF9FE00E94AB5A2A
:10FAE0006CEF7AE085EF9FE00E94AB5A6CEF7AE012
:10FAF0008FEE9FE00E94AB5A87E080931D0F10921B
:10FB00001F0FFF90EF90DF90CF90BF90AF909F902E
:10FB10008F900895CF93DF93CDB7DEB72C970FB6B4
:10FB2000F894DEBF0FBECDBF789484B5826084BDEB
:10FB300084B5816084BD85B5826085BD85B58160F1
:10FB400085BD80916E00816080936E00109281006F
:10FB5000809181008260809381008091810081602A
:10FB600080938100809180008160809380008091EB
:10FB7000B10084608093B1008091B0008160809377
:10FB8000B0008091910082608093910080919100FB
:10FB900081608093910080919000816080939000BB
:10FBA0008091A10082608093A1008091A10081607A
:10FBB0008093A1008091A00081608093A00080913B
:10FBC00021018260809321018091210181608093D5
:10FBD00021018091200181608093200180917A0031
:10FBE000846080937A0080917A00826080937A00AA
:10FBF00080917A00816080937A0080917A00806899
:10FC000080937A001092C10061E089E10E94355D25
:10FC100061E089E10E94065D0E94474262E47AE069
:10FC200083E79EE00E94A55B67E2C62ED12CE12C03
:10FC3000F12C00E010E08C2D0E9422410E94C04077
:10FC4000811127C06EE47AE083E79EE00E94C55BE5
:10FC500020E1B701A60183E79EE00E940D5B83E7E8
:10FC60009EE00E94A25BC09209116AE67AE083E7F7
:10FC70009EE00E94C55B20E1B701A60183E79EE0FC
:10FC80000E940D5B83E79EE00E94A25B0F5F1F4F07
:10FC900013C0843089F464E87AE083E79EE00E9430
:10FCA000C55B20E1B701A60183E79EE00E940D5BE2
:10FCB00083E79EE00E94A25B8FEFC81AD80AE80A89
:10FCC000F80AE0E4CE16D104E104F10409F0B3CF60
:10FCD000012B19F46FE97AE002C065EB7AE083E763
:10FCE0009EE00E94A55B0E94A76280E40E942C41D6
:10FCF0000EEA12E0F80161918F0185E091E10E9426
:10FD0000AC4DF2E0063B1F07A9F70E94216D0E944F
:10FD100044548EED93E090934911809348110E94D2
:10FD20002A8B80939B0C8FED93E00E942A8B80930B
:10FD30009C0C80919B0C90919C0C1816190654F405
:10FD40001092AD02019731F410929C0C10929B0C12
:10FD50000E94AA4468ED7BE0CE0101960E949B5A66
:10FD60004AE050E06FEF7FEFCE0101960E94B66E41
:10FD7000CE0101960E94E15940E052EC61E070E052
:10FD800083E79EE0BCDB8091AD02882331F068EE12
:10FD900073E080E090E00E94965D83E79EE00E9421
:10FDA0004257F82E82E7F81609F451C11092491112
:10FDB0001092481151E2C52E5CE0D52E00E010E013
:10FDC000C8010E942A8BF60181936F010F5F1F4FBC
:10FDD0000A371105A9F78091210C9091220CA0916E
:10FDE000230CB091240C85369105A105B1050CF4C6
:10FDF0002EC18093A9029093AA02A093AB02B09364
:10FE0000AC028091250C9091260CA091270CB0910A
:10FE1000280C8093A5029093A602A093A702B0930A
:10FE2000A8028091290C90912A0CA0912B0CB091E2
:10FE30002C0C8093A1029093A202A093A302B093F2
:10FE4000A4026DE37CE0CE0101960E94AB5ABE0194
:10FE50006F5F7F4F8FEF90E10E94A859CE0101960E
:10FE60000E94E15980912D0C90912E0CA0912F0CA5
:10FE7000B091300C80939D0290939E02A0939F02BC
:10FE8000B093A0028091310C9091320CA091330C70
:10FE9000B091340C8093990290939A02A0939B02A4
:10FEA000B0939C028091350C9091360CA091370C48
:10FEB000B091380C8093950290939602A09397028C
:10FEC000B09398028091390C90913A0CA0913B0C20
:10FED000B0913C0C8093910290939202A093930274
:10FEE000B09394028091450C9091460CA091470CE0
:10FEF000B091480C80934C0290934D02A0934E0217
:10FF0000B0934F028091490C90914A0CA0914B0CF8
:10FF1000B0914C0C8093480290934902A0934A02FE
:10FF2000B0934B0280914D0C90914E0CA0914F0CD0
:10FF3000B091500C8093440290934502A0934602E6
:10FF4000B09347028091510C9091520CA091530CA8
:10FF5000B091540C8093400290934102A0934202CE
:10FF6000B09343028091550C9091560CA091570C80
:10FF7000B091580C80938D0290938E02A0938F02C3
:10FF8000B093900280906B0C90906C0CA0906D0CD4
:10FF9000B0906E0CA5019401C501B4010E94A38E1E
:10FFA000811108C08092890290928A02A0928B02ED
:10FFB000B0928C026091970C7091980C072E000CF7
:10FFC000880B990B0E94148A9B01AC010E94A38E9E
:10FFD000882321F01092980C1092970C0091990CA4
:10FFE00010919A0CB801012E000C880B990B0E94FD
:10FFF000148A9B01AC010E94A38E811107C01016C8
:020000021000EC
:10000000110624F4109355020093540200E010E00E
:10001000F801E159F34F80809180A280B380A5015F
:100020009401C501B4010E94A38E811107C0F8019B
:10003000E05EFE4E80829182A282B3820C5F1F4FEF
:100040000832110529F781E090E00E9493554EE8AF
:10005000E42EEF0CF1E0FE1570F48091210C9091EC
:10006000220CA091230CB091240C85369105A1059A
:10007000B1050CF05EC18091A9029091AA02A091F5
:10008000AB02B091AC028093210C9093220CA09310
:10009000230CB093240C8091A5029091A602A0910C
:1000A000A702B091A8028093250C9093260CA093F0
:1000B000270CB093280C8091A1029091A202A091EC
:1000C000A302B091A4028093290C90932A0CA093D0
:1000D0002B0CB0932C0C82E7F81220C08DE39CE02F
:1000E000892BE1F000910311109104110115110504
:1000F00019F410923D0C12C00730110510F007E002
:1001000010E06091FF1070910011A8018DE39CE058
:100110000E946491F801E35CF34F108280919D028C
:1001200090919E02A0919F02B091A00280932D0C0D
:1001300090932E0CA0932F0CB093300C80919902C9
:1001400090919A02A0919B02B0919C028093310CF5
:100150009093320CA093330CB093340C80919502A1
:1001600090919602A0919702B09198028093350CDD
:100170009093360CA093370CB093380C8091910279
:1001800090919202A0919302B09194028093390CC5
:1001900090933A0CA0933B0CB0933C0C80914C0292
:1001A00090914D02A0914E02B0914F028093450C68
:1001B0009093460CA093470CB093480C8091480252
:1001C00090914902A0914A02B0914B028093490C50
:1001D00090934A0CA0934B0CB0934C0C809144022A
:1001E00090914502A0914602B091470280934D0C38
:1001F00090934E0CA0934F0CB093500C8091400202
:1002000090914102A0914202B09143028093510C1F
:100210009093520CA093530CB093540C80918D0288
:1002200090918E02A0918F02B09190028093550C14
:100230009093560CA093570CB093580C8091890260
:1002400090918A02A0918B02B0918C0280936B0CEA
:1002500090936C0CA0936D0CB0936E0C8091540233
:100260009091550290939A0C8093990CE0E2F1E101
:10027000AFE6BCE041915191619171914D935D93D5
:100280006D937D9381E1E834F807A1F762EC7BE0A0
:10029000CE0101960E949B5ACE0101960E94546F96
:1002A000CE0101960E94E15927E7C22E22E0D22E0C
:1002B00039E5A32E3CE0B32E00E010E080917702F8
:1002C00090917802801791074CF1F601808191811D
:1002D000F501819391935F0180911F118823C1F0F3
:1002E0006FEB7AE083E79EE00E94C55B4AE050E056
:1002F000B80183E79EE00E949C5B6CEB7AE083E7A9
:100300009EE00E94C55BF601808191810E948B5F17
:100310000F5F1F4FF2E0CF0ED11CD0CF81E08E15C2
:1003200040F0109249111092481180E090E00E9434
:10033000D1448091970C9091980C892B39F440E826
:1003400055E260E070E089E39DE0D9D88091970C98
:100350009091980C019739F440E052EC61E070E024
:1003600089E39DE0CCD864E670E080E090E00E94F4
:10037000965D64E670E080E090E00E94965DF894FF
:1003800082E08093B0008093B10094E69093B30034
:100390001092B20080937000789480931C0F10929A
:1003A000200F80911D0F60E00E94355D61EC7AE0C6
:1003B000CE0101960E94AB5A4AE050E06FEF7FEF0A
:1003C000CE0101960E94B66ECE0101960E94E159BF
:1003D0008091970C9091980C892B09F567E479E04E
:1003E000CE0107960E94AB5A6FEF70E1CE010796DF
:1003F0000E943359BC01CE0101960E94A35A4AE0E3
:1004000050E06FEF7FEFCE0101960E94856DCE0127
:1004100001960E94E159CE0107960E94E159809110
:10042000970C9091980C019709F56BE479E0CE0157
:1004300007960E94AB5A6FEF70E1CE0107960E94BB
:100440003359BC01CE0101960E94A35A4AE050E004
:100450006FEF7FEFCE0101960E94856DCE01019670
:100460000E94E159CE0107960E94E1596FEB7AE0B4
:10047000CE0107960E94AB5A6FEF70E1CE0107964E
:100480000E94335961ED7AE00E941C59BC01CE01F3
:1004900001960E94A35ACE0101960E94FD75CE01DD
:1004A00001960E94E159CE0107960E94E15964E647
:1004B00070E080E090E00E94965D2091540280916F
:1004C00052029091530280936610209367109C0112
:1004D0003327F901EB53F54FE491E0936810F901EC
:1004E000E158F54FE491E093691062E00E94355DB8
:1004F00080E398EFAFEFBFEF80936A1090936B109B
:10050000A0936C10B0936D100E94474264E670E0B7
:1005100080E090E00E94965D83E20E94224181E0AB
:1005200090E00E941D410E94C04083E090E09093C3
:100530001E1180931D118CE40E9483604B015C01AD
:1005400062E370E080E090E00E94965DA501940176
:10055000C501B4010E94A38E882309F47AC086E6FF
:100560000E9483604B015C0162E370E080E090E0F8
:100570000E94965DA5019401C501B4010E94A38E5D
:10058000882309F466C081E090E090931E11809367
:100590001D1140E052EC61E070E086ED9DE00E94AC
:1005A0007F7A64E670E080E090E00E94965D86EDE0
:1005B0009DE00E94BC5C40E052EC61E070E086EDA2
:1005C0009DE00E947F7A8CED95E0A0E0B0E0809302
:1005D000DA0D9093DB0DA093DC0DB093DD0D64E696
:1005E00070E080E090E00E94965D92E0C92ED12CF0
:1005F000E12C65E070E080E090E00E94965D00E014
:1006000010E0812C912C5401E11053C186ED9DE046
:100610000E946457892B39F4F5E18F169104A104E7
:10062000B1040CF046C1033011050CF488C141C17E
:10063000EE2009F44CC169EA7BE0CE0101960E94EC
:100640009B5ACE0101960E94546FCE0101960E94E2
:10065000E15980911D1190911E11039771F46AE781
:100660007BE0CE0101960E949B5ACE0101960E942A
:10067000546FCE0101960E94E15983E080931910D6
:100680000E94474280ED0E944F45853509F082C1A6
:100690008AEA0E94724590931B1080931A108CEA8C
:1006A0000E94724590931D1080931C108EEA0E9448
:1006B000724590931F1080931E1080EB0E9472452C
:1006C00090932B1080932A1082EB0E947245909396
:1006D0002D1080932C1084EB0E94724590932F1064
:1006E00080932E1086EB0E94724590932110809388
:1006F000201088EB0E947245909323108093221063
:100700008AEB0E94724590932510809324108CEB05
:100710000E94724590932710809326108EEB0E94C2
:100720007245909329108093281061E47BE08BEF51
:100730009FE00E9458590E94B44576D60E94FD8CD5
:1007400073D620E030E048EC52E40E94648CAB01A8
:10075000BC0122E0CE0107960E94155ABE01695FD6
:100760007F4FCE0101960E94A35A6CE077E0CE0144
:1007700001960E941C59BC018BEF9FE00E945259C8
:10078000CE0101960E94E159CE0107960E94E159DF
:100790006BEF7FE0CE0101960E94A35ACE01019635
:1007A0000E94546FCE0101960E94E1596BE27BE0FA
:1007B0008BEF9FE00E9458596091A9027091AA02A4
:1007C0008091AB029091AC022FD620E030E048EC53
:1007D00052E40E94648CAB01BC0122E0CE0107967A
:1007E0000E94155ABE01695F7F4FCE0101960E949B
:1007F000A35A6CE077E0CE0101960E941C59BC011F
:100800008BEF9FE00E945259CE0101960E94E15960
:10081000CE0107960E94E1596BEF7FE0CE01019671
:100820000E94A35ACE0101960E94546FCE010196F8
:100830000E94E15981E6F81205C081E00E94013B67
:1008400081E011C083E79EE00E944257182F64E6C2
:1008500070E080E090E00E94965D113671F380E0D8
:100860000E94013B80E00E947E7964E670E080E0B7
:1008700090E00E94965D1091AD02112331F068EE78
:1008800073E080E090E00E94965D65E875E087E0A7
:1008900090E10E947E5982E090E090931C11809339
:1008A0001B1111110E949B730E94A0070E941358F4
:1008B000FBCF64E670E080E090E00E94965DCA9411
:1008C000CD2809F4B5CECC24C394D12C92CE10926D
:1008D0001E1110921D1186ED9DE00E94BC5C64E625
:1008E00070E080E090E00E94965D40E855E260E0B4
:1008F00070E086ED9DE00E947F7A86ED9DE00E948B
:100900006457892B09F4A5CE6FE87BE0CE010196F0
:100910000E949B5ACE0101960E94546FCE0101960F
:100920000E94E15982E090E090931E1180931D1186
:1009300064E670E080E090E00E94965D8ACE86EDED
:100940009DE00E946457892B69F086ED9DE00E942E
:100950004257E1E0F0E0EC0FFD1FE00FF11F808354
:100960000F5F1F4F65E070E080E090E00E94965DB1
:10097000023011054CF089818B3B31F4EE24E39475
:100980008A818A3A09F0E12CEFEF8E1A9E0AAE0AAC
:10099000BE0A3ACE64E57BE0CE0101960E949B5AE6
:1009A000CE0101960E94FD75CE0101960E94E1598B
:1009B000109276025ACF8FEE9FE00E94E15985EFA8
:1009C0009FE00E94E1598BEF9FE00E94E15981E096
:1009D00090E10E94E15987E090E10E94E1598DE0A9
:1009E00090E10E94E15983E190E10E94E1598BE599
:1009F00090E10E94E15989EF90E10E94E1598FEF67
:100A000090E10C94E159CF92DF92EF92FF921F9305
:100A1000CF93DF93182FCAE0D0E0C12CD12C760100
:100A2000812F0E94715DBC01990F880B990BFCD43A
:100A30009B01AC01C701B60181D66B017C0162E369
:100A400070E080E090E00E94965D219749F720E0F9
:100A500030E040E251E4C701B60136D720E030E093
:100A600040EA50E440D520E030E040E85AE33BD58E
:100A7000DF91CF911F91FF90EF90DF90CF9008957D
:100A8000EF920F931F93CF93DF93E80147FD02C0CE
:100A900034E001C034E1E42F440FFF0BF7FF03C043
:100AA000F195E195F109E32E022F2E2FAE01BBD077
:100AB000CE01DF91CF911F910F91EF90089566279E
:100AC00077273EC21F93FC0199278827BC01E89431
:100AD00011911032E9F3193010F01E30C8F31B32B7
:100AE00049F01D3241F4689405C04ED0610F711D6C
:100AF000811D911D119110531A30B8F33EF4909559
:100B00008095709561957F4F8F4F9F4F1F910895EE
:100B1000FB01DC0105900D920020E1F70895FC0136
:100B200005900020E9F7809590958E0F9F1F0895FE
:100B30004532510518F4423008F004C0FB01108220
:100B4000CB010895BB274A3031F4992322F4BDE24A
:100B5000909581959F4F4FC02532310518F4223072
:100B600008F004C0FA011082CA010895BB272A3098
:100B700051F4992342F4BDE290958095709561956A
:100B80007F4F8F4F9F4F16C0592F482F372F262F3B
:100B9000660F771F881F991F660F771F881F991F81
:100BA000620F731F841F951F660F771F881F991F81
:100BB0000895BB27FA01A62F6217710581059105DB
:100BC000330B30FB66F0AA27660F771F881F991F2B
:100BD000AA1FA21710F0A21B63953850A9F7A05DB9
:100BE000AA3308F0A95DA19336F7B111B193108231
:100BF000CA0104C4BB27FB015527AA27880F991FE8
:100C0000AA1FA41710F0A41B83955051B9F7A05D3B
:100C1000AA3308F0A95DA193009779F7B111B193B8
:100C20001192CB01EBC34F925F926F927F929F9292
:100C3000AF92BF92CF92DF92EF92FF920F931F93EA
:100C4000CF93DF93CDB7DEB729970FB6F894DEBF09
:100C50000FBECDBF6A01122FB02E2BE3201720F05C
:100C6000FF24F394F00E02C0BCE3FB2E0F2D27E00F
:100C7000AE014F5F5F4FCAD2AC018981982F997046
:100C8000913031F0E1FC06C0E0FE06C090E205C004
:100C90009DE203C09BE201C090E0EE2DE07183FF76
:100CA0003CC0911102C083E001C084E0811718F4B8
:100CB000212F281B01C020E0E1110BC0F601822F7B
:100CC00030E2882319F031938150FBCFC20ED11C42
:100CD00020E0992329F0D6019C93F60131966F010B
:100CE000C6010396E2FE0AC03EE4D6013C9341E40D
:100CF00011964C93119712963C9306C03EE6F6016E
:100D0000308341E641833283FC01322F40E23323BA
:100D100009F442C041933150FACF82FF44C091118F
:100D200002C083E001C084E0811718F4212F281B42
:100D300001C020E0E1110BC0F601822F30E28823D0
:100D400019F031938150FBCFC20ED11C20E09923C2
:100D500029F0D6019C93F60131966F01C6010396E6
:100D6000E2FE0BC039E4D6013C933EE411963C937D
:100D7000119736E412963C9307C039E6F6013083AA
:100D80003EE6318336E63283FC01322F40E23323E4
:100D900019F041933150FBCFFC01E20FF11D10829D
:100DA0008EEF9FEFB7C0F1E0911101C0F0E06F2F1F
:100DB00070E01416150624F49A012F5F3F4F02C00D
:100DC00021E030E0260F371FBB2029F06B2D70E0AB
:100DD0006F5F7F4F02C060E070E0260F371F612F0A
:100DE00070E0261737071CF4121B212F01C020E0EA
:100DF0003E2D387159F4D601322F60E2332319F0B9
:100E00006D933150FBCFC20ED11C20E0FF2331F097
:100E1000D6019C93B6016F5F7F4F6B01E1110BC050
:100E2000F601922F30E3992319F031939150FBCFC3
:100E3000C20ED11C20E09F2D940F3A81782F707143
:100E4000A72E84FF03C0313309F49150191624F4FE
:100E5000993018F098E001C091E0E42F852F57FFFA
:100E600002C0E0E080E06E2F782FE0E0F0E0AEE23C
:100E70009A2E3A01691A71082A01461A570A0B2D4F
:100E800010E01195019511096F3F8FEF780729F454
:100E9000D6019C92C60101966C014617570784F053
:100EA000661677066CF47F01E40CF51CA1E0B0E057
:100EB000AC0FBD1FEA0EFB1ED7011196BC9002C0FD
:100EC00090E3B92E615071093196C60101967C01FB
:100ED0006017710724F0D601BC926C01D5CF64175E
:100EE000750741F4363320F4353321F4A11002C0E4
:100EF00081E3B82EF601B082F701822F90E28823B9
:100F000019F091938150FBCFF701E20FF11D108290
:100F100080E090E029960FB6F894DEBF0FBECDBFFB
:100F2000DF91CF911F910F91FF90EF90DF90CF90C5
:100F3000BF90AF909F907F906F905F904F9008957B
:100F40006F927F928F929F92AF92BF92CF92DF92D9
:100F5000EF92FF920F931F93CF93DF93EC017B01EE
:100F60006115710519F0DB018D939C938E010F5F64
:100F70001F4F7880872D90E021D2892B11F0E80156
:100F8000F5CFBDE27B1205C00F5F1F4F7980C1E036
:100F900008C0EBE27E1204C08E010E5F1F4F798005
:100FA000C0E06801F1E0CF1AD10843E050E06AE206
:100FB00072E0C6010BD2892BE9F4680122E0C20E6F
:100FC000D11C45E050E065E272E0C601FFD1892BFB
:100FD00021F4680187E0C80ED11CE114F10419F076
:100FE000D701CD92DC92C111F9C060E070E080E8D9
:100FF0009FE7FDC043E050E062E272E0C601E6D147
:10100000892B51F4E114F10409F4EDC00E5F1F4F78
:10101000F70111830083E7C0680160E070E0CB0155
:1010200000E010E0F601D0EDD70DDA3050F52C2FAE
:101030002260622E2C2F2870C2FF05C0211127C00C
:101040000F5F1F4F24C0222311F001501109A5E0AA
:10105000B0E09B01AC0130D34B015C01880C991CC2
:10106000AA1CBB1CC501B4016D0F711D811D911D12
:101070006839A9E97A078A07A9E19A0740F0C660AA
:1010800005C0DE3F51F4C3FD44C0C8606C2EBFEF05
:10109000CB1ADB0A7080C62DC5CF2D2F2F7D2531B1
:1010A000C1F540814D3211F4C06106C04B3221F0D0
:1010B000319621E030E006C03296D60111964C916F
:1010C00022E030E0A0EDA40FAA3018F0E21BF30BF1
:1010D00020C040E050E04038BCE05B075CF49A017F
:1010E000220F331F220F331F420F531F440F551F70
:1010F0004A0F511D3196DF0111972C91A0EDA20FDF
:10110000AA3048F3C4FF03C0519541955109040F1B
:10111000151FC1FF07C0E114F10421F03197D70179
:10112000ED93FC937FD1C370C33019F06B017C0148
:1011300006C06B017C01F7FAF094F7F8F09420E018
:1011400030E0A901C701B60169D1882309F443C081
:1011500017FF06C0119501951109C1E4D2E002C044
:10116000C9E5D2E05E01B8E1AB1AB1084601BE2D77
:10117000AF2D90E2E92EF12C0E151F057CF0FE013B
:101180002591359145915491B4018B2F9A2FABD174
:101190004B01B82FA92F0E191F09EECF2497F594F4
:1011A000E794CA15DB0541F76401EB2EFA2E8E2D6C
:1011B000880F8F2D881F8F3F41F020E030E0A9017C
:1011C000C701B6012BD1811106C082E290E0909355
:1011D000B7118093B611C701B60109C060E070E095
:1011E00080E89FEF04C060E070E080EC9FE7DF9153
:1011F000CF911F910F91FF90EF90DF90CF90BF9014
:10120000AF909F908F907F906F900895283008F056
:1012100027E03327DA01990F311D87FD9160009691
:101220006105710539F432602E5F3D9330E32A95F4
:10123000E1F708959F3F30F080387105610509F0AE
:101240003C5F3C5F3D93913008F08068911DDF93D7
:10125000CF931F930F93FF92EF92192F987F96953C
:10126000E92F96959695E90FFF27E954FD4F9927A9
:101270003327EE24FF24A701E70105900894079483
:1012800028F4360FE71EF81E491F511D660F771F01
:10129000881F991F0694A1F70590079428F4E70E7C
:1012A000F81E491F561FC11D770F881F991F661F03
:1012B0000694A1F70590079428F4F80E491F561FCD
:1012C000C71FD11D880F991F661F771F0694A1F7AE
:1012D0000590079420F4490F561FC71FD81F990F78
:1012E000661F771F881F0694A9F7849110951770C1
:1012F00041F0D695C79557954795F794E7941A9579
:10130000C1F7EDE5F2E0689415901591359165917E
:10131000959105907FE27395E118F10A430B560B06
:10132000C90BD009C0F7E10CF11E431F561FC91F9E
:10133000D01D7EF4703311F48A95E6CFE894015005
:1013400030F0080F0AF40027021708F4202F239525
:10135000022F7A3328F079E37D932A95E9F710C0BC
:101360007D932A9589F606949795679537951795F5
:101370001794E118F10A430B560BC90BD00998F0EA
:1013800023957E9173957A3308F070E37C93201354
:10139000B8F77E9170617D9330F0839571E37D9312
:1013A00070E32A95E1F71124EF90FF900F911F91C0
:1013B000CF91DF91992787FD909508959111F6C0FF
:1013C000803219F089508550D0F70895FB01DC0177
:1013D0004150504088F08D9181341CF08B350CF4D5
:1013E000805E659161341CF06B350CF4605E861B89
:1013F000611171F3990B0895881BFCCFDC01FC018E
:10140000672F71917723E1F7329704C07C916D9338
:1014100070836291AE17BF07C8F3089540D008F4F7
:1014200081E00895E89409C097FB3EF4909580957B
:10143000709561957F4F8F4F9F4F9923A9F0F92F9A
:1014400096E9BB279395F695879577956795B79518
:10145000F111F8CFFAF4BB0F11F460FF1BC06F5FFE
:101460007F4F8F4F9F4F16C0882311F096E911C010
:10147000772321F09EE8872F762F05C0662371F031
:1014800096E8862F70E060E02AF09A95660F771F45
:10149000881FDAF7880F9695879597F90895990F21
:1014A0000008550FAA0BE0E8FEEF16161706E8072E
:1014B000F907C0F012161306E407F50798F0621B4F
:1014C000730B840B950B39F40A2661F0232B242B24
:1014D000252B21F408950A2609F4A140A6958FEF43
:1014E000811D811D08950BD07BC06CD028F071D078
:1014F00018F0952309F05DC062C01124A5C081D009
:10150000A0F3959FD1F3950F50E0551F629FF00116
:10151000729FBB27F00DB11D639FAA27F00DB11D6F
:10152000AA1F649F6627B00DA11D661F829F2227F8
:10153000B00DA11D621F739FB00DA11D621F839F7F
:10154000A00D611D221F749F3327A00D611D231F55
:10155000849F600D211D822F762F6A2F11249F57A3
:1015600050408AF0E1F088234AF0EE0FFF1FBB1FC6
:10157000661F771F881F91505040A9F79E3F510565
:1015800070F017C061C05F3FECF3983EDCF38695C6
:1015900077956795B795F795E7959F5FC1F7FE2B10
:1015A000880F911D9695879597F908959927882713
:1015B000089597F99F6780E870E060E008959FEFD5
:1015C00080EC089500240A941616170618060906DA
:1015D000089500240A9412161306140605060895A9
:1015E000092E0394000C11F4882352F0BB0F40F431
:1015F000BF2B11F460FF04C06F5F7F4F8F4F9F4F71
:10160000089557FD9058440F551F59F05F3F71F0F2
:101610004795880F97FB991F61F09F3F79F0879559
:101620000895121613061406551FF2CF4695F1DFE2
:1016300008C0161617061806991FF1CF8695710572
:10164000610508940895E894BB2766277727CB01A6
:1016500097F90895F999FECF92BD81BDF89A99271F
:1016600080B50895262FF999FECF1FBA92BD81BD8E
:1016700020BD0FB6F894FA9AF99A0FBE0196089514
:10168000052E97FB16F400940FD057FD05D024D0FB
:1016900007FC02D046F408C050954095309521953E
:1016A0003F4F4F4F5F4F089590958095709561958E
:1016B0007F4F8F4F9F4F089531D0A59F900DB49FBE
:1016C000900DA49F800D911D11240895B7FFF4CFB4
:1016D000F3DF821B930B0895A1E21A2EAA1BBB1BFA
:1016E000FD010DC0AA1FBB1FEE1FFF1FA217B307EE
:1016F000E407F50720F0A21BB30BE40BF50B661F04
:10170000771F881F991F1A9469F7609570958095C7
:1017100090959B01AC01BD01CF010895A29FB0013E
:10172000B39FC001A39F700D811D1124911DB29F15
:10173000700D811D1124911D08955058BB27AA27B3
:101740000ED04ECF3FDF30F044DF20F031F49F3F2A
:1017500011F41EF434CF0EF4E095E7FB2ACFE92F05
:1017600050DF80F3BA17620773078407950718F0F4
:1017700071F49EF568CF0EF4E0950B2EBA2FA02DD4
:101780000B01B90190010C01CA01A0011124FF272E
:10179000591B99F0593F50F4503E68F11A16F04029
:1017A000A22F232F342F4427585FF3CF4695379528
:1017B0002795A795F0405395C9F77EF41F16BA0BED
:1017C000620B730B840BBAF09150A1F0FF0FBB1F9B
:1017D000661F771F881FC2F70EC0BA0F621F731FE4
:1017E000841F48F4879577956795B795F7959E3F41
:1017F00008F0B3CF9395880F08F09927EE0F9795CF
:1018000087950895DFDE58F080E891E009F49EEFB7
:10181000E0DE28F040E851E059F45EEF09C0CFCE99
:1018200012CFE92FE078EDDE68F3092E052AC1F327
:10183000261737074807590738F00E2E07F8E02516
:1018400069F0E025E0640AC0EF6307F8009407FA46
:10185000DB01B9019D01DC01CA01AD01EF9343D069
:10186000BFDE0AD05F91552331F02BED3FE049E414
:1018700050FD49EC63CF0895DF93DD27B92FBF7783
:1018800040E85FE31616170648075B0710F4D92FE8
:101890000ED19F938F937F936F9352D2E2E7F1E043
:1018A000DDD09EDE2F913F914F915F9128DEDD23A9
:1018B00049F09058A2EA2AED3FE049EC5FE3D07886
:1018C0005D274DDFDF918CCE0CD08ACE82DE40F0DA
:1018D00079DE30F021F45F3F19F06BCE5111B4CEB8
:1018E0006ECE8FDE98F39923C9F35523B1F3951B80
:1018F000550BBB27AA2762177307840738F09F5F31
:101900005F4F220F331F441FAA1FA9F333D00E2E9F
:101910003AF0E0E830D091505040E695001CCAF70C
:1019200029D0FE2F27D0660F771F881FBB1F2617D1
:1019300037074807AB07B0E809F0BB0B802DBF01A4
:10194000FF2793585F4F2AF09E3F510568F031CE34
:101950007BCE5F3FECF3983EDCF3869577956795F9
:10196000B795F7959F5FC9F7880F911D9695879555
:1019700097F90895E1E0660F771F881FBB1F621774
:1019800073078407BA0720F0621B730B840BBA0B32
:10199000EE1F88F7E095089519F40EF00ACE53CEA5
:1019A0000ECE37DEC8F39638C0F707F80F92E894EA
:1019B0002BE33AEA48EB5FE7A4DD0F920F920F9218
:1019C0004DB75EB70F92FBD0EFE9F1E047D04F91F2
:1019D0005F91EF91FF91E595EE1FFF1F49F0FE57D4
:1019E000E0684427EE0F441FFA95E1F74195550B47
:1019F00067D00F9007FE5BC0089504D06894B111C2
:101A000023CE089506DE88F09F5790F0B92F9927CE
:101A1000B751A0F0D1F0660F771F881F991F1AF0F9
:101A2000BA95C9F712C0B13081F00DDEB1E008956A
:101A30000ACE672F782F8827B85F39F0B93FCCF3EB
:101A4000869577956795B395D9F73EF490958095EF
:101A5000709561957F4F8F4F9F4F0895DF93CF9380
:101A60001F930F93FF92EF92DF927B018C0168949A
:101A700005C0DA2EEF0143DDFE01E894A591259122
:101A8000359145915591AEF3EF0169DEFE01970165
:101A9000A801DA9479F7DF90EF90FF900F911F91F2
:101AA000CF91DF910895FBDC08F48FEF08959B013F
:101AB000AC0160E070E080E89FE306CF7ACD47C1DB
:101AC000A8DDE8F39923D9F3940F511DBBF391508E
:101AD000504094F059F0882332F0660F771F881F2A
:101AE00091505040C1F79E3F510544F7880F911D1A
:101AF0009695879597F908955F3FACF0983E9CF0D6
:101B0000BB27869577956795B79508F4B16093954F
:101B1000C1F7BB0F58F711F460FFE8CF6F5F7F4F3D
:101B20008F4F9F4FE3CF90CD0AD029ED3BE54EED8F
:101B30005EE3D9CC0EF00BC142CD68943ACD69DD9D
:101B4000C8F39923D1F3C6F3DF93CF931F930F9379
:101B5000FF92C92FDD2788232AF02197660F771F70
:101B6000881FDAF720E030E040E85FEB9FE3883938
:101B700020F0803E30F021968F77E0DDE7ECF1E059
:101B800003C0DCDDE4EFF1E069DF8B01BE01EC01B5
:101B9000FB2E6F5771097595771F880B990B44DCE5
:101BA00028E132E741E35FE3AADCAF2D9801AE0103
:101BB000FF900F911F91CF91DF91D1DD11CDFA01EF
:101BC000DC01AA0FBB1F9B01AC01BF5728F42227E1
:101BD0003327442750781FC0B75188F4AB2F002417
:101BE000469537952795011CA395D2F3002069F0FF
:101BF000220F331F441FB395DAF30DD09ECD613011
:101C00007105A0E88A07B94630F49B01AC0166274C
